MPLINK 4.43, Linker
Linker Map File - Created Tue Jul 13 08:17:58 2021

                                 Section Info
                  Section       Type    Address   Location Size(Bytes)
                ---------  ---------  ---------  ---------  ---------
               _entry_scn       code   0x000000    program   0x000006
               HighVector       code   0x000018    program   0x000006
                   .cinit    romdata   0x000200    program   0x000002
     .code_CMSModifV1SD.o       code   0x000202    program   0x0139a6
                     PROG       code   0x013ba8    program   0x000626
         .code_i2c1writ.o       code   0x0141ce    program   0x000080
         .code_i2c1gets.o       code   0x01424e    program   0x000076
         .code_i2c1open.o       code   0x0142c4    program   0x000036
         .code_fxd1616u.o       code   0x0142fa    program   0x00002c
                    .code       code   0x014326    program   0x000020
         .code_fxd0808u.o       code   0x014346    program   0x00001c
         .code_i2c1read.o       code   0x014362    program   0x00001a
             _startup_scn       code   0x01437c    program   0x000018
           .code___init.o       code   0x014394    program   0x000002
      .romdata_fxd1616u.o    romdata   0x014396    program   0x000000
      .idata_i2c1open.o_i    romdata   0x014396    program   0x000000
      .romdata_i2c1open.o    romdata   0x014396    program   0x000000
      .idata_i2c1read.o_i    romdata   0x014396    program   0x000000
      .romdata_i2c1read.o    romdata   0x014396    program   0x000000
      .idata_i2c1writ.o_i    romdata   0x014396    program   0x000000
      .romdata_i2c1writ.o    romdata   0x014396    program   0x000000
        .idata___init.o_i    romdata   0x014396    program   0x000000
        .romdata___init.o    romdata   0x014396    program   0x000000
      .idata_i2c1gets.o_i    romdata   0x014396    program   0x000000
      .romdata_i2c1gets.o    romdata   0x014396    program   0x000000
          .idata_c018.o_i    romdata   0x014396    program   0x000000
  .idata_CMSModifV1SD.o_i    romdata   0x014396    program   0x000000
  .romdata_CMSModifV1SD.o    romdata   0x014396    program   0x000000
             .code_c018.o       code   0x014396    program   0x000000
          .romdata_c018.o    romdata   0x014396    program   0x000000
      .idata_fxd0808u.o_i    romdata   0x014396    program   0x000000
      .romdata_fxd0808u.o    romdata   0x014396    program   0x000000
      .idata_fxd1616u.o_i    romdata   0x014396    program   0x000000
.config_300001_CMSModifV1SD.o    romdata   0x300001    program   0x000001
.config_300002_CMSModifV1SD.o    romdata   0x300002    program   0x000001
.config_300003_CMSModifV1SD.o    romdata   0x300003    program   0x000001
.config_300004_CMSModifV1SD.o    romdata   0x300004    program   0x000001
.config_300005_CMSModifV1SD.o    romdata   0x300005    program   0x000001
.config_300006_CMSModifV1SD.o    romdata   0x300006    program   0x000001
.config_300008_CMSModifV1SD.o    romdata   0x300008    program   0x000001
.config_300009_CMSModifV1SD.o    romdata   0x300009    program   0x000001
.config_30000a_CMSModifV1SD.o    romdata   0x30000a    program   0x000001
.config_30000b_CMSModifV1SD.o    romdata   0x30000b    program   0x000001
.config_30000c_CMSModifV1SD.o    romdata   0x30000c    program   0x000001
.config_30000d_CMSModifV1SD.o    romdata   0x30000d    program   0x000001
                MATH_DATA      udata   0x000000       data   0x000014
                 .tmpdata      udata   0x000014       data   0x00000a
                   udata1      udata   0x000100       data   0x0000fa
        .idata_i2c1gets.o      idata   0x0001fa       data   0x000000
        .udata_i2c1gets.o      udata   0x0001fa       data   0x000000
          .idata___init.o      idata   0x0001fa       data   0x000000
          .udata___init.o      udata   0x0001fa       data   0x000000
        .idata_i2c1writ.o      idata   0x0001fa       data   0x000000
        .udata_i2c1writ.o      udata   0x0001fa       data   0x000000
        .idata_i2c1read.o      idata   0x0001fa       data   0x000000
        .udata_i2c1read.o      udata   0x0001fa       data   0x000000
        .idata_i2c1open.o      idata   0x0001fa       data   0x000000
        .udata_i2c1open.o      udata   0x0001fa       data   0x000000
        .idata_fxd1616u.o      idata   0x0001fa       data   0x000000
        .udata_fxd1616u.o      udata   0x0001fa       data   0x000000
        .idata_fxd0808u.o      idata   0x0001fa       data   0x000000
        .udata_fxd0808u.o      udata   0x0001fa       data   0x000000
    .idata_CMSModifV1SD.o      idata   0x0001fa       data   0x000000
    .udata_CMSModifV1SD.o      udata   0x0001fa       data   0x000000
            .idata_c018.o      idata   0x0001fa       data   0x000000
            .udata_c018.o      udata   0x0001fa       data   0x000000
                   udata2      udata   0x000200       data   0x0000f2
                   udata3      udata   0x000300       data   0x0000f0
                   .stack      udata   0x000e00       data   0x0000e0
                   udata4      udata   0x000f00       data   0x000046
            SFR_UNBANKED0      udata   0x000f62       data   0x00009e



                              Program Memory Usage 
                               Start         End      
                           ---------   ---------      
                            0x000000    0x000005      
                            0x000018    0x00001d      
                            0x000200    0x014395      
                            0x300001    0x300006      
                            0x300008    0x30000d      
            82350 out of 132120 program addresses used, program memory utilization is 62%



                              Symbols - Sorted by Name
                     Name    Address   Location    Storage File                     
                ---------  ---------  ---------  --------- ---------                
              AQUIENVOYER   0x00bd92    program     extern C:\Users\LFRAD\Documents\CMS2Luc\ProjetsNettoyesCMSGit\ProjetCarteMere\project\CMSModifV1SD.c
                  AVERAGE   0x00ee34    program     extern C:\Users\LFRAD\Documents\CMS2Luc\ProjetsNettoyesCMSGit\ProjetCarteMere\project\CMSModifV1SD.c
                      CAN   0x00ed32    program     extern C:\Users\LFRAD\Documents\CMS2Luc\ProjetsNettoyesCMSGit\ProjetCarteMere\project\CMSModifV1SD.c
 CHERCHER_DONNNEES_CABLES   0x0109d8    program     extern C:\Users\LFRAD\Documents\CMS2Luc\ProjetsNettoyesCMSGit\ProjetCarteMere\project\CMSModifV1SD.c
     CONTROLE_CHARGE_BATT   0x00f0d8    program     extern C:\Users\LFRAD\Documents\CMS2Luc\ProjetsNettoyesCMSGit\ProjetCarteMere\project\CMSModifV1SD.c
                    CRC16   0x011aca    program     extern C:\Users\LFRAD\Documents\CMS2Luc\ProjetsNettoyesCMSGit\ProjetCarteMere\project\CMSModifV1SD.c
                CRC_verif   0x0119b8    program     extern C:\Users\LFRAD\Documents\CMS2Luc\ProjetsNettoyesCMSGit\ProjetCarteMere\project\CMSModifV1SD.c
                   D0808S   0x013eb8    program     static E:\MPASM_MPLINK_PIC18_LT_Branch_3_42\pic18-lt\cxx-framework\src\traditional\math\fxd0808s.asm
                D0808SNEG   0x013ec6    program     static E:\MPASM_MPLINK_PIC18_LT_Branch_3_42\pic18-lt\cxx-framework\src\traditional\math\fxd0808s.asm
                 D0808SOK   0x013ec2    program     static E:\MPASM_MPLINK_PIC18_LT_Branch_3_42\pic18-lt\cxx-framework\src\traditional\math\fxd0808s.asm
                  D0808SX   0x013ecc    program     static E:\MPASM_MPLINK_PIC18_LT_Branch_3_42\pic18-lt\cxx-framework\src\traditional\math\fxd0808s.asm
                   D1616S   0x013ef8    program     static E:\MPASM_MPLINK_PIC18_LT_Branch_3_42\pic18-lt\cxx-framework\src\traditional\math\fxd1616s.asm
                D1616SNEG   0x013f06    program     static E:\MPASM_MPLINK_PIC18_LT_Branch_3_42\pic18-lt\cxx-framework\src\traditional\math\fxd1616s.asm
                 D1616SOK   0x013f02    program     static E:\MPASM_MPLINK_PIC18_LT_Branch_3_42\pic18-lt\cxx-framework\src\traditional\math\fxd1616s.asm
                  D1616SX   0x013f18    program     static E:\MPASM_MPLINK_PIC18_LT_Branch_3_42\pic18-lt\cxx-framework\src\traditional\math\fxd1616s.asm
                  DA0808S   0x013eae    program     static E:\MPASM_MPLINK_PIC18_LT_Branch_3_42\pic18-lt\cxx-framework\src\traditional\math\fxd0808s.asm
                  DA1616S   0x013ee8    program     static E:\MPASM_MPLINK_PIC18_LT_Branch_3_42\pic18-lt\cxx-framework\src\traditional\math\fxd1616s.asm
        ECRIRE_EEPROMBYTE   0x00b5f2    program     extern C:\Users\LFRAD\Documents\CMS2Luc\ProjetsNettoyesCMSGit\ProjetCarteMere\project\CMSModifV1SD.c
           ECRIRE_HORLOGE   0x00f7e8    program     extern C:\Users\LFRAD\Documents\CMS2Luc\ProjetsNettoyesCMSGit\ProjetCarteMere\project\CMSModifV1SD.c
               EFFACEMENT   0x00dc58    program     extern C:\Users\LFRAD\Documents\CMS2Luc\ProjetsNettoyesCMSGit\ProjetCarteMere\project\CMSModifV1SD.c
   EFFACER_CAPTEUR_SUR_CM   0x010614    program     extern C:\Users\LFRAD\Documents\CMS2Luc\ProjetsNettoyesCMSGit\ProjetCarteMere\project\CMSModifV1SD.c
            EFFACER_LISTE   0x00f49c    program     extern C:\Users\LFRAD\Documents\CMS2Luc\ProjetsNettoyesCMSGit\ProjetCarteMere\project\CMSModifV1SD.c
        ENVOIE_DES_TRAMES   0x00194c    program     extern C:\Users\LFRAD\Documents\CMS2Luc\ProjetsNettoyesCMSGit\ProjetCarteMere\project\CMSModifV1SD.c
                 FLO0832S   0x013bac    program     extern E:\MPASM_MPLINK_PIC18_LT_Branch_3_42\pic18-lt\cxx-framework\src\traditional\math\cast08FP.asm
                 FLO0832U   0x013ba8    program     extern E:\MPASM_MPLINK_PIC18_LT_Branch_3_42\pic18-lt\cxx-framework\src\traditional\math\cast08FP.asm
                 FLO1632S   0x013bce    program     extern E:\MPASM_MPLINK_PIC18_LT_Branch_3_42\pic18-lt\cxx-framework\src\traditional\math\cast16FP.asm
                 FLO1632U   0x013bca    program     extern E:\MPASM_MPLINK_PIC18_LT_Branch_3_42\pic18-lt\cxx-framework\src\traditional\math\cast16FP.asm
                    FPA32   0x013bf6    program     extern E:\MPASM_MPLINK_PIC18_LT_Branch_3_42\pic18-lt\cxx-framework\src\traditional\math\addFP.asm
                    FPD32   0x013d22    program     extern E:\MPASM_MPLINK_PIC18_LT_Branch_3_42\pic18-lt\cxx-framework\src\traditional\math\divFP.asm
                    FPM32   0x013dc8    program     extern E:\MPASM_MPLINK_PIC18_LT_Branch_3_42\pic18-lt\cxx-framework\src\traditional\math\mulFP.asm
                    FPS32   0x013bf4    program     extern E:\MPASM_MPLINK_PIC18_LT_Branch_3_42\pic18-lt\cxx-framework\src\traditional\math\addFP.asm
                 FXD0808S   0x013ea2    program     extern E:\MPASM_MPLINK_PIC18_LT_Branch_3_42\pic18-lt\cxx-framework\src\traditional\math\fxd0808s.asm
                 FXD0808U   0x014346    program     extern E:\MPASM_MPLINK_PIC18_LT_Branch_3_42\pic18-lt\cxx-framework\src\traditional\math\fxd0808u.c
                 FXD1616S   0x013ed6    program     extern E:\MPASM_MPLINK_PIC18_LT_Branch_3_42\pic18-lt\cxx-framework\src\traditional\math\fxd1616s.asm
                 FXD1616U   0x0142fa    program     extern E:\MPASM_MPLINK_PIC18_LT_Branch_3_42\pic18-lt\cxx-framework\src\traditional\math\fxd1616u.c
                 FXM1616S   0x013f22    program     extern E:\MPASM_MPLINK_PIC18_LT_Branch_3_42\pic18-lt\cxx-framework\src\traditional\math\fxm1616s.asm
                 FXM1616U   0x013f7c    program     extern E:\MPASM_MPLINK_PIC18_LT_Branch_3_42\pic18-lt\cxx-framework\src\traditional\math\fxm1616u.asm
        GROUPE_EN_MEMOIRE   0x00f6a6    program     extern C:\Users\LFRAD\Documents\CMS2Luc\ProjetsNettoyesCMSGit\ProjetCarteMere\project\CMSModifV1SD.c
               HighVector   0x000018    program     extern C:\Users\LFRAD\Documents\CMS2Luc\ProjetsNettoyesCMSGit\ProjetCarteMere\project\CMSModifV1SD.c
       IDENTIF_TYPE_CARTE   0x01108c    program     extern C:\Users\LFRAD\Documents\CMS2Luc\ProjetsNettoyesCMSGit\ProjetCarteMere\project\CMSModifV1SD.c
                  INT3208   0x013fb8    program     extern E:\MPASM_MPLINK_PIC18_LT_Branch_3_42\pic18-lt\cxx-framework\src\traditional\math\castFP08.asm
INTERROGER_TOUT_LES_CAPTEURS   0x00f18a    program     extern C:\Users\LFRAD\Documents\CMS2Luc\ProjetsNettoyesCMSGit\ProjetCarteMere\project\CMSModifV1SD.c
                 Init_I2C   0x00b5e0    program     extern C:\Users\LFRAD\Documents\CMS2Luc\ProjetsNettoyesCMSGit\ProjetCarteMere\project\CMSModifV1SD.c
               Init_RS485   0x0016aa    program     extern C:\Users\LFRAD\Documents\CMS2Luc\ProjetsNettoyesCMSGit\ProjetCarteMere\project\CMSModifV1SD.c
                IntToChar   0x00e278    program     extern C:\Users\LFRAD\Documents\CMS2Luc\ProjetsNettoyesCMSGit\ProjetCarteMere\project\CMSModifV1SD.c
               IntToChar5   0x011bca    program     extern C:\Users\LFRAD\Documents\CMS2Luc\ProjetsNettoyesCMSGit\ProjetCarteMere\project\CMSModifV1SD.c
              LIRE_EEPROM   0x00b308    program     extern C:\Users\LFRAD\Documents\CMS2Luc\ProjetsNettoyesCMSGit\ProjetCarteMere\project\CMSModifV1SD.c
             LIRE_HORLOGE   0x00f8c0    program     extern C:\Users\LFRAD\Documents\CMS2Luc\ProjetsNettoyesCMSGit\ProjetCarteMere\project\CMSModifV1SD.c
      MESURE_DES_TENSIONS   0x00e936    program     extern C:\Users\LFRAD\Documents\CMS2Luc\ProjetsNettoyesCMSGit\ProjetCarteMere\project\CMSModifV1SD.c
  METTRE_EN_MEMOIRE_LISTE   0x00f578    program     extern C:\Users\LFRAD\Documents\CMS2Luc\ProjetsNettoyesCMSGit\ProjetCarteMere\project\CMSModifV1SD.c
MODIFICATION_TABLE_DEXISTENCE   0x0106fc    program     extern C:\Users\LFRAD\Documents\CMS2Luc\ProjetsNettoyesCMSGit\ProjetCarteMere\project\CMSModifV1SD.c
                 OpenI2C1   0x0142c4    program     extern E:\MPASM_MPLINK_PIC18_LT_Branch_3_42\pic18-lt\cxx-framework\src\pmc_common\i2c\i2c1open.c
    PREPARATION_PAGE_AUTO   0x00dd70    program     extern C:\Users\LFRAD\Documents\CMS2Luc\ProjetsNettoyesCMSGit\ProjetCarteMere\project\CMSModifV1SD.c
         RECEVOIRST_RS485   0x00170a    program     extern C:\Users\LFRAD\Documents\CMS2Luc\ProjetsNettoyesCMSGit\ProjetCarteMere\project\CMSModifV1SD.c
           RECEVOIR_RS485   0x001740    program     extern C:\Users\LFRAD\Documents\CMS2Luc\ProjetsNettoyesCMSGit\ProjetCarteMere\project\CMSModifV1SD.c
 RECHERCHE_DONNEES_GROUPE   0x0105ac    program     extern C:\Users\LFRAD\Documents\CMS2Luc\ProjetsNettoyesCMSGit\ProjetCarteMere\project\CMSModifV1SD.c
  RECUPERATION_DES_TRAMES   0x003644    program     extern C:\Users\LFRAD\Documents\CMS2Luc\ProjetsNettoyesCMSGit\ProjetCarteMere\project\CMSModifV1SD.c
     REMISE_EN_FORME_PAGE   0x011524    program     extern C:\Users\LFRAD\Documents\CMS2Luc\ProjetsNettoyesCMSGit\ProjetCarteMere\project\CMSModifV1SD.c
         REPOSAQUIENVOYER   0x00bef6    program     extern C:\Users\LFRAD\Documents\CMS2Luc\ProjetsNettoyesCMSGit\ProjetCarteMere\project\CMSModifV1SD.c
                    RS485   0x00182e    program     extern C:\Users\LFRAD\Documents\CMS2Luc\ProjetsNettoyesCMSGit\ProjetCarteMere\project\CMSModifV1SD.c
                 ReadI2C1   0x014362    program     extern E:\MPASM_MPLINK_PIC18_LT_Branch_3_42\pic18-lt\cxx-framework\src\pmc_common\i2c\i2c1read.c
            SAV_EXISTENCE   0x01034e    program     extern C:\Users\LFRAD\Documents\CMS2Luc\ProjetsNettoyesCMSGit\ProjetCarteMere\project\CMSModifV1SD.c
                      SDR   0x012c04    program     extern C:\Users\LFRAD\Documents\CMS2Luc\ProjetsNettoyesCMSGit\ProjetCarteMere\project\CMSModifV1SD.c
                    SDRBN   0x012af2    program     extern C:\Users\LFRAD\Documents\CMS2Luc\ProjetsNettoyesCMSGit\ProjetCarteMere\project\CMSModifV1SD.c
                      SDW   0x012558    program     extern C:\Users\LFRAD\Documents\CMS2Luc\ProjetsNettoyesCMSGit\ProjetCarteMere\project\CMSModifV1SD.c
                    SDWBN   0x01247e    program     extern C:\Users\LFRAD\Documents\CMS2Luc\ProjetsNettoyesCMSGit\ProjetCarteMere\project\CMSModifV1SD.c
       SD_ReadSingleBlock   0x00fedc    program     extern C:\Users\LFRAD\Documents\CMS2Luc\ProjetsNettoyesCMSGit\ProjetCarteMere\project\CMSModifV1SD.c
           SD_SendCommand   0x010074    program     extern C:\Users\LFRAD\Documents\CMS2Luc\ProjetsNettoyesCMSGit\ProjetCarteMere\project\CMSModifV1SD.c
      SD_WriteSingleBlock   0x00fd82    program     extern C:\Users\LFRAD\Documents\CMS2Luc\ProjetsNettoyesCMSGit\ProjetCarteMere\project\CMSModifV1SD.c
            SERIALISATION   0x00b804    program     extern C:\Users\LFRAD\Documents\CMS2Luc\ProjetsNettoyesCMSGit\ProjetCarteMere\project\CMSModifV1SD.c
            SPI_WriteByte   0x010184    program     extern C:\Users\LFRAD\Documents\CMS2Luc\ProjetsNettoyesCMSGit\ProjetCarteMere\project\CMSModifV1SD.c
                  TAGTB32   0x014006    program     extern E:\MPASM_MPLINK_PIC18_LT_Branch_3_42\pic18-lt\cxx-framework\src\traditional\math\gtFP.asm
                    TEMPO   0x00fcea    program     extern C:\Users\LFRAD\Documents\CMS2Luc\ProjetsNettoyesCMSGit\ProjetCarteMere\project\CMSModifV1SD.c
   TRAMEENVOIRS485DONNEES   0x0018da    program     extern C:\Users\LFRAD\Documents\CMS2Luc\ProjetsNettoyesCMSGit\ProjetCarteMere\project\CMSModifV1SD.c
TRAMERECEPTIONRS485DONNEES   0x001856    program     extern C:\Users\LFRAD\Documents\CMS2Luc\ProjetsNettoyesCMSGit\ProjetCarteMere\project\CMSModifV1SD.c
TRANSFORMER_TRAME_MEM_EN_COM   0x00c05c    program     extern C:\Users\LFRAD\Documents\CMS2Luc\ProjetsNettoyesCMSGit\ProjetCarteMere\project\CMSModifV1SD.c
          TROUVER_ROBINET   0x01139e    program     extern C:\Users\LFRAD\Documents\CMS2Luc\ProjetsNettoyesCMSGit\ProjetCarteMere\project\CMSModifV1SD.c
               TSIGN1616A   0x013f6e    program     static E:\MPASM_MPLINK_PIC18_LT_Branch_3_42\pic18-lt\cxx-framework\src\traditional\math\fxm1616s.asm
       VALIDER_CAPTEUR_CM   0x010f20    program     extern C:\Users\LFRAD\Documents\CMS2Luc\ProjetsNettoyesCMSGit\ProjetCarteMere\project\CMSModifV1SD.c
                WriteI2C1   0x0141ce    program     extern E:\MPASM_MPLINK_PIC18_LT_Branch_3_42\pic18-lt\cxx-framework\src\pmc_common\i2c\i2c1writ.c
              __FpCompare   0x014018    program     extern E:\MPASM_MPLINK_PIC18_LT_Branch_3_42\pic18-lt\cxx-framework\src\traditional\math\compFP.asm
                 __FpExit   0x0140ce    program     extern E:\MPASM_MPLINK_PIC18_LT_Branch_3_42\pic18-lt\cxx-framework\src\traditional\math\packFP.asm
                 __FpPack   0x0140fa    program     extern E:\MPASM_MPLINK_PIC18_LT_Branch_3_42\pic18-lt\cxx-framework\src\traditional\math\packFP.asm
            __FpReturnNaN   0x0140c2    program     extern E:\MPASM_MPLINK_PIC18_LT_Branch_3_42\pic18-lt\cxx-framework\src\traditional\math\packFP.asm
         __FpReturnNegInf   0x0140d4    program     extern E:\MPASM_MPLINK_PIC18_LT_Branch_3_42\pic18-lt\cxx-framework\src\traditional\math\packFP.asm
        __FpReturnNegZero   0x0140ec    program     extern E:\MPASM_MPLINK_PIC18_LT_Branch_3_42\pic18-lt\cxx-framework\src\traditional\math\packFP.asm
         __FpReturnPosInf   0x0140da    program     extern E:\MPASM_MPLINK_PIC18_LT_Branch_3_42\pic18-lt\cxx-framework\src\traditional\math\packFP.asm
        __FpReturnPosZero   0x0140f4    program     extern E:\MPASM_MPLINK_PIC18_LT_Branch_3_42\pic18-lt\cxx-framework\src\traditional\math\packFP.asm
        __FpReturnSignInf   0x0140d0    program     extern E:\MPASM_MPLINK_PIC18_LT_Branch_3_42\pic18-lt\cxx-framework\src\traditional\math\packFP.asm
       __FpReturnSignZero   0x0140e8    program     extern E:\MPASM_MPLINK_PIC18_LT_Branch_3_42\pic18-lt\cxx-framework\src\traditional\math\packFP.asm
              __FpReturnW   0x014152    program     extern E:\MPASM_MPLINK_PIC18_LT_Branch_3_42\pic18-lt\cxx-framework\src\traditional\math\packFP.asm
              __FpUnPackA   0x014172    program     extern E:\MPASM_MPLINK_PIC18_LT_Branch_3_42\pic18-lt\cxx-framework\src\traditional\math\UnpackFP.asm
              __FpUnPackB   0x0141a2    program     extern E:\MPASM_MPLINK_PIC18_LT_Branch_3_42\pic18-lt\cxx-framework\src\traditional\math\UnpackFP.asm
       ___return_lbl00000   0x000004    program     static                          
       ___return_lbl00000   0x00001c    program     static                          
       ___return_lbl00000   0x014360    program     static                          
       ___return_lbl00000   0x014324    program     static                          
       ___return_lbl00001   0x014392    program     static                          
       ___return_lbl01865   0x013ab4    program     static                          
        ___while_lbl01866   0x013aac    program     static                          
        ___while_lbl01867   0x013ab0    program     static                          
               __config_0   0x300001    program     static C:\Users\LFRAD\Documents\CMS2Luc\ProjetsNettoyesCMSGit\ProjetCarteMere\project\CMSModifV1SD.c
               __config_1   0x300002    program     static C:\Users\LFRAD\Documents\CMS2Luc\ProjetsNettoyesCMSGit\ProjetCarteMere\project\CMSModifV1SD.c
              __config_10   0x30000c    program     static C:\Users\LFRAD\Documents\CMS2Luc\ProjetsNettoyesCMSGit\ProjetCarteMere\project\CMSModifV1SD.c
              __config_11   0x30000d    program     static C:\Users\LFRAD\Documents\CMS2Luc\ProjetsNettoyesCMSGit\ProjetCarteMere\project\CMSModifV1SD.c
               __config_2   0x300003    program     static C:\Users\LFRAD\Documents\CMS2Luc\ProjetsNettoyesCMSGit\ProjetCarteMere\project\CMSModifV1SD.c
               __config_3   0x300004    program     static C:\Users\LFRAD\Documents\CMS2Luc\ProjetsNettoyesCMSGit\ProjetCarteMere\project\CMSModifV1SD.c
               __config_4   0x300005    program     static C:\Users\LFRAD\Documents\CMS2Luc\ProjetsNettoyesCMSGit\ProjetCarteMere\project\CMSModifV1SD.c
               __config_5   0x300006    program     static C:\Users\LFRAD\Documents\CMS2Luc\ProjetsNettoyesCMSGit\ProjetCarteMere\project\CMSModifV1SD.c
               __config_6   0x300008    program     static C:\Users\LFRAD\Documents\CMS2Luc\ProjetsNettoyesCMSGit\ProjetCarteMere\project\CMSModifV1SD.c
               __config_7   0x300009    program     static C:\Users\LFRAD\Documents\CMS2Luc\ProjetsNettoyesCMSGit\ProjetCarteMere\project\CMSModifV1SD.c
               __config_8   0x30000a    program     static C:\Users\LFRAD\Documents\CMS2Luc\ProjetsNettoyesCMSGit\ProjetCarteMere\project\CMSModifV1SD.c
               __config_9   0x30000b    program     static C:\Users\LFRAD\Documents\CMS2Luc\ProjetsNettoyesCMSGit\ProjetCarteMere\project\CMSModifV1SD.c
                   __init   0x014394    program     extern E:\MPASM_MPLINK_PIC18_LT_Branch_3_42\pic18-lt\cxx-framework\src\traditional\stdclib\__init.c
            __tmplbl_1038   0x012422    program     static                          
             __tmplbl_719   0x0011f0    program     static                          
             __tmplbl_768   0x000888    program     static                          
             __tmplbl_771   0x00326a    program     static                          
             __tmplbl_772   0x003158    program     static                          
             __tmplbl_773   0x002fe4    program     static                          
             __tmplbl_774   0x002f06    program     static                          
             __tmplbl_775   0x002c4e    program     static                          
             __tmplbl_776   0x002942    program     static                          
             __tmplbl_777   0x002828    program     static                          
             __tmplbl_778   0x002710    program     static                          
             __tmplbl_783   0x003630    program     static                          
             __tmplbl_784   0x003630    program     static                          
             __tmplbl_785   0x003630    program     static                          
             __tmplbl_786   0x003630    program     static                          
             __tmplbl_787   0x003630    program     static                          
             __tmplbl_788   0x003630    program     static                          
             __tmplbl_789   0x003630    program     static                          
             __tmplbl_791   0x003630    program     static                          
             __tmplbl_802   0x003630    program     static                          
             __tmplbl_803   0x003630    program     static                          
             __tmplbl_804   0x003630    program     static                          
             __tmplbl_806   0x003630    program     static                          
             __tmplbl_807   0x003630    program     static                          
             __tmplbl_808   0x003630    program     static                          
             __tmplbl_810   0x003630    program     static                          
             __tmplbl_811   0x003630    program     static                          
             __tmplbl_828   0x006b8c    program     static                          
             __tmplbl_829   0x006a4c    program     static                          
             __tmplbl_830   0x0067b6    program     static                          
             __tmplbl_831   0x0067ae    program     static                          
             __tmplbl_832   0x00677e    program     static                          
             __tmplbl_833   0x00668e    program     static                          
             __tmplbl_834   0x006686    program     static                          
             __tmplbl_835   0x0065a2    program     static                          
             __tmplbl_836   0x006276    program     static                          
             __tmplbl_837   0x007370    program     static                          
             __tmplbl_838   0x0067ae    program     static                          
             __tmplbl_839   0x005fb0    program     static                          
             __tmplbl_840   0x005b44    program     static                          
             __tmplbl_841   0x00588c    program     static                          
             __tmplbl_842   0x0056e0    program     static                          
             __tmplbl_843   0x0054d0    program     static                          
             __tmplbl_844   0x005218    program     static                          
             __tmplbl_845   0x00483a    program     static                          
             __tmplbl_846   0x004718    program     static                          
             __tmplbl_847   0x004472    program     static                          
             __tmplbl_856   0x007366    program     static                          
             __tmplbl_857   0x007366    program     static                          
             __tmplbl_858   0x007342    program     static                          
             __tmplbl_859   0x007370    program     static                          
             __tmplbl_860   0x007370    program     static                          
             __tmplbl_861   0x007370    program     static                          
             __tmplbl_862   0x007362    program     static                          
             __tmplbl_863   0x007342    program     static                          
             __tmplbl_864   0x007370    program     static                          
             __tmplbl_865   0x005212    program     static                          
             __tmplbl_867   0x006270    program     static                          
             __tmplbl_868   0x007362    program     static                          
             __tmplbl_869   0x007362    program     static                          
             __tmplbl_871   0x007370    program     static                          
             __tmplbl_872   0x00679c    program     static                          
             __tmplbl_873   0x007362    program     static                          
             __tmplbl_874   0x005b40    program     static                          
             __tmplbl_875   0x005b20    program     static                          
             __tmplbl_876   0x005b32    program     static                          
             __tmplbl_880   0x005b40    program     static                          
             __tmplbl_881   0x0054cc    program     static                          
             __tmplbl_910   0x007362    program     static                          
             __tmplbl_911   0x005faa    program     static                          
             __tmplbl_912   0x005faa    program     static                          
             __tmplbl_913   0x007362    program     static                          
             __tmplbl_925   0x007362    program     static                          
             __tmplbl_928   0x007362    program     static                          
             __tmplbl_931   0x007370    program     static                          
             __tmplbl_932   0x007370    program     static                          
             __tmplbl_933   0x007370    program     static                          
             __tmplbl_934   0x007342    program     static                          
             __tmplbl_935   0x007354    program     static                          
            __zero_memory   0x014326    program     extern E:\MPASM_MPLINK_PIC18_LT_Branch_3_42\pic18-lt\cxx-framework\src\traditional\proc\p18f8723.asm
                   _entry   0x000000    program     extern E:\MPASM_MPLINK_PIC18_LT_Branch_3_42\pic18-lt\cxx-framework\src\traditional\startup\c018.c
                 _startup   0x01437c    program     extern E:\MPASM_MPLINK_PIC18_LT_Branch_3_42\pic18-lt\cxx-framework\src\traditional\startup\c018.c
               calcul_CRC   0x00ac16    program     extern C:\Users\LFRAD\Documents\CMS2Luc\ProjetsNettoyesCMSGit\ProjetCarteMere\project\CMSModifV1SD.c
        calcul_addmemoire   0x00ad7c    program     extern C:\Users\LFRAD\Documents\CMS2Luc\ProjetsNettoyesCMSGit\ProjetCarteMere\project\CMSModifV1SD.c
            choix_memoire   0x00b13c    program     extern C:\Users\LFRAD\Documents\CMS2Luc\ProjetsNettoyesCMSGit\ProjetCarteMere\project\CMSModifV1SD.c
                compare_l   0x01433c    program     static E:\MPASM_MPLINK_PIC18_LT_Branch_3_42\pic18-lt\cxx-framework\src\traditional\proc\p18f8723.asm
 construire_trame_memoire   0x009102    program     extern C:\Users\LFRAD\Documents\CMS2Luc\ProjetsNettoyesCMSGit\ProjetCarteMere\project\CMSModifV1SD.c
             controle_CRC   0x00acae    program     extern C:\Users\LFRAD\Documents\CMS2Luc\ProjetsNettoyesCMSGit\ProjetCarteMere\project\CMSModifV1SD.c
       controleheureRESET   0x013ade    program     extern C:\Users\LFRAD\Documents\CMS2Luc\ProjetsNettoyesCMSGit\ProjetCarteMere\project\CMSModifV1SD.c
      creer_trame_horloge   0x00f93e    program     extern C:\Users\LFRAD\Documents\CMS2Luc\ProjetsNettoyesCMSGit\ProjetCarteMere\project\CMSModifV1SD.c
                 delay_ms   0x00b55c    program     extern C:\Users\LFRAD\Documents\CMS2Luc\ProjetsNettoyesCMSGit\ProjetCarteMere\project\CMSModifV1SD.c
                 delay_us   0x01031a    program     extern C:\Users\LFRAD\Documents\CMS2Luc\ProjetsNettoyesCMSGit\ProjetCarteMere\project\CMSModifV1SD.c
                  endloop   0x014320    program     static                          
                  endloop   0x01435c    program     static                          
     entrer_trame_horloge   0x00fa7e    program     extern C:\Users\LFRAD\Documents\CMS2Luc\ProjetsNettoyesCMSGit\ProjetCarteMere\project\CMSModifV1SD.c
       envoyerHORLOGE_i2c   0x00f74a    program     extern C:\Users\LFRAD\Documents\CMS2Luc\ProjetsNettoyesCMSGit\ProjetCarteMere\project\CMSModifV1SD.c
      envoyer_TRAME_PICSD   0x01316e    program     extern C:\Users\LFRAD\Documents\CMS2Luc\ProjetsNettoyesCMSGit\ProjetCarteMere\project\CMSModifV1SD.c
                 getsI2C1   0x01424e    program     extern E:\MPASM_MPLINK_PIC18_LT_Branch_3_42\pic18-lt\cxx-framework\src\pmc_common\i2c\i2c1gets.c
      identificationINTER   0x00b8f4    program     extern C:\Users\LFRAD\Documents\CMS2Luc\ProjetsNettoyesCMSGit\ProjetCarteMere\project\CMSModifV1SD.c
                 init_spi   0x0102fe    program     extern C:\Users\LFRAD\Documents\CMS2Luc\ProjetsNettoyesCMSGit\ProjetCarteMere\project\CMSModifV1SD.c
                    inter   0x000202    program     extern C:\Users\LFRAD\Documents\CMS2Luc\ProjetsNettoyesCMSGit\ProjetCarteMere\project\CMSModifV1SD.c
        intervertirOUT_IN   0x01053c    program     extern C:\Users\LFRAD\Documents\CMS2Luc\ProjetsNettoyesCMSGit\ProjetCarteMere\project\CMSModifV1SD.c
                 jANotInf   0x013d40    program     static E:\MPASM_MPLINK_PIC18_LT_Branch_3_42\pic18-lt\cxx-framework\src\traditional\math\divFP.asm
                 jANotInf   0x013de6    program     static E:\MPASM_MPLINK_PIC18_LT_Branch_3_42\pic18-lt\cxx-framework\src\traditional\math\mulFP.asm
                 jANotInf   0x013c1e    program     static E:\MPASM_MPLINK_PIC18_LT_Branch_3_42\pic18-lt\cxx-framework\src\traditional\math\addFP.asm
                 jANotNeg   0x013cb2    program     static E:\MPASM_MPLINK_PIC18_LT_Branch_3_42\pic18-lt\cxx-framework\src\traditional\math\addFP.asm
                jANotZero   0x013d54    program     static E:\MPASM_MPLINK_PIC18_LT_Branch_3_42\pic18-lt\cxx-framework\src\traditional\math\divFP.asm
              jAandWsetup   0x013c82    program     static E:\MPASM_MPLINK_PIC18_LT_Branch_3_42\pic18-lt\cxx-framework\src\traditional\math\addFP.asm
                  jAisNeg   0x014094    program     static E:\MPASM_MPLINK_PIC18_LT_Branch_3_42\pic18-lt\cxx-framework\src\traditional\math\compFP.asm
                 jAltBexp   0x013c70    program     static E:\MPASM_MPLINK_PIC18_LT_Branch_3_42\pic18-lt\cxx-framework\src\traditional\math\addFP.asm
                jBANotInf   0x013c14    program     static E:\MPASM_MPLINK_PIC18_LT_Branch_3_42\pic18-lt\cxx-framework\src\traditional\math\addFP.asm
                 jBNotInf   0x013c2c    program     static E:\MPASM_MPLINK_PIC18_LT_Branch_3_42\pic18-lt\cxx-framework\src\traditional\math\addFP.asm
              jBothFinite   0x013df4    program     static E:\MPASM_MPLINK_PIC18_LT_Branch_3_42\pic18-lt\cxx-framework\src\traditional\math\mulFP.asm
             jBothNotZero   0x014036    program     static E:\MPASM_MPLINK_PIC18_LT_Branch_3_42\pic18-lt\cxx-framework\src\traditional\math\compFP.asm
             jBothNotZero   0x013e00    program     static E:\MPASM_MPLINK_PIC18_LT_Branch_3_42\pic18-lt\cxx-framework\src\traditional\math\mulFP.asm
            jDifOrPosSign   0x013c40    program     static E:\MPASM_MPLINK_PIC18_LT_Branch_3_42\pic18-lt\cxx-framework\src\traditional\math\addFP.asm
                      jEQ   0x014052    program     static E:\MPASM_MPLINK_PIC18_LT_Branch_3_42\pic18-lt\cxx-framework\src\traditional\math\compFP.asm
                    jExch   0x01405e    program     static E:\MPASM_MPLINK_PIC18_LT_Branch_3_42\pic18-lt\cxx-framework\src\traditional\math\compFP.asm
                    jExit   0x014004    program     static E:\MPASM_MPLINK_PIC18_LT_Branch_3_42\pic18-lt\cxx-framework\src\traditional\math\castFP08.asm
                   jExpEQ   0x0140a4    program     static E:\MPASM_MPLINK_PIC18_LT_Branch_3_42\pic18-lt\cxx-framework\src\traditional\math\compFP.asm
                   jFinal   0x014088    program     static E:\MPASM_MPLINK_PIC18_LT_Branch_3_42\pic18-lt\cxx-framework\src\traditional\math\compFP.asm
               jFinalSign   0x013d1a    program     static E:\MPASM_MPLINK_PIC18_LT_Branch_3_42\pic18-lt\cxx-framework\src\traditional\math\addFP.asm
                jHaveZero   0x013dfc    program     static E:\MPASM_MPLINK_PIC18_LT_Branch_3_42\pic18-lt\cxx-framework\src\traditional\math\mulFP.asm
                jI2F08Beg   0x013bb6    program     static E:\MPASM_MPLINK_PIC18_LT_Branch_3_42\pic18-lt\cxx-framework\src\traditional\math\cast08FP.asm
                jI2F16Beg   0x013bde    program     static E:\MPASM_MPLINK_PIC18_LT_Branch_3_42\pic18-lt\cxx-framework\src\traditional\math\cast16FP.asm
                    jLoop   0x013d7c    program     static E:\MPASM_MPLINK_PIC18_LT_Branch_3_42\pic18-lt\cxx-framework\src\traditional\math\divFP.asm
                    jLoop   0x013fec    program     static E:\MPASM_MPLINK_PIC18_LT_Branch_3_42\pic18-lt\cxx-framework\src\traditional\math\castFP08.asm
                jLoopExit   0x013ffa    program     static E:\MPASM_MPLINK_PIC18_LT_Branch_3_42\pic18-lt\cxx-framework\src\traditional\math\castFP08.asm
                     jMax   0x013fc8    program     static E:\MPASM_MPLINK_PIC18_LT_Branch_3_42\pic18-lt\cxx-framework\src\traditional\math\castFP08.asm
                  jMaxNeg   0x013fd2    program     static E:\MPASM_MPLINK_PIC18_LT_Branch_3_42\pic18-lt\cxx-framework\src\traditional\math\castFP08.asm
                  jMaxPos   0x013fcc    program     static E:\MPASM_MPLINK_PIC18_LT_Branch_3_42\pic18-lt\cxx-framework\src\traditional\math\castFP08.asm
                      jNE   0x014056    program     static E:\MPASM_MPLINK_PIC18_LT_Branch_3_42\pic18-lt\cxx-framework\src\traditional\math\compFP.asm
                    jNext   0x013da2    program     static E:\MPASM_MPLINK_PIC18_LT_Branch_3_42\pic18-lt\cxx-framework\src\traditional\math\divFP.asm
                jNoAdjust   0x013da0    program     static E:\MPASM_MPLINK_PIC18_LT_Branch_3_42\pic18-lt\cxx-framework\src\traditional\math\divFP.asm
                  jNoExch   0x01407e    program     static E:\MPASM_MPLINK_PIC18_LT_Branch_3_42\pic18-lt\cxx-framework\src\traditional\math\compFP.asm
             jNotBothZero   0x013c44    program     static E:\MPASM_MPLINK_PIC18_LT_Branch_3_42\pic18-lt\cxx-framework\src\traditional\math\addFP.asm
                  jNotInf   0x013fdc    program     static E:\MPASM_MPLINK_PIC18_LT_Branch_3_42\pic18-lt\cxx-framework\src\traditional\math\castFP08.asm
                  jPkLoop   0x014108    program     static E:\MPASM_MPLINK_PIC18_LT_Branch_3_42\pic18-lt\cxx-framework\src\traditional\math\packFP.asm
             jPkRoundDone   0x014152    program     static E:\MPASM_MPLINK_PIC18_LT_Branch_3_42\pic18-lt\cxx-framework\src\traditional\math\packFP.asm
               jPkRoundIt   0x01413a    program     static E:\MPASM_MPLINK_PIC18_LT_Branch_3_42\pic18-lt\cxx-framework\src\traditional\math\packFP.asm
             jPkShiftDone   0x014124    program     static E:\MPASM_MPLINK_PIC18_LT_Branch_3_42\pic18-lt\cxx-framework\src\traditional\math\packFP.asm
           jReturnPosInf0   0x0140de    program     static E:\MPASM_MPLINK_PIC18_LT_Branch_3_42\pic18-lt\cxx-framework\src\traditional\math\packFP.asm
                  jRotate   0x0140b0    program     static E:\MPASM_MPLINK_PIC18_LT_Branch_3_42\pic18-lt\cxx-framework\src\traditional\math\compFP.asm
                   jShift   0x01409a    program     static E:\MPASM_MPLINK_PIC18_LT_Branch_3_42\pic18-lt\cxx-framework\src\traditional\math\compFP.asm
               jShiftDone   0x013cda    program     static E:\MPASM_MPLINK_PIC18_LT_Branch_3_42\pic18-lt\cxx-framework\src\traditional\math\addFP.asm
               jShiftLoop   0x013ccc    program     static E:\MPASM_MPLINK_PIC18_LT_Branch_3_42\pic18-lt\cxx-framework\src\traditional\math\addFP.asm
                jSignDone   0x013d0a    program     static E:\MPASM_MPLINK_PIC18_LT_Branch_3_42\pic18-lt\cxx-framework\src\traditional\math\addFP.asm
              jSignedZero   0x013d4a    program     static E:\MPASM_MPLINK_PIC18_LT_Branch_3_42\pic18-lt\cxx-framework\src\traditional\math\divFP.asm
                 jSignsEQ   0x01403a    program     static E:\MPASM_MPLINK_PIC18_LT_Branch_3_42\pic18-lt\cxx-framework\src\traditional\math\compFP.asm
                  jUnpkA1   0x01417c    program     static E:\MPASM_MPLINK_PIC18_LT_Branch_3_42\pic18-lt\cxx-framework\src\traditional\math\UnpackFP.asm
                  jUnpkA2   0x014194    program     static E:\MPASM_MPLINK_PIC18_LT_Branch_3_42\pic18-lt\cxx-framework\src\traditional\math\UnpackFP.asm
                 jUnpkANZ   0x01418a    program     static E:\MPASM_MPLINK_PIC18_LT_Branch_3_42\pic18-lt\cxx-framework\src\traditional\math\UnpackFP.asm
                  jUnpkB1   0x0141ac    program     static E:\MPASM_MPLINK_PIC18_LT_Branch_3_42\pic18-lt\cxx-framework\src\traditional\math\UnpackFP.asm
                  jUnpkB2   0x0141c4    program     static E:\MPASM_MPLINK_PIC18_LT_Branch_3_42\pic18-lt\cxx-framework\src\traditional\math\UnpackFP.asm
                 jUnpkBNZ   0x0141ba    program     static E:\MPASM_MPLINK_PIC18_LT_Branch_3_42\pic18-lt\cxx-framework\src\traditional\math\UnpackFP.asm
                 jUnpkNaN   0x01419e    program     static E:\MPASM_MPLINK_PIC18_LT_Branch_3_42\pic18-lt\cxx-framework\src\traditional\math\UnpackFP.asm
                 jWNotNeg   0x013cc6    program     static E:\MPASM_MPLINK_PIC18_LT_Branch_3_42\pic18-lt\cxx-framework\src\traditional\math\addFP.asm
                    jZero   0x013fd8    program     static E:\MPASM_MPLINK_PIC18_LT_Branch_3_42\pic18-lt\cxx-framework\src\traditional\math\castFP08.asm
               jZero1and2   0x0140e2    program     static E:\MPASM_MPLINK_PIC18_LT_Branch_3_42\pic18-lt\cxx-framework\src\traditional\math\packFP.asm
             lire_horloge   0x00c03e    program     extern C:\Users\LFRAD\Documents\CMS2Luc\ProjetsNettoyesCMSGit\ProjetCarteMere\project\CMSModifV1SD.c
           litHORLOGE_i2c   0x00f794    program     extern C:\Users\LFRAD\Documents\CMS2Luc\ProjetsNettoyesCMSGit\ProjetCarteMere\project\CMSModifV1SD.c
                     loop   0x014388    program     static                          
                     loop   0x014304    program     static                          
                     loop   0x01434e    program     static                          
                   loop_h   0x014334    program     static E:\MPASM_MPLINK_PIC18_LT_Branch_3_42\pic18-lt\cxx-framework\src\traditional\proc\p18f8723.asm
                   loop_l   0x01433e    program     static E:\MPASM_MPLINK_PIC18_LT_Branch_3_42\pic18-lt\cxx-framework\src\traditional\proc\p18f8723.asm
                     main   0x0002c4    program     extern C:\Users\LFRAD\Documents\CMS2Luc\ProjetsNettoyesCMSGit\ProjetCarteMere\project\CMSModifV1SD.c
          pic_eeprom_read   0x013abc    program     extern C:\Users\LFRAD\Documents\CMS2Luc\ProjetsNettoyesCMSGit\ProjetCarteMere\project\CMSModifV1SD.c
         pic_eeprom_write   0x013a88    program     extern C:\Users\LFRAD\Documents\CMS2Luc\ProjetsNettoyesCMSGit\ProjetCarteMere\project\CMSModifV1SD.c
             putstringI2C   0x00e1b8    program     extern C:\Users\LFRAD\Documents\CMS2Luc\ProjetsNettoyesCMSGit\ProjetCarteMere\project\CMSModifV1SD.c
  recuperer_trame_memoire   0x007384    program     extern C:\Users\LFRAD\Documents\CMS2Luc\ProjetsNettoyesCMSGit\ProjetCarteMere\project\CMSModifV1SD.c
            reglerhorloge   0x00c032    program     extern C:\Users\LFRAD\Documents\CMS2Luc\ProjetsNettoyesCMSGit\ProjetCarteMere\project\CMSModifV1SD.c
      reglerhorlogeautres   0x0138aa    program     extern C:\Users\LFRAD\Documents\CMS2Luc\ProjetsNettoyesCMSGit\ProjetCarteMere\project\CMSModifV1SD.c
                  resetTO   0x00ad22    program     extern C:\Users\LFRAD\Documents\CMS2Luc\ProjetsNettoyesCMSGit\ProjetCarteMere\project\CMSModifV1SD.c
                 sd_reset   0x0101a2    program     extern C:\Users\LFRAD\Documents\CMS2Luc\ProjetsNettoyesCMSGit\ProjetCarteMere\project\CMSModifV1SD.c
                 spi_high   0x0102f8    program     extern C:\Users\LFRAD\Documents\CMS2Luc\ProjetsNettoyesCMSGit\ProjetCarteMere\project\CMSModifV1SD.c
                  spi_low   0x0102f2    program     extern C:\Users\LFRAD\Documents\CMS2Luc\ProjetsNettoyesCMSGit\ProjetCarteMere\project\CMSModifV1SD.c
                   stopIO   0x013a7a    program     extern C:\Users\LFRAD\Documents\CMS2Luc\ProjetsNettoyesCMSGit\ProjetCarteMere\project\CMSModifV1SD.c
trouver_carte_suivantvoie   0x00fb28    program     extern C:\Users\LFRAD\Documents\CMS2Luc\ProjetsNettoyesCMSGit\ProjetCarteMere\project\CMSModifV1SD.c
               zero_block   0x014334    program     static E:\MPASM_MPLINK_PIC18_LT_Branch_3_42\pic18-lt\cxx-framework\src\traditional\proc\p18f8723.asm
                   ADCON0   0x000fc2       data     extern E:\MPASM_MPLINK_PIC18_LT_Branch_3_42\pic18-lt\cxx-framework\src\traditional\proc\p18f8723.asm
               ADCON0bits   0x000fc2       data     extern E:\MPASM_MPLINK_PIC18_LT_Branch_3_42\pic18-lt\cxx-framework\src\traditional\proc\p18f8723.asm
                   ADCON1   0x000fc1       data     extern E:\MPASM_MPLINK_PIC18_LT_Branch_3_42\pic18-lt\cxx-framework\src\traditional\proc\p18f8723.asm
               ADCON1bits   0x000fc1       data     extern E:\MPASM_MPLINK_PIC18_LT_Branch_3_42\pic18-lt\cxx-framework\src\traditional\proc\p18f8723.asm
                   ADCON2   0x000fc0       data     extern E:\MPASM_MPLINK_PIC18_LT_Branch_3_42\pic18-lt\cxx-framework\src\traditional\proc\p18f8723.asm
               ADCON2bits   0x000fc0       data     extern E:\MPASM_MPLINK_PIC18_LT_Branch_3_42\pic18-lt\cxx-framework\src\traditional\proc\p18f8723.asm
                    ADRES   0x000fc3       data     extern E:\MPASM_MPLINK_PIC18_LT_Branch_3_42\pic18-lt\cxx-framework\src\traditional\proc\p18f8723.asm
                   ADRESH   0x000fc4       data     extern E:\MPASM_MPLINK_PIC18_LT_Branch_3_42\pic18-lt\cxx-framework\src\traditional\proc\p18f8723.asm
                   ADRESL   0x000fc3       data     extern E:\MPASM_MPLINK_PIC18_LT_Branch_3_42\pic18-lt\cxx-framework\src\traditional\proc\p18f8723.asm
                    ANNEE   0x0002f0       data     extern C:\Users\LFRAD\Documents\CMS2Luc\ProjetsNettoyesCMSGit\ProjetCarteMere\project\CMSModifV1SD.c
                  BAUDCON   0x000f7e       data     extern E:\MPASM_MPLINK_PIC18_LT_Branch_3_42\pic18-lt\cxx-framework\src\traditional\proc\p18f8723.asm
                 BAUDCON1   0x000f7e       data     extern E:\MPASM_MPLINK_PIC18_LT_Branch_3_42\pic18-lt\cxx-framework\src\traditional\proc\p18f8723.asm
             BAUDCON1bits   0x000f7e       data     extern E:\MPASM_MPLINK_PIC18_LT_Branch_3_42\pic18-lt\cxx-framework\src\traditional\proc\p18f8723.asm
                 BAUDCON2   0x000f7c       data     extern E:\MPASM_MPLINK_PIC18_LT_Branch_3_42\pic18-lt\cxx-framework\src\traditional\proc\p18f8723.asm
             BAUDCON2bits   0x000f7c       data     extern E:\MPASM_MPLINK_PIC18_LT_Branch_3_42\pic18-lt\cxx-framework\src\traditional\proc\p18f8723.asm
              BAUDCONbits   0x000f7e       data     extern E:\MPASM_MPLINK_PIC18_LT_Branch_3_42\pic18-lt\cxx-framework\src\traditional\proc\p18f8723.asm
                      BSR   0x000fe0       data     extern E:\MPASM_MPLINK_PIC18_LT_Branch_3_42\pic18-lt\cxx-framework\src\traditional\proc\p18f8723.asm
                    CABLE   0x000234       data     extern C:\Users\LFRAD\Documents\CMS2Luc\ProjetsNettoyesCMSGit\ProjetCarteMere\project\CMSModifV1SD.c
        CAPTEUR_A_EFFACER   0x00028e       data     extern C:\Users\LFRAD\Documents\CMS2Luc\ProjetsNettoyesCMSGit\ProjetCarteMere\project\CMSModifV1SD.c
                     CCON   0x00020b       data     extern C:\Users\LFRAD\Documents\CMS2Luc\ProjetsNettoyesCMSGit\ProjetCarteMere\project\CMSModifV1SD.c
                  CCP1CON   0x000fbd       data     extern E:\MPASM_MPLINK_PIC18_LT_Branch_3_42\pic18-lt\cxx-framework\src\traditional\proc\p18f8723.asm
              CCP1CONbits   0x000fbd       data     extern E:\MPASM_MPLINK_PIC18_LT_Branch_3_42\pic18-lt\cxx-framework\src\traditional\proc\p18f8723.asm
                  CCP2CON   0x000fba       data     extern E:\MPASM_MPLINK_PIC18_LT_Branch_3_42\pic18-lt\cxx-framework\src\traditional\proc\p18f8723.asm
              CCP2CONbits   0x000fba       data     extern E:\MPASM_MPLINK_PIC18_LT_Branch_3_42\pic18-lt\cxx-framework\src\traditional\proc\p18f8723.asm
                  CCP3CON   0x000fb7       data     extern E:\MPASM_MPLINK_PIC18_LT_Branch_3_42\pic18-lt\cxx-framework\src\traditional\proc\p18f8723.asm
              CCP3CONbits   0x000fb7       data     extern E:\MPASM_MPLINK_PIC18_LT_Branch_3_42\pic18-lt\cxx-framework\src\traditional\proc\p18f8723.asm
                  CCP4CON   0x000f73       data     extern E:\MPASM_MPLINK_PIC18_LT_Branch_3_42\pic18-lt\cxx-framework\src\traditional\proc\p18f8723.asm
              CCP4CONbits   0x000f73       data     extern E:\MPASM_MPLINK_PIC18_LT_Branch_3_42\pic18-lt\cxx-framework\src\traditional\proc\p18f8723.asm
                  CCP5CON   0x000f70       data     extern E:\MPASM_MPLINK_PIC18_LT_Branch_3_42\pic18-lt\cxx-framework\src\traditional\proc\p18f8723.asm
              CCP5CONbits   0x000f70       data     extern E:\MPASM_MPLINK_PIC18_LT_Branch_3_42\pic18-lt\cxx-framework\src\traditional\proc\p18f8723.asm
                    CCPR1   0x000fbe       data     extern E:\MPASM_MPLINK_PIC18_LT_Branch_3_42\pic18-lt\cxx-framework\src\traditional\proc\p18f8723.asm
                   CCPR1H   0x000fbf       data     extern E:\MPASM_MPLINK_PIC18_LT_Branch_3_42\pic18-lt\cxx-framework\src\traditional\proc\p18f8723.asm
                   CCPR1L   0x000fbe       data     extern E:\MPASM_MPLINK_PIC18_LT_Branch_3_42\pic18-lt\cxx-framework\src\traditional\proc\p18f8723.asm
                    CCPR2   0x000fbb       data     extern E:\MPASM_MPLINK_PIC18_LT_Branch_3_42\pic18-lt\cxx-framework\src\traditional\proc\p18f8723.asm
                   CCPR2H   0x000fbc       data     extern E:\MPASM_MPLINK_PIC18_LT_Branch_3_42\pic18-lt\cxx-framework\src\traditional\proc\p18f8723.asm
                   CCPR2L   0x000fbb       data     extern E:\MPASM_MPLINK_PIC18_LT_Branch_3_42\pic18-lt\cxx-framework\src\traditional\proc\p18f8723.asm
                    CCPR3   0x000fb8       data     extern E:\MPASM_MPLINK_PIC18_LT_Branch_3_42\pic18-lt\cxx-framework\src\traditional\proc\p18f8723.asm
                   CCPR3H   0x000fb9       data     extern E:\MPASM_MPLINK_PIC18_LT_Branch_3_42\pic18-lt\cxx-framework\src\traditional\proc\p18f8723.asm
                   CCPR3L   0x000fb8       data     extern E:\MPASM_MPLINK_PIC18_LT_Branch_3_42\pic18-lt\cxx-framework\src\traditional\proc\p18f8723.asm
                    CCPR4   0x000f74       data     extern E:\MPASM_MPLINK_PIC18_LT_Branch_3_42\pic18-lt\cxx-framework\src\traditional\proc\p18f8723.asm
                   CCPR4H   0x000f75       data     extern E:\MPASM_MPLINK_PIC18_LT_Branch_3_42\pic18-lt\cxx-framework\src\traditional\proc\p18f8723.asm
                   CCPR4L   0x000f74       data     extern E:\MPASM_MPLINK_PIC18_LT_Branch_3_42\pic18-lt\cxx-framework\src\traditional\proc\p18f8723.asm
                    CCPR5   0x000f71       data     extern E:\MPASM_MPLINK_PIC18_LT_Branch_3_42\pic18-lt\cxx-framework\src\traditional\proc\p18f8723.asm
                   CCPR5H   0x000f72       data     extern E:\MPASM_MPLINK_PIC18_LT_Branch_3_42\pic18-lt\cxx-framework\src\traditional\proc\p18f8723.asm
                   CCPR5L   0x000f71       data     extern E:\MPASM_MPLINK_PIC18_LT_Branch_3_42\pic18-lt\cxx-framework\src\traditional\proc\p18f8723.asm
                    CMCON   0x000fb4       data     extern E:\MPASM_MPLINK_PIC18_LT_Branch_3_42\pic18-lt\cxx-framework\src\traditional\proc\p18f8723.asm
                CMCONbits   0x000fb4       data     extern E:\MPASM_MPLINK_PIC18_LT_Branch_3_42\pic18-lt\cxx-framework\src\traditional\proc\p18f8723.asm
                     CMOD   0x000207       data     extern C:\Users\LFRAD\Documents\CMS2Luc\ProjetsNettoyesCMSGit\ProjetCarteMere\project\CMSModifV1SD.c
                      COD   0x000240       data     extern C:\Users\LFRAD\Documents\CMS2Luc\ProjetsNettoyesCMSGit\ProjetCarteMere\project\CMSModifV1SD.c
              COMMENTAIRE   0x000220       data     extern C:\Users\LFRAD\Documents\CMS2Luc\ProjetsNettoyesCMSGit\ProjetCarteMere\project\CMSModifV1SD.c
             CONSTITUTION   0x000213       data     extern C:\Users\LFRAD\Documents\CMS2Luc\ProjetsNettoyesCMSGit\ProjetCarteMere\project\CMSModifV1SD.c
                      CRC   0x000264       data     extern C:\Users\LFRAD\Documents\CMS2Luc\ProjetsNettoyesCMSGit\ProjetCarteMere\project\CMSModifV1SD.c
                 CRC_ETAT   0x000f1e       data     extern C:\Users\LFRAD\Documents\CMS2Luc\ProjetsNettoyesCMSGit\ProjetCarteMere\project\CMSModifV1SD.c
                     CREP   0x00020f       data     extern C:\Users\LFRAD\Documents\CMS2Luc\ProjetsNettoyesCMSGit\ProjetCarteMere\project\CMSModifV1SD.c
                   CVRCON   0x000fb5       data     extern E:\MPASM_MPLINK_PIC18_LT_Branch_3_42\pic18-lt\cxx-framework\src\traditional\proc\p18f8723.asm
               CVRCONbits   0x000fb5       data     extern E:\MPASM_MPLINK_PIC18_LT_Branch_3_42\pic18-lt\cxx-framework\src\traditional\proc\p18f8723.asm
                  DATAFIX   0x0003e6       data     extern C:\Users\LFRAD\Documents\CMS2Luc\ProjetsNettoyesCMSGit\ProjetCarteMere\project\CMSModifV1SD.c
                     DATE   0x0002f1       data     extern C:\Users\LFRAD\Documents\CMS2Luc\ProjetsNettoyesCMSGit\ProjetCarteMere\project\CMSModifV1SD.c
                     DDRA   0x000f92       data     extern E:\MPASM_MPLINK_PIC18_LT_Branch_3_42\pic18-lt\cxx-framework\src\traditional\proc\p18f8723.asm
                 DDRAbits   0x000f92       data     extern E:\MPASM_MPLINK_PIC18_LT_Branch_3_42\pic18-lt\cxx-framework\src\traditional\proc\p18f8723.asm
                     DDRB   0x000f93       data     extern E:\MPASM_MPLINK_PIC18_LT_Branch_3_42\pic18-lt\cxx-framework\src\traditional\proc\p18f8723.asm
                 DDRBbits   0x000f93       data     extern E:\MPASM_MPLINK_PIC18_LT_Branch_3_42\pic18-lt\cxx-framework\src\traditional\proc\p18f8723.asm
                     DDRC   0x000f94       data     extern E:\MPASM_MPLINK_PIC18_LT_Branch_3_42\pic18-lt\cxx-framework\src\traditional\proc\p18f8723.asm
                 DDRCbits   0x000f94       data     extern E:\MPASM_MPLINK_PIC18_LT_Branch_3_42\pic18-lt\cxx-framework\src\traditional\proc\p18f8723.asm
                     DDRD   0x000f95       data     extern E:\MPASM_MPLINK_PIC18_LT_Branch_3_42\pic18-lt\cxx-framework\src\traditional\proc\p18f8723.asm
                 DDRDbits   0x000f95       data     extern E:\MPASM_MPLINK_PIC18_LT_Branch_3_42\pic18-lt\cxx-framework\src\traditional\proc\p18f8723.asm
                     DDRE   0x000f96       data     extern E:\MPASM_MPLINK_PIC18_LT_Branch_3_42\pic18-lt\cxx-framework\src\traditional\proc\p18f8723.asm
                 DDREbits   0x000f96       data     extern E:\MPASM_MPLINK_PIC18_LT_Branch_3_42\pic18-lt\cxx-framework\src\traditional\proc\p18f8723.asm
                     DDRF   0x000f97       data     extern E:\MPASM_MPLINK_PIC18_LT_Branch_3_42\pic18-lt\cxx-framework\src\traditional\proc\p18f8723.asm
                 DDRFbits   0x000f97       data     extern E:\MPASM_MPLINK_PIC18_LT_Branch_3_42\pic18-lt\cxx-framework\src\traditional\proc\p18f8723.asm
                     DDRG   0x000f98       data     extern E:\MPASM_MPLINK_PIC18_LT_Branch_3_42\pic18-lt\cxx-framework\src\traditional\proc\p18f8723.asm
                 DDRGbits   0x000f98       data     extern E:\MPASM_MPLINK_PIC18_LT_Branch_3_42\pic18-lt\cxx-framework\src\traditional\proc\p18f8723.asm
                     DDRH   0x000f99       data     extern E:\MPASM_MPLINK_PIC18_LT_Branch_3_42\pic18-lt\cxx-framework\src\traditional\proc\p18f8723.asm
                 DDRHbits   0x000f99       data     extern E:\MPASM_MPLINK_PIC18_LT_Branch_3_42\pic18-lt\cxx-framework\src\traditional\proc\p18f8723.asm
                     DDRJ   0x000f9a       data     extern E:\MPASM_MPLINK_PIC18_LT_Branch_3_42\pic18-lt\cxx-framework\src\traditional\proc\p18f8723.asm
                 DDRJbits   0x000f9a       data     extern E:\MPASM_MPLINK_PIC18_LT_Branch_3_42\pic18-lt\cxx-framework\src\traditional\proc\p18f8723.asm
             DEBIT_GLOBAL   0x0003b5       data     extern C:\Users\LFRAD\Documents\CMS2Luc\ProjetsNettoyesCMSGit\ProjetCarteMere\project\CMSModifV1SD.c
             DEMANDEZIGIO   0x000f3c       data     extern C:\Users\LFRAD\Documents\CMS2Luc\ProjetsNettoyesCMSGit\ProjetCarteMere\project\CMSModifV1SD.c
             DEMANDEZPLIO   0x000f41       data     extern C:\Users\LFRAD\Documents\CMS2Luc\ProjetsNettoyesCMSGit\ProjetCarteMere\project\CMSModifV1SD.c
   DEMANDE_INFOS_CAPTEURS   0x000293       data     extern C:\Users\LFRAD\Documents\CMS2Luc\ProjetsNettoyesCMSGit\ProjetCarteMere\project\CMSModifV1SD.c
                 DISTANCE   0x000248       data     extern C:\Users\LFRAD\Documents\CMS2Luc\ProjetsNettoyesCMSGit\ProjetCarteMere\project\CMSModifV1SD.c
                  ECCP1AS   0x000fb6       data     extern E:\MPASM_MPLINK_PIC18_LT_Branch_3_42\pic18-lt\cxx-framework\src\traditional\proc\p18f8723.asm
              ECCP1ASbits   0x000fb6       data     extern E:\MPASM_MPLINK_PIC18_LT_Branch_3_42\pic18-lt\cxx-framework\src\traditional\proc\p18f8723.asm
                 ECCP1CON   0x000fbd       data     extern E:\MPASM_MPLINK_PIC18_LT_Branch_3_42\pic18-lt\cxx-framework\src\traditional\proc\p18f8723.asm
             ECCP1CONbits   0x000fbd       data     extern E:\MPASM_MPLINK_PIC18_LT_Branch_3_42\pic18-lt\cxx-framework\src\traditional\proc\p18f8723.asm
                 ECCP1DEL   0x000f79       data     extern E:\MPASM_MPLINK_PIC18_LT_Branch_3_42\pic18-lt\cxx-framework\src\traditional\proc\p18f8723.asm
             ECCP1DELbits   0x000f79       data     extern E:\MPASM_MPLINK_PIC18_LT_Branch_3_42\pic18-lt\cxx-framework\src\traditional\proc\p18f8723.asm
                  ECCP2AS   0x000f68       data     extern E:\MPASM_MPLINK_PIC18_LT_Branch_3_42\pic18-lt\cxx-framework\src\traditional\proc\p18f8723.asm
              ECCP2ASbits   0x000f68       data     extern E:\MPASM_MPLINK_PIC18_LT_Branch_3_42\pic18-lt\cxx-framework\src\traditional\proc\p18f8723.asm
                 ECCP2CON   0x000fba       data     extern E:\MPASM_MPLINK_PIC18_LT_Branch_3_42\pic18-lt\cxx-framework\src\traditional\proc\p18f8723.asm
             ECCP2CONbits   0x000fba       data     extern E:\MPASM_MPLINK_PIC18_LT_Branch_3_42\pic18-lt\cxx-framework\src\traditional\proc\p18f8723.asm
                 ECCP2DEL   0x000f67       data     extern E:\MPASM_MPLINK_PIC18_LT_Branch_3_42\pic18-lt\cxx-framework\src\traditional\proc\p18f8723.asm
             ECCP2DELbits   0x000f67       data     extern E:\MPASM_MPLINK_PIC18_LT_Branch_3_42\pic18-lt\cxx-framework\src\traditional\proc\p18f8723.asm
                  ECCP3AS   0x000f6a       data     extern E:\MPASM_MPLINK_PIC18_LT_Branch_3_42\pic18-lt\cxx-framework\src\traditional\proc\p18f8723.asm
              ECCP3ASbits   0x000f6a       data     extern E:\MPASM_MPLINK_PIC18_LT_Branch_3_42\pic18-lt\cxx-framework\src\traditional\proc\p18f8723.asm
                 ECCP3CON   0x000fb7       data     extern E:\MPASM_MPLINK_PIC18_LT_Branch_3_42\pic18-lt\cxx-framework\src\traditional\proc\p18f8723.asm
             ECCP3CONbits   0x000fb7       data     extern E:\MPASM_MPLINK_PIC18_LT_Branch_3_42\pic18-lt\cxx-framework\src\traditional\proc\p18f8723.asm
                 ECCP3DEL   0x000f69       data     extern E:\MPASM_MPLINK_PIC18_LT_Branch_3_42\pic18-lt\cxx-framework\src\traditional\proc\p18f8723.asm
             ECCP3DELbits   0x000f69       data     extern E:\MPASM_MPLINK_PIC18_LT_Branch_3_42\pic18-lt\cxx-framework\src\traditional\proc\p18f8723.asm
                    EEADR   0x000fa9       data     extern E:\MPASM_MPLINK_PIC18_LT_Branch_3_42\pic18-lt\cxx-framework\src\traditional\proc\p18f8723.asm
                   EEADRH   0x000faa       data     extern E:\MPASM_MPLINK_PIC18_LT_Branch_3_42\pic18-lt\cxx-framework\src\traditional\proc\p18f8723.asm
                   EECON1   0x000fa6       data     extern E:\MPASM_MPLINK_PIC18_LT_Branch_3_42\pic18-lt\cxx-framework\src\traditional\proc\p18f8723.asm
               EECON1bits   0x000fa6       data     extern E:\MPASM_MPLINK_PIC18_LT_Branch_3_42\pic18-lt\cxx-framework\src\traditional\proc\p18f8723.asm
                   EECON2   0x000fa7       data     extern E:\MPASM_MPLINK_PIC18_LT_Branch_3_42\pic18-lt\cxx-framework\src\traditional\proc\p18f8723.asm
                   EEDATA   0x000fa8       data     extern E:\MPASM_MPLINK_PIC18_LT_Branch_3_42\pic18-lt\cxx-framework\src\traditional\proc\p18f8723.asm
                 ENTREES1   0x0002e9       data     extern C:\Users\LFRAD\Documents\CMS2Luc\ProjetsNettoyesCMSGit\ProjetCarteMere\project\CMSModifV1SD.c
                 ENTREES2   0x0002ea       data     extern C:\Users\LFRAD\Documents\CMS2Luc\ProjetsNettoyesCMSGit\ProjetCarteMere\project\CMSModifV1SD.c
                    ERRMM   0x000f42       data     extern C:\Users\LFRAD\Documents\CMS2Luc\ProjetsNettoyesCMSGit\ProjetCarteMere\project\CMSModifV1SD.c
                     ETAT   0x00024d       data     extern C:\Users\LFRAD\Documents\CMS2Luc\ProjetsNettoyesCMSGit\ProjetCarteMere\project\CMSModifV1SD.c
   ETATZIZCRATIONAUTOMATE   0x000f3a       data     extern C:\Users\LFRAD\Documents\CMS2Luc\ProjetsNettoyesCMSGit\ProjetCarteMere\project\CMSModifV1SD.c
                  ETAT_IO   0x000f1f       data     extern C:\Users\LFRAD\Documents\CMS2Luc\ProjetsNettoyesCMSGit\ProjetCarteMere\project\CMSModifV1SD.c
                   FCYCLE   0x000f44       data     extern C:\Users\LFRAD\Documents\CMS2Luc\ProjetsNettoyesCMSGit\ProjetCarteMere\project\CMSModifV1SD.c
              FIRST_DEMAR   0x000f20       data     extern C:\Users\LFRAD\Documents\CMS2Luc\ProjetsNettoyesCMSGit\ProjetCarteMere\project\CMSModifV1SD.c
                 FONCTION   0x000261       data     extern C:\Users\LFRAD\Documents\CMS2Luc\ProjetsNettoyesCMSGit\ProjetCarteMere\project\CMSModifV1SD.c
 FONCTION_ACTIVATION_AUTO   0x000f1b       data     extern C:\Users\LFRAD\Documents\CMS2Luc\ProjetsNettoyesCMSGit\ProjetCarteMere\project\CMSModifV1SD.c
                     FSR0   0x000fe9       data     extern E:\MPASM_MPLINK_PIC18_LT_Branch_3_42\pic18-lt\cxx-framework\src\traditional\proc\p18f8723.asm
                    FSR0H   0x000fea       data     extern E:\MPASM_MPLINK_PIC18_LT_Branch_3_42\pic18-lt\cxx-framework\src\traditional\proc\p18f8723.asm
                    FSR0L   0x000fe9       data     extern E:\MPASM_MPLINK_PIC18_LT_Branch_3_42\pic18-lt\cxx-framework\src\traditional\proc\p18f8723.asm
                     FSR1   0x000fe1       data     extern E:\MPASM_MPLINK_PIC18_LT_Branch_3_42\pic18-lt\cxx-framework\src\traditional\proc\p18f8723.asm
                    FSR1H   0x000fe2       data     extern E:\MPASM_MPLINK_PIC18_LT_Branch_3_42\pic18-lt\cxx-framework\src\traditional\proc\p18f8723.asm
                    FSR1L   0x000fe1       data     extern E:\MPASM_MPLINK_PIC18_LT_Branch_3_42\pic18-lt\cxx-framework\src\traditional\proc\p18f8723.asm
                     FSR2   0x000fd9       data     extern E:\MPASM_MPLINK_PIC18_LT_Branch_3_42\pic18-lt\cxx-framework\src\traditional\proc\p18f8723.asm
                    FSR2H   0x000fda       data     extern E:\MPASM_MPLINK_PIC18_LT_Branch_3_42\pic18-lt\cxx-framework\src\traditional\proc\p18f8723.asm
                    FSR2L   0x000fd9       data     extern E:\MPASM_MPLINK_PIC18_LT_Branch_3_42\pic18-lt\cxx-framework\src\traditional\proc\p18f8723.asm
                    HEURE   0x0002eb       data     extern C:\Users\LFRAD\Documents\CMS2Luc\ProjetsNettoyesCMSGit\ProjetCarteMere\project\CMSModifV1SD.c
                       HH   0x00023b       data     extern C:\Users\LFRAD\Documents\CMS2Luc\ProjetsNettoyesCMSGit\ProjetCarteMere\project\CMSModifV1SD.c
                  HLVDCON   0x000fd2       data     extern E:\MPASM_MPLINK_PIC18_LT_Branch_3_42\pic18-lt\cxx-framework\src\traditional\proc\p18f8723.asm
              HLVDCONbits   0x000fd2       data     extern E:\MPASM_MPLINK_PIC18_LT_Branch_3_42\pic18-lt\cxx-framework\src\traditional\proc\p18f8723.asm
                  HORLOGE   0x000282       data     extern C:\Users\LFRAD\Documents\CMS2Luc\ProjetsNettoyesCMSGit\ProjetCarteMere\project\CMSModifV1SD.c
                      ID1   0x00025d       data     extern C:\Users\LFRAD\Documents\CMS2Luc\ProjetsNettoyesCMSGit\ProjetCarteMere\project\CMSModifV1SD.c
                      ID2   0x00025f       data     extern C:\Users\LFRAD\Documents\CMS2Luc\ProjetsNettoyesCMSGit\ProjetCarteMere\project\CMSModifV1SD.c
                    INDF0   0x000fef       data     extern E:\MPASM_MPLINK_PIC18_LT_Branch_3_42\pic18-lt\cxx-framework\src\traditional\proc\p18f8723.asm
                    INDF1   0x000fe7       data     extern E:\MPASM_MPLINK_PIC18_LT_Branch_3_42\pic18-lt\cxx-framework\src\traditional\proc\p18f8723.asm
                    INDF2   0x000fdf       data     extern E:\MPASM_MPLINK_PIC18_LT_Branch_3_42\pic18-lt\cxx-framework\src\traditional\proc\p18f8723.asm
       INFORMATION_ERREUR   0x00026c       data     extern C:\Users\LFRAD\Documents\CMS2Luc\ProjetsNettoyesCMSGit\ProjetCarteMere\project\CMSModifV1SD.c
              INSTRUCTION   0x0002a8       data     extern C:\Users\LFRAD\Documents\CMS2Luc\ProjetsNettoyesCMSGit\ProjetCarteMere\project\CMSModifV1SD.c
                   INTCON   0x000ff2       data     extern E:\MPASM_MPLINK_PIC18_LT_Branch_3_42\pic18-lt\cxx-framework\src\traditional\proc\p18f8723.asm
                  INTCON2   0x000ff1       data     extern E:\MPASM_MPLINK_PIC18_LT_Branch_3_42\pic18-lt\cxx-framework\src\traditional\proc\p18f8723.asm
              INTCON2bits   0x000ff1       data     extern E:\MPASM_MPLINK_PIC18_LT_Branch_3_42\pic18-lt\cxx-framework\src\traditional\proc\p18f8723.asm
                  INTCON3   0x000ff0       data     extern E:\MPASM_MPLINK_PIC18_LT_Branch_3_42\pic18-lt\cxx-framework\src\traditional\proc\p18f8723.asm
              INTCON3bits   0x000ff0       data     extern E:\MPASM_MPLINK_PIC18_LT_Branch_3_42\pic18-lt\cxx-framework\src\traditional\proc\p18f8723.asm
               INTCONbits   0x000ff2       data     extern E:\MPASM_MPLINK_PIC18_LT_Branch_3_42\pic18-lt\cxx-framework\src\traditional\proc\p18f8723.asm
                IOTRAVAIL   0x000f24       data     extern C:\Users\LFRAD\Documents\CMS2Luc\ProjetsNettoyesCMSGit\ProjetCarteMere\project\CMSModifV1SD.c
                     IPR1   0x000f9f       data     extern E:\MPASM_MPLINK_PIC18_LT_Branch_3_42\pic18-lt\cxx-framework\src\traditional\proc\p18f8723.asm
                 IPR1bits   0x000f9f       data     extern E:\MPASM_MPLINK_PIC18_LT_Branch_3_42\pic18-lt\cxx-framework\src\traditional\proc\p18f8723.asm
                     IPR2   0x000fa2       data     extern E:\MPASM_MPLINK_PIC18_LT_Branch_3_42\pic18-lt\cxx-framework\src\traditional\proc\p18f8723.asm
                 IPR2bits   0x000fa2       data     extern E:\MPASM_MPLINK_PIC18_LT_Branch_3_42\pic18-lt\cxx-framework\src\traditional\proc\p18f8723.asm
                     IPR3   0x000fa5       data     extern E:\MPASM_MPLINK_PIC18_LT_Branch_3_42\pic18-lt\cxx-framework\src\traditional\proc\p18f8723.asm
                 IPR3bits   0x000fa5       data     extern E:\MPASM_MPLINK_PIC18_LT_Branch_3_42\pic18-lt\cxx-framework\src\traditional\proc\p18f8723.asm
                       JJ   0x000237       data     extern C:\Users\LFRAD\Documents\CMS2Luc\ProjetsNettoyesCMSGit\ProjetCarteMere\project\CMSModifV1SD.c
                     JOUR   0x0002ef       data     extern C:\Users\LFRAD\Documents\CMS2Luc\ProjetsNettoyesCMSGit\ProjetCarteMere\project\CMSModifV1SD.c
                     LATA   0x000f89       data     extern E:\MPASM_MPLINK_PIC18_LT_Branch_3_42\pic18-lt\cxx-framework\src\traditional\proc\p18f8723.asm
                 LATAbits   0x000f89       data     extern E:\MPASM_MPLINK_PIC18_LT_Branch_3_42\pic18-lt\cxx-framework\src\traditional\proc\p18f8723.asm
                     LATB   0x000f8a       data     extern E:\MPASM_MPLINK_PIC18_LT_Branch_3_42\pic18-lt\cxx-framework\src\traditional\proc\p18f8723.asm
                 LATBbits   0x000f8a       data     extern E:\MPASM_MPLINK_PIC18_LT_Branch_3_42\pic18-lt\cxx-framework\src\traditional\proc\p18f8723.asm
                     LATC   0x000f8b       data     extern E:\MPASM_MPLINK_PIC18_LT_Branch_3_42\pic18-lt\cxx-framework\src\traditional\proc\p18f8723.asm
                 LATCbits   0x000f8b       data     extern E:\MPASM_MPLINK_PIC18_LT_Branch_3_42\pic18-lt\cxx-framework\src\traditional\proc\p18f8723.asm
                     LATD   0x000f8c       data     extern E:\MPASM_MPLINK_PIC18_LT_Branch_3_42\pic18-lt\cxx-framework\src\traditional\proc\p18f8723.asm
                 LATDbits   0x000f8c       data     extern E:\MPASM_MPLINK_PIC18_LT_Branch_3_42\pic18-lt\cxx-framework\src\traditional\proc\p18f8723.asm
                     LATE   0x000f8d       data     extern E:\MPASM_MPLINK_PIC18_LT_Branch_3_42\pic18-lt\cxx-framework\src\traditional\proc\p18f8723.asm
                 LATEbits   0x000f8d       data     extern E:\MPASM_MPLINK_PIC18_LT_Branch_3_42\pic18-lt\cxx-framework\src\traditional\proc\p18f8723.asm
                     LATF   0x000f8e       data     extern E:\MPASM_MPLINK_PIC18_LT_Branch_3_42\pic18-lt\cxx-framework\src\traditional\proc\p18f8723.asm
                 LATFbits   0x000f8e       data     extern E:\MPASM_MPLINK_PIC18_LT_Branch_3_42\pic18-lt\cxx-framework\src\traditional\proc\p18f8723.asm
                     LATG   0x000f8f       data     extern E:\MPASM_MPLINK_PIC18_LT_Branch_3_42\pic18-lt\cxx-framework\src\traditional\proc\p18f8723.asm
                 LATGbits   0x000f8f       data     extern E:\MPASM_MPLINK_PIC18_LT_Branch_3_42\pic18-lt\cxx-framework\src\traditional\proc\p18f8723.asm
                     LATH   0x000f90       data     extern E:\MPASM_MPLINK_PIC18_LT_Branch_3_42\pic18-lt\cxx-framework\src\traditional\proc\p18f8723.asm
                 LATHbits   0x000f90       data     extern E:\MPASM_MPLINK_PIC18_LT_Branch_3_42\pic18-lt\cxx-framework\src\traditional\proc\p18f8723.asm
                     LATJ   0x000f91       data     extern E:\MPASM_MPLINK_PIC18_LT_Branch_3_42\pic18-lt\cxx-framework\src\traditional\proc\p18f8723.asm
                 LATJbits   0x000f91       data     extern E:\MPASM_MPLINK_PIC18_LT_Branch_3_42\pic18-lt\cxx-framework\src\traditional\proc\p18f8723.asm
                   LVDCON   0x000fd2       data     extern E:\MPASM_MPLINK_PIC18_LT_Branch_3_42\pic18-lt\cxx-framework\src\traditional\proc\p18f8723.asm
               LVDCONbits   0x000fd2       data     extern E:\MPASM_MPLINK_PIC18_LT_Branch_3_42\pic18-lt\cxx-framework\src\traditional\proc\p18f8723.asm
                  MAJBLOC   0x000f40       data     extern C:\Users\LFRAD\Documents\CMS2Luc\ProjetsNettoyesCMSGit\ProjetCarteMere\project\CMSModifV1SD.c
                  MAXBITE   0x000f3f       data     extern C:\Users\LFRAD\Documents\CMS2Luc\ProjetsNettoyesCMSGit\ProjetCarteMere\project\CMSModifV1SD.c
                   MEMCON   0x000f9c       data     extern E:\MPASM_MPLINK_PIC18_LT_Branch_3_42\pic18-lt\cxx-framework\src\traditional\proc\p18f8723.asm
               MEMCONbits   0x000f9c       data     extern E:\MPASM_MPLINK_PIC18_LT_Branch_3_42\pic18-lt\cxx-framework\src\traditional\proc\p18f8723.asm
              MINIRESETRI   0x000f35       data     extern C:\Users\LFRAD\Documents\CMS2Luc\ProjetsNettoyesCMSGit\ProjetCarteMere\project\CMSModifV1SD.c
                   MINUTE   0x0002ec       data     extern C:\Users\LFRAD\Documents\CMS2Luc\ProjetsNettoyesCMSGit\ProjetCarteMere\project\CMSModifV1SD.c
                       MM   0x000239       data     extern C:\Users\LFRAD\Documents\CMS2Luc\ProjetsNettoyesCMSGit\ProjetCarteMere\project\CMSModifV1SD.c
                MODERAPID   0x000f21       data     extern C:\Users\LFRAD\Documents\CMS2Luc\ProjetsNettoyesCMSGit\ProjetCarteMere\project\CMSModifV1SD.c
                     MOIS   0x0002ee       data     extern C:\Users\LFRAD\Documents\CMS2Luc\ProjetsNettoyesCMSGit\ProjetCarteMere\project\CMSModifV1SD.c
                     NBMM   0x000f43       data     extern C:\Users\LFRAD\Documents\CMS2Luc\ProjetsNettoyesCMSGit\ProjetCarteMere\project\CMSModifV1SD.c
       NBRECAPTEURS_CABLE   0x000280       data     extern C:\Users\LFRAD\Documents\CMS2Luc\ProjetsNettoyesCMSGit\ProjetCarteMere\project\CMSModifV1SD.c
            NBREDEMANDEIO   0x000f29       data     extern C:\Users\LFRAD\Documents\CMS2Luc\ProjetsNettoyesCMSGit\ProjetCarteMere\project\CMSModifV1SD.c
              NORECEPTION   0x0002e2       data     extern C:\Users\LFRAD\Documents\CMS2Luc\ProjetsNettoyesCMSGit\ProjetCarteMere\project\CMSModifV1SD.c
              NUMEROCARTE   0x000f28       data     extern C:\Users\LFRAD\Documents\CMS2Luc\ProjetsNettoyesCMSGit\ProjetCarteMere\project\CMSModifV1SD.c
             OEIL_CAPTEUR   0x00029d       data     extern C:\Users\LFRAD\Documents\CMS2Luc\ProjetsNettoyesCMSGit\ProjetCarteMere\project\CMSModifV1SD.c
                   OSCCON   0x000fd3       data     extern E:\MPASM_MPLINK_PIC18_LT_Branch_3_42\pic18-lt\cxx-framework\src\traditional\proc\p18f8723.asm
               OSCCONbits   0x000fd3       data     extern E:\MPASM_MPLINK_PIC18_LT_Branch_3_42\pic18-lt\cxx-framework\src\traditional\proc\p18f8723.asm
                  OSCTUNE   0x000f9b       data     extern E:\MPASM_MPLINK_PIC18_LT_Branch_3_42\pic18-lt\cxx-framework\src\traditional\proc\p18f8723.asm
              OSCTUNEbits   0x000f9b       data     extern E:\MPASM_MPLINK_PIC18_LT_Branch_3_42\pic18-lt\cxx-framework\src\traditional\proc\p18f8723.asm
                     PAGE   0x0002a2       data     extern C:\Users\LFRAD\Documents\CMS2Luc\ProjetsNettoyesCMSGit\ProjetCarteMere\project\CMSModifV1SD.c
                  PASDE_S   0x000f25       data     extern C:\Users\LFRAD\Documents\CMS2Luc\ProjetsNettoyesCMSGit\ProjetCarteMere\project\CMSModifV1SD.c
                       PC   0x000ff9       data     extern E:\MPASM_MPLINK_PIC18_LT_Branch_3_42\pic18-lt\cxx-framework\src\traditional\proc\p18f8723.asm
                      PCL   0x000ff9       data     extern E:\MPASM_MPLINK_PIC18_LT_Branch_3_42\pic18-lt\cxx-framework\src\traditional\proc\p18f8723.asm
                   PCLATH   0x000ffa       data     extern E:\MPASM_MPLINK_PIC18_LT_Branch_3_42\pic18-lt\cxx-framework\src\traditional\proc\p18f8723.asm
                   PCLATU   0x000ffb       data     extern E:\MPASM_MPLINK_PIC18_LT_Branch_3_42\pic18-lt\cxx-framework\src\traditional\proc\p18f8723.asm
                     PIE1   0x000f9d       data     extern E:\MPASM_MPLINK_PIC18_LT_Branch_3_42\pic18-lt\cxx-framework\src\traditional\proc\p18f8723.asm
                 PIE1bits   0x000f9d       data     extern E:\MPASM_MPLINK_PIC18_LT_Branch_3_42\pic18-lt\cxx-framework\src\traditional\proc\p18f8723.asm
                     PIE2   0x000fa0       data     extern E:\MPASM_MPLINK_PIC18_LT_Branch_3_42\pic18-lt\cxx-framework\src\traditional\proc\p18f8723.asm
                 PIE2bits   0x000fa0       data     extern E:\MPASM_MPLINK_PIC18_LT_Branch_3_42\pic18-lt\cxx-framework\src\traditional\proc\p18f8723.asm
                     PIE3   0x000fa3       data     extern E:\MPASM_MPLINK_PIC18_LT_Branch_3_42\pic18-lt\cxx-framework\src\traditional\proc\p18f8723.asm
                 PIE3bits   0x000fa3       data     extern E:\MPASM_MPLINK_PIC18_LT_Branch_3_42\pic18-lt\cxx-framework\src\traditional\proc\p18f8723.asm
                     PIR1   0x000f9e       data     extern E:\MPASM_MPLINK_PIC18_LT_Branch_3_42\pic18-lt\cxx-framework\src\traditional\proc\p18f8723.asm
                 PIR1bits   0x000f9e       data     extern E:\MPASM_MPLINK_PIC18_LT_Branch_3_42\pic18-lt\cxx-framework\src\traditional\proc\p18f8723.asm
                     PIR2   0x000fa1       data     extern E:\MPASM_MPLINK_PIC18_LT_Branch_3_42\pic18-lt\cxx-framework\src\traditional\proc\p18f8723.asm
                 PIR2bits   0x000fa1       data     extern E:\MPASM_MPLINK_PIC18_LT_Branch_3_42\pic18-lt\cxx-framework\src\traditional\proc\p18f8723.asm
                     PIR3   0x000fa4       data     extern E:\MPASM_MPLINK_PIC18_LT_Branch_3_42\pic18-lt\cxx-framework\src\traditional\proc\p18f8723.asm
                 PIR3bits   0x000fa4       data     extern E:\MPASM_MPLINK_PIC18_LT_Branch_3_42\pic18-lt\cxx-framework\src\traditional\proc\p18f8723.asm
                   PLUSW0   0x000feb       data     extern E:\MPASM_MPLINK_PIC18_LT_Branch_3_42\pic18-lt\cxx-framework\src\traditional\proc\p18f8723.asm
                   PLUSW1   0x000fe3       data     extern E:\MPASM_MPLINK_PIC18_LT_Branch_3_42\pic18-lt\cxx-framework\src\traditional\proc\p18f8723.asm
                   PLUSW2   0x000fdb       data     extern E:\MPASM_MPLINK_PIC18_LT_Branch_3_42\pic18-lt\cxx-framework\src\traditional\proc\p18f8723.asm
              POINT_ROSEE   0x0003aa       data     extern C:\Users\LFRAD\Documents\CMS2Luc\ProjetsNettoyesCMSGit\ProjetCarteMere\project\CMSModifV1SD.c
                    PORTA   0x000f80       data     extern E:\MPASM_MPLINK_PIC18_LT_Branch_3_42\pic18-lt\cxx-framework\src\traditional\proc\p18f8723.asm
                PORTAbits   0x000f80       data     extern E:\MPASM_MPLINK_PIC18_LT_Branch_3_42\pic18-lt\cxx-framework\src\traditional\proc\p18f8723.asm
                    PORTB   0x000f81       data     extern E:\MPASM_MPLINK_PIC18_LT_Branch_3_42\pic18-lt\cxx-framework\src\traditional\proc\p18f8723.asm
                PORTBbits   0x000f81       data     extern E:\MPASM_MPLINK_PIC18_LT_Branch_3_42\pic18-lt\cxx-framework\src\traditional\proc\p18f8723.asm
                    PORTC   0x000f82       data     extern E:\MPASM_MPLINK_PIC18_LT_Branch_3_42\pic18-lt\cxx-framework\src\traditional\proc\p18f8723.asm
                PORTCbits   0x000f82       data     extern E:\MPASM_MPLINK_PIC18_LT_Branch_3_42\pic18-lt\cxx-framework\src\traditional\proc\p18f8723.asm
                    PORTD   0x000f83       data     extern E:\MPASM_MPLINK_PIC18_LT_Branch_3_42\pic18-lt\cxx-framework\src\traditional\proc\p18f8723.asm
                PORTDbits   0x000f83       data     extern E:\MPASM_MPLINK_PIC18_LT_Branch_3_42\pic18-lt\cxx-framework\src\traditional\proc\p18f8723.asm
                    PORTE   0x000f84       data     extern E:\MPASM_MPLINK_PIC18_LT_Branch_3_42\pic18-lt\cxx-framework\src\traditional\proc\p18f8723.asm
                PORTEbits   0x000f84       data     extern E:\MPASM_MPLINK_PIC18_LT_Branch_3_42\pic18-lt\cxx-framework\src\traditional\proc\p18f8723.asm
                    PORTF   0x000f85       data     extern E:\MPASM_MPLINK_PIC18_LT_Branch_3_42\pic18-lt\cxx-framework\src\traditional\proc\p18f8723.asm
                PORTFbits   0x000f85       data     extern E:\MPASM_MPLINK_PIC18_LT_Branch_3_42\pic18-lt\cxx-framework\src\traditional\proc\p18f8723.asm
                    PORTG   0x000f86       data     extern E:\MPASM_MPLINK_PIC18_LT_Branch_3_42\pic18-lt\cxx-framework\src\traditional\proc\p18f8723.asm
                PORTGbits   0x000f86       data     extern E:\MPASM_MPLINK_PIC18_LT_Branch_3_42\pic18-lt\cxx-framework\src\traditional\proc\p18f8723.asm
                    PORTH   0x000f87       data     extern E:\MPASM_MPLINK_PIC18_LT_Branch_3_42\pic18-lt\cxx-framework\src\traditional\proc\p18f8723.asm
                PORTHbits   0x000f87       data     extern E:\MPASM_MPLINK_PIC18_LT_Branch_3_42\pic18-lt\cxx-framework\src\traditional\proc\p18f8723.asm
                    PORTJ   0x000f88       data     extern E:\MPASM_MPLINK_PIC18_LT_Branch_3_42\pic18-lt\cxx-framework\src\traditional\proc\p18f8723.asm
                PORTJbits   0x000f88       data     extern E:\MPASM_MPLINK_PIC18_LT_Branch_3_42\pic18-lt\cxx-framework\src\traditional\proc\p18f8723.asm
                      POS   0x000242       data     extern C:\Users\LFRAD\Documents\CMS2Luc\ProjetsNettoyesCMSGit\ProjetCarteMere\project\CMSModifV1SD.c
                 POSTDEC0   0x000fed       data     extern E:\MPASM_MPLINK_PIC18_LT_Branch_3_42\pic18-lt\cxx-framework\src\traditional\proc\p18f8723.asm
                 POSTDEC1   0x000fe5       data     extern E:\MPASM_MPLINK_PIC18_LT_Branch_3_42\pic18-lt\cxx-framework\src\traditional\proc\p18f8723.asm
                 POSTDEC2   0x000fdd       data     extern E:\MPASM_MPLINK_PIC18_LT_Branch_3_42\pic18-lt\cxx-framework\src\traditional\proc\p18f8723.asm
                 POSTINC0   0x000fee       data     extern E:\MPASM_MPLINK_PIC18_LT_Branch_3_42\pic18-lt\cxx-framework\src\traditional\proc\p18f8723.asm
                 POSTINC1   0x000fe6       data     extern E:\MPASM_MPLINK_PIC18_LT_Branch_3_42\pic18-lt\cxx-framework\src\traditional\proc\p18f8723.asm
                 POSTINC2   0x000fde       data     extern E:\MPASM_MPLINK_PIC18_LT_Branch_3_42\pic18-lt\cxx-framework\src\traditional\proc\p18f8723.asm
                      PR2   0x000fcb       data     extern E:\MPASM_MPLINK_PIC18_LT_Branch_3_42\pic18-lt\cxx-framework\src\traditional\proc\p18f8723.asm
                      PR4   0x000f77       data     extern E:\MPASM_MPLINK_PIC18_LT_Branch_3_42\pic18-lt\cxx-framework\src\traditional\proc\p18f8723.asm
                  PREINC0   0x000fec       data     extern E:\MPASM_MPLINK_PIC18_LT_Branch_3_42\pic18-lt\cxx-framework\src\traditional\proc\p18f8723.asm
                  PREINC1   0x000fe4       data     extern E:\MPASM_MPLINK_PIC18_LT_Branch_3_42\pic18-lt\cxx-framework\src\traditional\proc\p18f8723.asm
                  PREINC2   0x000fdc       data     extern E:\MPASM_MPLINK_PIC18_LT_Branch_3_42\pic18-lt\cxx-framework\src\traditional\proc\p18f8723.asm
          PRESENCEDEBITSD   0x000f2a       data     extern C:\Users\LFRAD\Documents\CMS2Luc\ProjetsNettoyesCMSGit\ProjetCarteMere\project\CMSModifV1SD.c
            PRESENCE_220V   0x0003da       data     extern C:\Users\LFRAD\Documents\CMS2Luc\ProjetsNettoyesCMSGit\ProjetCarteMere\project\CMSModifV1SD.c
             PRESENCE_48V   0x0003e0       data     extern C:\Users\LFRAD\Documents\CMS2Luc\ProjetsNettoyesCMSGit\ProjetCarteMere\project\CMSModifV1SD.c
             PRIO_AUTO_IO   0x000281       data     extern C:\Users\LFRAD\Documents\CMS2Luc\ProjetsNettoyesCMSGit\ProjetCarteMere\project\CMSModifV1SD.c
                     PROD   0x000ff3       data     extern E:\MPASM_MPLINK_PIC18_LT_Branch_3_42\pic18-lt\cxx-framework\src\traditional\proc\p18f8723.asm
                    PRODH   0x000ff4       data     extern E:\MPASM_MPLINK_PIC18_LT_Branch_3_42\pic18-lt\cxx-framework\src\traditional\proc\p18f8723.asm
                    PRODL   0x000ff3       data     extern E:\MPASM_MPLINK_PIC18_LT_Branch_3_42\pic18-lt\cxx-framework\src\traditional\proc\p18f8723.asm
                   PSPCON   0x000fb0       data     extern E:\MPASM_MPLINK_PIC18_LT_Branch_3_42\pic18-lt\cxx-framework\src\traditional\proc\p18f8723.asm
               PSPCONbits   0x000fb0       data     extern E:\MPASM_MPLINK_PIC18_LT_Branch_3_42\pic18-lt\cxx-framework\src\traditional\proc\p18f8723.asm
              P_RESERVOIR   0x00037d       data     extern C:\Users\LFRAD\Documents\CMS2Luc\ProjetsNettoyesCMSGit\ProjetCarteMere\project\CMSModifV1SD.c
                P_SECOURS   0x00039b       data     extern C:\Users\LFRAD\Documents\CMS2Luc\ProjetsNettoyesCMSGit\ProjetCarteMere\project\CMSModifV1SD.c
                 P_SORTIE   0x00038c       data     extern C:\Users\LFRAD\Documents\CMS2Luc\ProjetsNettoyesCMSGit\ProjetCarteMere\project\CMSModifV1SD.c
                  R1NOREP   0x000f2b       data     extern C:\Users\LFRAD\Documents\CMS2Luc\ProjetsNettoyesCMSGit\ProjetCarteMere\project\CMSModifV1SD.c
                  R2NOREP   0x000f2c       data     extern C:\Users\LFRAD\Documents\CMS2Luc\ProjetsNettoyesCMSGit\ProjetCarteMere\project\CMSModifV1SD.c
                  R3NOREP   0x000f2d       data     extern C:\Users\LFRAD\Documents\CMS2Luc\ProjetsNettoyesCMSGit\ProjetCarteMere\project\CMSModifV1SD.c
                  R4NOREP   0x000f2e       data     extern C:\Users\LFRAD\Documents\CMS2Luc\ProjetsNettoyesCMSGit\ProjetCarteMere\project\CMSModifV1SD.c
                  R5NOREP   0x000f2f       data     extern C:\Users\LFRAD\Documents\CMS2Luc\ProjetsNettoyesCMSGit\ProjetCarteMere\project\CMSModifV1SD.c
                     RCON   0x000fd0       data     extern E:\MPASM_MPLINK_PIC18_LT_Branch_3_42\pic18-lt\cxx-framework\src\traditional\proc\p18f8723.asm
                 RCONbits   0x000fd0       data     extern E:\MPASM_MPLINK_PIC18_LT_Branch_3_42\pic18-lt\cxx-framework\src\traditional\proc\p18f8723.asm
                    RCREG   0x000fae       data     extern E:\MPASM_MPLINK_PIC18_LT_Branch_3_42\pic18-lt\cxx-framework\src\traditional\proc\p18f8723.asm
                   RCREG1   0x000fae       data     extern E:\MPASM_MPLINK_PIC18_LT_Branch_3_42\pic18-lt\cxx-framework\src\traditional\proc\p18f8723.asm
                   RCREG2   0x000f6e       data     extern E:\MPASM_MPLINK_PIC18_LT_Branch_3_42\pic18-lt\cxx-framework\src\traditional\proc\p18f8723.asm
                    RCSTA   0x000fab       data     extern E:\MPASM_MPLINK_PIC18_LT_Branch_3_42\pic18-lt\cxx-framework\src\traditional\proc\p18f8723.asm
                   RCSTA1   0x000fab       data     extern E:\MPASM_MPLINK_PIC18_LT_Branch_3_42\pic18-lt\cxx-framework\src\traditional\proc\p18f8723.asm
               RCSTA1bits   0x000fab       data     extern E:\MPASM_MPLINK_PIC18_LT_Branch_3_42\pic18-lt\cxx-framework\src\traditional\proc\p18f8723.asm
                   RCSTA2   0x000f6b       data     extern E:\MPASM_MPLINK_PIC18_LT_Branch_3_42\pic18-lt\cxx-framework\src\traditional\proc\p18f8723.asm
               RCSTA2bits   0x000f6b       data     extern E:\MPASM_MPLINK_PIC18_LT_Branch_3_42\pic18-lt\cxx-framework\src\traditional\proc\p18f8723.asm
                RCSTAbits   0x000fab       data     extern E:\MPASM_MPLINK_PIC18_LT_Branch_3_42\pic18-lt\cxx-framework\src\traditional\proc\p18f8723.asm
             RESCRUTATION   0x000f27       data     extern C:\Users\LFRAD\Documents\CMS2Luc\ProjetsNettoyesCMSGit\ProjetCarteMere\project\CMSModifV1SD.c
             SAVAUTOCYCLE   0x000f3e       data     extern C:\Users\LFRAD\Documents\CMS2Luc\ProjetsNettoyesCMSGit\ProjetCarteMere\project\CMSModifV1SD.c
                   SAVTAB   0x000f00       data     extern C:\Users\LFRAD\Documents\CMS2Luc\ProjetsNettoyesCMSGit\ProjetCarteMere\project\CMSModifV1SD.c
                  SECONDE   0x0002ed       data     extern C:\Users\LFRAD\Documents\CMS2Luc\ProjetsNettoyesCMSGit\ProjetCarteMere\project\CMSModifV1SD.c
                    SEUIL   0x000253       data     extern C:\Users\LFRAD\Documents\CMS2Luc\ProjetsNettoyesCMSGit\ProjetCarteMere\project\CMSModifV1SD.c
                     SIGN   0x000000       data     extern E:\MPASM_MPLINK_PIC18_LT_Branch_3_42\pic18-lt\cxx-framework\src\traditional\math\cmath18.asm
                    SPBRG   0x000faf       data     extern E:\MPASM_MPLINK_PIC18_LT_Branch_3_42\pic18-lt\cxx-framework\src\traditional\proc\p18f8723.asm
                   SPBRG1   0x000faf       data     extern E:\MPASM_MPLINK_PIC18_LT_Branch_3_42\pic18-lt\cxx-framework\src\traditional\proc\p18f8723.asm
                   SPBRG2   0x000f6f       data     extern E:\MPASM_MPLINK_PIC18_LT_Branch_3_42\pic18-lt\cxx-framework\src\traditional\proc\p18f8723.asm
                   SPBRGH   0x000f7f       data     extern E:\MPASM_MPLINK_PIC18_LT_Branch_3_42\pic18-lt\cxx-framework\src\traditional\proc\p18f8723.asm
                  SPBRGH1   0x000f7f       data     extern E:\MPASM_MPLINK_PIC18_LT_Branch_3_42\pic18-lt\cxx-framework\src\traditional\proc\p18f8723.asm
                  SPBRGH2   0x000f7d       data     extern E:\MPASM_MPLINK_PIC18_LT_Branch_3_42\pic18-lt\cxx-framework\src\traditional\proc\p18f8723.asm
                  SSP1ADD   0x000fc8       data     extern E:\MPASM_MPLINK_PIC18_LT_Branch_3_42\pic18-lt\cxx-framework\src\traditional\proc\p18f8723.asm
                  SSP1BUF   0x000fc9       data     extern E:\MPASM_MPLINK_PIC18_LT_Branch_3_42\pic18-lt\cxx-framework\src\traditional\proc\p18f8723.asm
                 SSP1CON1   0x000fc6       data     extern E:\MPASM_MPLINK_PIC18_LT_Branch_3_42\pic18-lt\cxx-framework\src\traditional\proc\p18f8723.asm
             SSP1CON1bits   0x000fc6       data     extern E:\MPASM_MPLINK_PIC18_LT_Branch_3_42\pic18-lt\cxx-framework\src\traditional\proc\p18f8723.asm
                 SSP1CON2   0x000fc5       data     extern E:\MPASM_MPLINK_PIC18_LT_Branch_3_42\pic18-lt\cxx-framework\src\traditional\proc\p18f8723.asm
             SSP1CON2bits   0x000fc5       data     extern E:\MPASM_MPLINK_PIC18_LT_Branch_3_42\pic18-lt\cxx-framework\src\traditional\proc\p18f8723.asm
                 SSP1STAT   0x000fc7       data     extern E:\MPASM_MPLINK_PIC18_LT_Branch_3_42\pic18-lt\cxx-framework\src\traditional\proc\p18f8723.asm
             SSP1STATbits   0x000fc7       data     extern E:\MPASM_MPLINK_PIC18_LT_Branch_3_42\pic18-lt\cxx-framework\src\traditional\proc\p18f8723.asm
                  SSP2ADD   0x000f65       data     extern E:\MPASM_MPLINK_PIC18_LT_Branch_3_42\pic18-lt\cxx-framework\src\traditional\proc\p18f8723.asm
                  SSP2BUF   0x000f66       data     extern E:\MPASM_MPLINK_PIC18_LT_Branch_3_42\pic18-lt\cxx-framework\src\traditional\proc\p18f8723.asm
                 SSP2CON1   0x000f63       data     extern E:\MPASM_MPLINK_PIC18_LT_Branch_3_42\pic18-lt\cxx-framework\src\traditional\proc\p18f8723.asm
             SSP2CON1bits   0x000f63       data     extern E:\MPASM_MPLINK_PIC18_LT_Branch_3_42\pic18-lt\cxx-framework\src\traditional\proc\p18f8723.asm
                 SSP2CON2   0x000f62       data     extern E:\MPASM_MPLINK_PIC18_LT_Branch_3_42\pic18-lt\cxx-framework\src\traditional\proc\p18f8723.asm
             SSP2CON2bits   0x000f62       data     extern E:\MPASM_MPLINK_PIC18_LT_Branch_3_42\pic18-lt\cxx-framework\src\traditional\proc\p18f8723.asm
                 SSP2STAT   0x000f64       data     extern E:\MPASM_MPLINK_PIC18_LT_Branch_3_42\pic18-lt\cxx-framework\src\traditional\proc\p18f8723.asm
             SSP2STATbits   0x000f64       data     extern E:\MPASM_MPLINK_PIC18_LT_Branch_3_42\pic18-lt\cxx-framework\src\traditional\proc\p18f8723.asm
                   SSPADD   0x000fc8       data     extern E:\MPASM_MPLINK_PIC18_LT_Branch_3_42\pic18-lt\cxx-framework\src\traditional\proc\p18f8723.asm
                   SSPBUF   0x000fc9       data     extern E:\MPASM_MPLINK_PIC18_LT_Branch_3_42\pic18-lt\cxx-framework\src\traditional\proc\p18f8723.asm
                  SSPCON1   0x000fc6       data     extern E:\MPASM_MPLINK_PIC18_LT_Branch_3_42\pic18-lt\cxx-framework\src\traditional\proc\p18f8723.asm
              SSPCON1bits   0x000fc6       data     extern E:\MPASM_MPLINK_PIC18_LT_Branch_3_42\pic18-lt\cxx-framework\src\traditional\proc\p18f8723.asm
                  SSPCON2   0x000fc5       data     extern E:\MPASM_MPLINK_PIC18_LT_Branch_3_42\pic18-lt\cxx-framework\src\traditional\proc\p18f8723.asm
              SSPCON2bits   0x000fc5       data     extern E:\MPASM_MPLINK_PIC18_LT_Branch_3_42\pic18-lt\cxx-framework\src\traditional\proc\p18f8723.asm
                  SSPSTAT   0x000fc7       data     extern E:\MPASM_MPLINK_PIC18_LT_Branch_3_42\pic18-lt\cxx-framework\src\traditional\proc\p18f8723.asm
              SSPSTATbits   0x000fc7       data     extern E:\MPASM_MPLINK_PIC18_LT_Branch_3_42\pic18-lt\cxx-framework\src\traditional\proc\p18f8723.asm
                    START   0x00025c       data     extern C:\Users\LFRAD\Documents\CMS2Luc\ProjetsNettoyesCMSGit\ProjetCarteMere\project\CMSModifV1SD.c
                   STATUS   0x000fd8       data     extern E:\MPASM_MPLINK_PIC18_LT_Branch_3_42\pic18-lt\cxx-framework\src\traditional\proc\p18f8723.asm
               STATUSbits   0x000fd8       data     extern E:\MPASM_MPLINK_PIC18_LT_Branch_3_42\pic18-lt\cxx-framework\src\traditional\proc\p18f8723.asm
                   STKPTR   0x000ffc       data     extern E:\MPASM_MPLINK_PIC18_LT_Branch_3_42\pic18-lt\cxx-framework\src\traditional\proc\p18f8723.asm
               STKPTRbits   0x000ffc       data     extern E:\MPASM_MPLINK_PIC18_LT_Branch_3_42\pic18-lt\cxx-framework\src\traditional\proc\p18f8723.asm
                     STOP   0x000269       data     extern C:\Users\LFRAD\Documents\CMS2Luc\ProjetsNettoyesCMSGit\ProjetCarteMere\project\CMSModifV1SD.c
                    T0CON   0x000fd5       data     extern E:\MPASM_MPLINK_PIC18_LT_Branch_3_42\pic18-lt\cxx-framework\src\traditional\proc\p18f8723.asm
                T0CONbits   0x000fd5       data     extern E:\MPASM_MPLINK_PIC18_LT_Branch_3_42\pic18-lt\cxx-framework\src\traditional\proc\p18f8723.asm
                    T1CON   0x000fcd       data     extern E:\MPASM_MPLINK_PIC18_LT_Branch_3_42\pic18-lt\cxx-framework\src\traditional\proc\p18f8723.asm
                T1CONbits   0x000fcd       data     extern E:\MPASM_MPLINK_PIC18_LT_Branch_3_42\pic18-lt\cxx-framework\src\traditional\proc\p18f8723.asm
                    T2CON   0x000fca       data     extern E:\MPASM_MPLINK_PIC18_LT_Branch_3_42\pic18-lt\cxx-framework\src\traditional\proc\p18f8723.asm
                T2CONbits   0x000fca       data     extern E:\MPASM_MPLINK_PIC18_LT_Branch_3_42\pic18-lt\cxx-framework\src\traditional\proc\p18f8723.asm
                    T3CON   0x000fb1       data     extern E:\MPASM_MPLINK_PIC18_LT_Branch_3_42\pic18-lt\cxx-framework\src\traditional\proc\p18f8723.asm
                T3CONbits   0x000fb1       data     extern E:\MPASM_MPLINK_PIC18_LT_Branch_3_42\pic18-lt\cxx-framework\src\traditional\proc\p18f8723.asm
                    T4CON   0x000f76       data     extern E:\MPASM_MPLINK_PIC18_LT_Branch_3_42\pic18-lt\cxx-framework\src\traditional\proc\p18f8723.asm
                T4CONbits   0x000f76       data     extern E:\MPASM_MPLINK_PIC18_LT_Branch_3_42\pic18-lt\cxx-framework\src\traditional\proc\p18f8723.asm
                   TABLAT   0x000ff5       data     extern E:\MPASM_MPLINK_PIC18_LT_Branch_3_42\pic18-lt\cxx-framework\src\traditional\proc\p18f8723.asm
                   TBLPTR   0x000ff6       data     extern E:\MPASM_MPLINK_PIC18_LT_Branch_3_42\pic18-lt\cxx-framework\src\traditional\proc\p18f8723.asm
                  TBLPTRH   0x000ff7       data     extern E:\MPASM_MPLINK_PIC18_LT_Branch_3_42\pic18-lt\cxx-framework\src\traditional\proc\p18f8723.asm
                  TBLPTRL   0x000ff6       data     extern E:\MPASM_MPLINK_PIC18_LT_Branch_3_42\pic18-lt\cxx-framework\src\traditional\proc\p18f8723.asm
                  TBLPTRU   0x000ff8       data     extern E:\MPASM_MPLINK_PIC18_LT_Branch_3_42\pic18-lt\cxx-framework\src\traditional\proc\p18f8723.asm
       TEMPS_CYCLE_MOTEUR   0x0003c0       data     extern C:\Users\LFRAD\Documents\CMS2Luc\ProjetsNettoyesCMSGit\ProjetCarteMere\project\CMSModifV1SD.c
             TEMPS_MOTEUR   0x0003cb       data     extern C:\Users\LFRAD\Documents\CMS2Luc\ProjetsNettoyesCMSGit\ProjetCarteMere\project\CMSModifV1SD.c
                TESTCYCLE   0x000f45       data     extern C:\Users\LFRAD\Documents\CMS2Luc\ProjetsNettoyesCMSGit\ProjetCarteMere\project\CMSModifV1SD.c
             TIMEOUTCYCLE   0x000f37       data     extern C:\Users\LFRAD\Documents\CMS2Luc\ProjetsNettoyesCMSGit\ProjetCarteMere\project\CMSModifV1SD.c
                      TMP   0x000300       data     extern C:\Users\LFRAD\Documents\CMS2Luc\ProjetsNettoyesCMSGit\ProjetCarteMere\project\CMSModifV1SD.c
                     TMPI   0x0002e7       data     extern C:\Users\LFRAD\Documents\CMS2Luc\ProjetsNettoyesCMSGit\ProjetCarteMere\project\CMSModifV1SD.c
                    TMR0H   0x000fd7       data     extern E:\MPASM_MPLINK_PIC18_LT_Branch_3_42\pic18-lt\cxx-framework\src\traditional\proc\p18f8723.asm
                    TMR0L   0x000fd6       data     extern E:\MPASM_MPLINK_PIC18_LT_Branch_3_42\pic18-lt\cxx-framework\src\traditional\proc\p18f8723.asm
                    TMR1H   0x000fcf       data     extern E:\MPASM_MPLINK_PIC18_LT_Branch_3_42\pic18-lt\cxx-framework\src\traditional\proc\p18f8723.asm
                    TMR1L   0x000fce       data     extern E:\MPASM_MPLINK_PIC18_LT_Branch_3_42\pic18-lt\cxx-framework\src\traditional\proc\p18f8723.asm
                     TMR2   0x000fcc       data     extern E:\MPASM_MPLINK_PIC18_LT_Branch_3_42\pic18-lt\cxx-framework\src\traditional\proc\p18f8723.asm
                    TMR3H   0x000fb3       data     extern E:\MPASM_MPLINK_PIC18_LT_Branch_3_42\pic18-lt\cxx-framework\src\traditional\proc\p18f8723.asm
                    TMR3L   0x000fb2       data     extern E:\MPASM_MPLINK_PIC18_LT_Branch_3_42\pic18-lt\cxx-framework\src\traditional\proc\p18f8723.asm
                     TMR4   0x000f78       data     extern E:\MPASM_MPLINK_PIC18_LT_Branch_3_42\pic18-lt\cxx-framework\src\traditional\proc\p18f8723.asm
                      TOS   0x000ffd       data     extern E:\MPASM_MPLINK_PIC18_LT_Branch_3_42\pic18-lt\cxx-framework\src\traditional\proc\p18f8723.asm
                     TOSH   0x000ffe       data     extern E:\MPASM_MPLINK_PIC18_LT_Branch_3_42\pic18-lt\cxx-framework\src\traditional\proc\p18f8723.asm
                     TOSL   0x000ffd       data     extern E:\MPASM_MPLINK_PIC18_LT_Branch_3_42\pic18-lt\cxx-framework\src\traditional\proc\p18f8723.asm
                     TOSU   0x000fff       data     extern E:\MPASM_MPLINK_PIC18_LT_Branch_3_42\pic18-lt\cxx-framework\src\traditional\proc\p18f8723.asm
                  TRAMEIN   0x00017d       data     extern C:\Users\LFRAD\Documents\CMS2Luc\ProjetsNettoyesCMSGit\ProjetCarteMere\project\CMSModifV1SD.c
                 TRAMEOUT   0x000100       data     extern C:\Users\LFRAD\Documents\CMS2Luc\ProjetsNettoyesCMSGit\ProjetCarteMere\project\CMSModifV1SD.c
                    TRISA   0x000f92       data     extern E:\MPASM_MPLINK_PIC18_LT_Branch_3_42\pic18-lt\cxx-framework\src\traditional\proc\p18f8723.asm
                TRISAbits   0x000f92       data     extern E:\MPASM_MPLINK_PIC18_LT_Branch_3_42\pic18-lt\cxx-framework\src\traditional\proc\p18f8723.asm
                    TRISB   0x000f93       data     extern E:\MPASM_MPLINK_PIC18_LT_Branch_3_42\pic18-lt\cxx-framework\src\traditional\proc\p18f8723.asm
                TRISBbits   0x000f93       data     extern E:\MPASM_MPLINK_PIC18_LT_Branch_3_42\pic18-lt\cxx-framework\src\traditional\proc\p18f8723.asm
                    TRISC   0x000f94       data     extern E:\MPASM_MPLINK_PIC18_LT_Branch_3_42\pic18-lt\cxx-framework\src\traditional\proc\p18f8723.asm
                TRISCbits   0x000f94       data     extern E:\MPASM_MPLINK_PIC18_LT_Branch_3_42\pic18-lt\cxx-framework\src\traditional\proc\p18f8723.asm
                    TRISD   0x000f95       data     extern E:\MPASM_MPLINK_PIC18_LT_Branch_3_42\pic18-lt\cxx-framework\src\traditional\proc\p18f8723.asm
                TRISDbits   0x000f95       data     extern E:\MPASM_MPLINK_PIC18_LT_Branch_3_42\pic18-lt\cxx-framework\src\traditional\proc\p18f8723.asm
                    TRISE   0x000f96       data     extern E:\MPASM_MPLINK_PIC18_LT_Branch_3_42\pic18-lt\cxx-framework\src\traditional\proc\p18f8723.asm
                TRISEbits   0x000f96       data     extern E:\MPASM_MPLINK_PIC18_LT_Branch_3_42\pic18-lt\cxx-framework\src\traditional\proc\p18f8723.asm
                    TRISF   0x000f97       data     extern E:\MPASM_MPLINK_PIC18_LT_Branch_3_42\pic18-lt\cxx-framework\src\traditional\proc\p18f8723.asm
                TRISFbits   0x000f97       data     extern E:\MPASM_MPLINK_PIC18_LT_Branch_3_42\pic18-lt\cxx-framework\src\traditional\proc\p18f8723.asm
                    TRISG   0x000f98       data     extern E:\MPASM_MPLINK_PIC18_LT_Branch_3_42\pic18-lt\cxx-framework\src\traditional\proc\p18f8723.asm
                TRISGbits   0x000f98       data     extern E:\MPASM_MPLINK_PIC18_LT_Branch_3_42\pic18-lt\cxx-framework\src\traditional\proc\p18f8723.asm
                    TRISH   0x000f99       data     extern E:\MPASM_MPLINK_PIC18_LT_Branch_3_42\pic18-lt\cxx-framework\src\traditional\proc\p18f8723.asm
                TRISHbits   0x000f99       data     extern E:\MPASM_MPLINK_PIC18_LT_Branch_3_42\pic18-lt\cxx-framework\src\traditional\proc\p18f8723.asm
                    TRISJ   0x000f9a       data     extern E:\MPASM_MPLINK_PIC18_LT_Branch_3_42\pic18-lt\cxx-framework\src\traditional\proc\p18f8723.asm
                TRISJbits   0x000f9a       data     extern E:\MPASM_MPLINK_PIC18_LT_Branch_3_42\pic18-lt\cxx-framework\src\traditional\proc\p18f8723.asm
         TROPDENONREPONSE   0x000f1d       data     extern C:\Users\LFRAD\Documents\CMS2Luc\ProjetsNettoyesCMSGit\ProjetCarteMere\project\CMSModifV1SD.c
                    TXREG   0x000fad       data     extern E:\MPASM_MPLINK_PIC18_LT_Branch_3_42\pic18-lt\cxx-framework\src\traditional\proc\p18f8723.asm
                   TXREG1   0x000fad       data     extern E:\MPASM_MPLINK_PIC18_LT_Branch_3_42\pic18-lt\cxx-framework\src\traditional\proc\p18f8723.asm
                   TXREG2   0x000f6d       data     extern E:\MPASM_MPLINK_PIC18_LT_Branch_3_42\pic18-lt\cxx-framework\src\traditional\proc\p18f8723.asm
                    TXSTA   0x000fac       data     extern E:\MPASM_MPLINK_PIC18_LT_Branch_3_42\pic18-lt\cxx-framework\src\traditional\proc\p18f8723.asm
                   TXSTA1   0x000fac       data     extern E:\MPASM_MPLINK_PIC18_LT_Branch_3_42\pic18-lt\cxx-framework\src\traditional\proc\p18f8723.asm
               TXSTA1bits   0x000fac       data     extern E:\MPASM_MPLINK_PIC18_LT_Branch_3_42\pic18-lt\cxx-framework\src\traditional\proc\p18f8723.asm
                   TXSTA2   0x000f6c       data     extern E:\MPASM_MPLINK_PIC18_LT_Branch_3_42\pic18-lt\cxx-framework\src\traditional\proc\p18f8723.asm
               TXSTA2bits   0x000f6c       data     extern E:\MPASM_MPLINK_PIC18_LT_Branch_3_42\pic18-lt\cxx-framework\src\traditional\proc\p18f8723.asm
                TXSTAbits   0x000fac       data     extern E:\MPASM_MPLINK_PIC18_LT_Branch_3_42\pic18-lt\cxx-framework\src\traditional\proc\p18f8723.asm
                     TYPE   0x000206       data     extern C:\Users\LFRAD\Documents\CMS2Luc\ProjetsNettoyesCMSGit\ProjetCarteMere\project\CMSModifV1SD.c
                TYPECARTE   0x000257       data     extern C:\Users\LFRAD\Documents\CMS2Luc\ProjetsNettoyesCMSGit\ProjetCarteMere\project\CMSModifV1SD.c
             TYPECOMMANDE   0x000f22       data     extern C:\Users\LFRAD\Documents\CMS2Luc\ProjetsNettoyesCMSGit\ProjetCarteMere\project\CMSModifV1SD.c
          TYPEDECARTEOEIL   0x000f36       data     extern C:\Users\LFRAD\Documents\CMS2Luc\ProjetsNettoyesCMSGit\ProjetCarteMere\project\CMSModifV1SD.c
              TYPE_ERREUR   0x00026a       data     extern C:\Users\LFRAD\Documents\CMS2Luc\ProjetsNettoyesCMSGit\ProjetCarteMere\project\CMSModifV1SD.c
               UNRESETRI1   0x000f30       data     extern C:\Users\LFRAD\Documents\CMS2Luc\ProjetsNettoyesCMSGit\ProjetCarteMere\project\CMSModifV1SD.c
               UNRESETRI2   0x000f31       data     extern C:\Users\LFRAD\Documents\CMS2Luc\ProjetsNettoyesCMSGit\ProjetCarteMere\project\CMSModifV1SD.c
               UNRESETRI3   0x000f32       data     extern C:\Users\LFRAD\Documents\CMS2Luc\ProjetsNettoyesCMSGit\ProjetCarteMere\project\CMSModifV1SD.c
               UNRESETRI4   0x000f33       data     extern C:\Users\LFRAD\Documents\CMS2Luc\ProjetsNettoyesCMSGit\ProjetCarteMere\project\CMSModifV1SD.c
               UNRESETRI5   0x000f34       data     extern C:\Users\LFRAD\Documents\CMS2Luc\ProjetsNettoyesCMSGit\ProjetCarteMere\project\CMSModifV1SD.c
                   VALEUR   0x00024f       data     extern C:\Users\LFRAD\Documents\CMS2Luc\ProjetsNettoyesCMSGit\ProjetCarteMere\project\CMSModifV1SD.c
                     VBAT   0x0002de       data     extern C:\Users\LFRAD\Documents\CMS2Luc\ProjetsNettoyesCMSGit\ProjetCarteMere\project\CMSModifV1SD.c
                     VDD1   0x0002c2       data     extern C:\Users\LFRAD\Documents\CMS2Luc\ProjetsNettoyesCMSGit\ProjetCarteMere\project\CMSModifV1SD.c
                     VDD2   0x0002c6       data     extern C:\Users\LFRAD\Documents\CMS2Luc\ProjetsNettoyesCMSGit\ProjetCarteMere\project\CMSModifV1SD.c
                     VDD3   0x0002ca       data     extern C:\Users\LFRAD\Documents\CMS2Luc\ProjetsNettoyesCMSGit\ProjetCarteMere\project\CMSModifV1SD.c
                     VDD4   0x0002ce       data     extern C:\Users\LFRAD\Documents\CMS2Luc\ProjetsNettoyesCMSGit\ProjetCarteMere\project\CMSModifV1SD.c
                     VDD5   0x0002d2       data     extern C:\Users\LFRAD\Documents\CMS2Luc\ProjetsNettoyesCMSGit\ProjetCarteMere\project\CMSModifV1SD.c
                     VDD6   0x0002da       data     extern C:\Users\LFRAD\Documents\CMS2Luc\ProjetsNettoyesCMSGit\ProjetCarteMere\project\CMSModifV1SD.c
                  VOIECOD   0x000200       data     extern C:\Users\LFRAD\Documents\CMS2Luc\ProjetsNettoyesCMSGit\ProjetCarteMere\project\CMSModifV1SD.c
                    Vtemp   0x0002d6       data     extern C:\Users\LFRAD\Documents\CMS2Luc\ProjetsNettoyesCMSGit\ProjetCarteMere\project\CMSModifV1SD.c
                   WDTCON   0x000fd1       data     extern E:\MPASM_MPLINK_PIC18_LT_Branch_3_42\pic18-lt\cxx-framework\src\traditional\proc\p18f8723.asm
               WDTCONbits   0x000fd1       data     extern E:\MPASM_MPLINK_PIC18_LT_Branch_3_42\pic18-lt\cxx-framework\src\traditional\proc\p18f8723.asm
                     WREG   0x000fe8       data     extern E:\MPASM_MPLINK_PIC18_LT_Branch_3_42\pic18-lt\cxx-framework\src\traditional\proc\p18f8723.asm
                 __AARGB0   0x000009       data     extern E:\MPASM_MPLINK_PIC18_LT_Branch_3_42\pic18-lt\cxx-framework\src\traditional\math\aarg.asm
                 __AARGB1   0x000008       data     extern E:\MPASM_MPLINK_PIC18_LT_Branch_3_42\pic18-lt\cxx-framework\src\traditional\math\aarg.asm
                 __AARGB2   0x000007       data     extern E:\MPASM_MPLINK_PIC18_LT_Branch_3_42\pic18-lt\cxx-framework\src\traditional\math\aarg.asm
                 __AARGB3   0x000006       data     extern E:\MPASM_MPLINK_PIC18_LT_Branch_3_42\pic18-lt\cxx-framework\src\traditional\math\aarg.asm
                 __AARGB4   0x000005       data     extern E:\MPASM_MPLINK_PIC18_LT_Branch_3_42\pic18-lt\cxx-framework\src\traditional\math\aarg.asm
                 __AARGB5   0x000004       data     extern E:\MPASM_MPLINK_PIC18_LT_Branch_3_42\pic18-lt\cxx-framework\src\traditional\math\aarg.asm
                 __AARGB6   0x000003       data     extern E:\MPASM_MPLINK_PIC18_LT_Branch_3_42\pic18-lt\cxx-framework\src\traditional\math\aarg.asm
                 __AARGB7   0x000002       data     extern E:\MPASM_MPLINK_PIC18_LT_Branch_3_42\pic18-lt\cxx-framework\src\traditional\math\aarg.asm
                   __AEXP   0x00000a       data     extern E:\MPASM_MPLINK_PIC18_LT_Branch_3_42\pic18-lt\cxx-framework\src\traditional\math\aarg.asm
                 __BARGB0   0x00000e       data     extern E:\MPASM_MPLINK_PIC18_LT_Branch_3_42\pic18-lt\cxx-framework\src\traditional\math\barg.asm
                 __BARGB1   0x00000d       data     extern E:\MPASM_MPLINK_PIC18_LT_Branch_3_42\pic18-lt\cxx-framework\src\traditional\math\barg.asm
                 __BARGB2   0x00000c       data     extern E:\MPASM_MPLINK_PIC18_LT_Branch_3_42\pic18-lt\cxx-framework\src\traditional\math\barg.asm
                 __BARGB3   0x00000b       data     extern E:\MPASM_MPLINK_PIC18_LT_Branch_3_42\pic18-lt\cxx-framework\src\traditional\math\barg.asm
                   __BEXP   0x00000f       data     extern E:\MPASM_MPLINK_PIC18_LT_Branch_3_42\pic18-lt\cxx-framework\src\traditional\math\barg.asm
                __FPFLAGS   0x000001       data     extern E:\MPASM_MPLINK_PIC18_LT_Branch_3_42\pic18-lt\cxx-framework\src\traditional\math\cmath18.asm
            __FPFLAGSbits   0x000001       data     extern E:\MPASM_MPLINK_PIC18_LT_Branch_3_42\pic18-lt\cxx-framework\src\traditional\math\cmath18.asm
                  __REMB0   0x000005       data     extern E:\MPASM_MPLINK_PIC18_LT_Branch_3_42\pic18-lt\cxx-framework\src\traditional\math\aarg.asm
                  __REMB1   0x000004       data     extern E:\MPASM_MPLINK_PIC18_LT_Branch_3_42\pic18-lt\cxx-framework\src\traditional\math\aarg.asm
                  __REMB2   0x000003       data     extern E:\MPASM_MPLINK_PIC18_LT_Branch_3_42\pic18-lt\cxx-framework\src\traditional\math\aarg.asm
                  __REMB3   0x000002       data     extern E:\MPASM_MPLINK_PIC18_LT_Branch_3_42\pic18-lt\cxx-framework\src\traditional\math\aarg.asm
                   __TEMP   0x000013       data     extern E:\MPASM_MPLINK_PIC18_LT_Branch_3_42\pic18-lt\cxx-framework\src\traditional\math\temparg.asm
                 __TEMPB0   0x000013       data     extern E:\MPASM_MPLINK_PIC18_LT_Branch_3_42\pic18-lt\cxx-framework\src\traditional\math\temparg.asm
                 __TEMPB1   0x000012       data     extern E:\MPASM_MPLINK_PIC18_LT_Branch_3_42\pic18-lt\cxx-framework\src\traditional\math\temparg.asm
                 __TEMPB2   0x000011       data     extern E:\MPASM_MPLINK_PIC18_LT_Branch_3_42\pic18-lt\cxx-framework\src\traditional\math\temparg.asm
                 __TEMPB3   0x000010       data     extern E:\MPASM_MPLINK_PIC18_LT_Branch_3_42\pic18-lt\cxx-framework\src\traditional\math\temparg.asm
                  __tmp_0   0x000014       data     static C:\Users\LFRAD\Documents\CMS2Luc\ProjetsNettoyesCMSGit\ProjetCarteMere\project\CMSModifV1SD.c
                  __tmp_0   0x000014       data     static E:\MPASM_MPLINK_PIC18_LT_Branch_3_42\pic18-lt\cxx-framework\src\pmc_common\i2c\i2c1writ.c
               calculBLOC   0x000f19       data     extern C:\Users\LFRAD\Documents\CMS2Luc\ProjetsNettoyesCMSGit\ProjetCarteMere\project\CMSModifV1SD.c
               capt_exist   0x0002c1       data     extern C:\Users\LFRAD\Documents\CMS2Luc\ProjetsNettoyesCMSGit\ProjetCarteMere\project\CMSModifV1SD.c
                   cycleN   0x000f26       data     extern C:\Users\LFRAD\Documents\CMS2Luc\ProjetsNettoyesCMSGit\ProjetCarteMere\project\CMSModifV1SD.c
                       ii   0x00023f       data     extern C:\Users\LFRAD\Documents\CMS2Luc\ProjetsNettoyesCMSGit\ProjetCarteMere\project\CMSModifV1SD.c
                     iiii   0x000244       data     extern C:\Users\LFRAD\Documents\CMS2Luc\ProjetsNettoyesCMSGit\ProjetCarteMere\project\CMSModifV1SD.c
                       mm   0x00023d       data     extern C:\Users\LFRAD\Documents\CMS2Luc\ProjetsNettoyesCMSGit\ProjetCarteMere\project\CMSModifV1SD.c
             mouchardINT0   0x000f3b       data     extern C:\Users\LFRAD\Documents\CMS2Luc\ProjetsNettoyesCMSGit\ProjetCarteMere\project\CMSModifV1SD.c
             numdecarteRI   0x000f1c       data     extern C:\Users\LFRAD\Documents\CMS2Luc\ProjetsNettoyesCMSGit\ProjetCarteMere\project\CMSModifV1SD.c
          pointeur_out_in   0x0002e3       data     extern C:\Users\LFRAD\Documents\CMS2Luc\ProjetsNettoyesCMSGit\ProjetCarteMere\project\CMSModifV1SD.c
           resetheurefixe   0x000f3d       data     extern C:\Users\LFRAD\Documents\CMS2Luc\ProjetsNettoyesCMSGit\ProjetCarteMere\project\CMSModifV1SD.c
        scrutationunevoie   0x000f39       data     extern C:\Users\LFRAD\Documents\CMS2Luc\ProjetsNettoyesCMSGit\ProjetCarteMere\project\CMSModifV1SD.c
         temoinfinvoieZIZ   0x000f23       data     extern C:\Users\LFRAD\Documents\CMS2Luc\ProjetsNettoyesCMSGit\ProjetCarteMere\project\CMSModifV1SD.c
                      tmp   0x0002e5       data     extern C:\Users\LFRAD\Documents\CMS2Luc\ProjetsNettoyesCMSGit\ProjetCarteMere\project\CMSModifV1SD.c
                     tmp2   0x0002e6       data     extern C:\Users\LFRAD\Documents\CMS2Luc\ProjetsNettoyesCMSGit\ProjetCarteMere\project\CMSModifV1SD.c



                              Symbols - Sorted by Address
                     Name    Address   Location    Storage File                     
                ---------  ---------  ---------  --------- ---------                
                   _entry   0x000000    program     extern E:\MPASM_MPLINK_PIC18_LT_Branch_3_42\pic18-lt\cxx-framework\src\traditional\startup\c018.c
       ___return_lbl00000   0x000004    program     static                          
               HighVector   0x000018    program     extern C:\Users\LFRAD\Documents\CMS2Luc\ProjetsNettoyesCMSGit\ProjetCarteMere\project\CMSModifV1SD.c
       ___return_lbl00000   0x00001c    program     static                          
                    inter   0x000202    program     extern C:\Users\LFRAD\Documents\CMS2Luc\ProjetsNettoyesCMSGit\ProjetCarteMere\project\CMSModifV1SD.c
                     main   0x0002c4    program     extern C:\Users\LFRAD\Documents\CMS2Luc\ProjetsNettoyesCMSGit\ProjetCarteMere\project\CMSModifV1SD.c
             __tmplbl_768   0x000888    program     static                          
             __tmplbl_719   0x0011f0    program     static                          
               Init_RS485   0x0016aa    program     extern C:\Users\LFRAD\Documents\CMS2Luc\ProjetsNettoyesCMSGit\ProjetCarteMere\project\CMSModifV1SD.c
         RECEVOIRST_RS485   0x00170a    program     extern C:\Users\LFRAD\Documents\CMS2Luc\ProjetsNettoyesCMSGit\ProjetCarteMere\project\CMSModifV1SD.c
           RECEVOIR_RS485   0x001740    program     extern C:\Users\LFRAD\Documents\CMS2Luc\ProjetsNettoyesCMSGit\ProjetCarteMere\project\CMSModifV1SD.c
                    RS485   0x00182e    program     extern C:\Users\LFRAD\Documents\CMS2Luc\ProjetsNettoyesCMSGit\ProjetCarteMere\project\CMSModifV1SD.c
TRAMERECEPTIONRS485DONNEES   0x001856    program     extern C:\Users\LFRAD\Documents\CMS2Luc\ProjetsNettoyesCMSGit\ProjetCarteMere\project\CMSModifV1SD.c
   TRAMEENVOIRS485DONNEES   0x0018da    program     extern C:\Users\LFRAD\Documents\CMS2Luc\ProjetsNettoyesCMSGit\ProjetCarteMere\project\CMSModifV1SD.c
        ENVOIE_DES_TRAMES   0x00194c    program     extern C:\Users\LFRAD\Documents\CMS2Luc\ProjetsNettoyesCMSGit\ProjetCarteMere\project\CMSModifV1SD.c
             __tmplbl_778   0x002710    program     static                          
             __tmplbl_777   0x002828    program     static                          
             __tmplbl_776   0x002942    program     static                          
             __tmplbl_775   0x002c4e    program     static                          
             __tmplbl_774   0x002f06    program     static                          
             __tmplbl_773   0x002fe4    program     static                          
             __tmplbl_772   0x003158    program     static                          
             __tmplbl_771   0x00326a    program     static                          
             __tmplbl_783   0x003630    program     static                          
             __tmplbl_784   0x003630    program     static                          
             __tmplbl_785   0x003630    program     static                          
             __tmplbl_786   0x003630    program     static                          
             __tmplbl_787   0x003630    program     static                          
             __tmplbl_788   0x003630    program     static                          
             __tmplbl_789   0x003630    program     static                          
             __tmplbl_811   0x003630    program     static                          
             __tmplbl_810   0x003630    program     static                          
             __tmplbl_808   0x003630    program     static                          
             __tmplbl_807   0x003630    program     static                          
             __tmplbl_806   0x003630    program     static                          
             __tmplbl_804   0x003630    program     static                          
             __tmplbl_803   0x003630    program     static                          
             __tmplbl_802   0x003630    program     static                          
             __tmplbl_791   0x003630    program     static                          
  RECUPERATION_DES_TRAMES   0x003644    program     extern C:\Users\LFRAD\Documents\CMS2Luc\ProjetsNettoyesCMSGit\ProjetCarteMere\project\CMSModifV1SD.c
             __tmplbl_847   0x004472    program     static                          
             __tmplbl_846   0x004718    program     static                          
             __tmplbl_845   0x00483a    program     static                          
             __tmplbl_865   0x005212    program     static                          
             __tmplbl_844   0x005218    program     static                          
             __tmplbl_881   0x0054cc    program     static                          
             __tmplbl_843   0x0054d0    program     static                          
             __tmplbl_842   0x0056e0    program     static                          
             __tmplbl_841   0x00588c    program     static                          
             __tmplbl_875   0x005b20    program     static                          
             __tmplbl_876   0x005b32    program     static                          
             __tmplbl_880   0x005b40    program     static                          
             __tmplbl_874   0x005b40    program     static                          
             __tmplbl_840   0x005b44    program     static                          
             __tmplbl_912   0x005faa    program     static                          
             __tmplbl_911   0x005faa    program     static                          
             __tmplbl_839   0x005fb0    program     static                          
             __tmplbl_867   0x006270    program     static                          
             __tmplbl_836   0x006276    program     static                          
             __tmplbl_835   0x0065a2    program     static                          
             __tmplbl_834   0x006686    program     static                          
             __tmplbl_833   0x00668e    program     static                          
             __tmplbl_832   0x00677e    program     static                          
             __tmplbl_872   0x00679c    program     static                          
             __tmplbl_831   0x0067ae    program     static                          
             __tmplbl_838   0x0067ae    program     static                          
             __tmplbl_830   0x0067b6    program     static                          
             __tmplbl_829   0x006a4c    program     static                          
             __tmplbl_828   0x006b8c    program     static                          
             __tmplbl_863   0x007342    program     static                          
             __tmplbl_858   0x007342    program     static                          
             __tmplbl_934   0x007342    program     static                          
             __tmplbl_935   0x007354    program     static                          
             __tmplbl_869   0x007362    program     static                          
             __tmplbl_928   0x007362    program     static                          
             __tmplbl_925   0x007362    program     static                          
             __tmplbl_868   0x007362    program     static                          
             __tmplbl_913   0x007362    program     static                          
             __tmplbl_873   0x007362    program     static                          
             __tmplbl_862   0x007362    program     static                          
             __tmplbl_910   0x007362    program     static                          
             __tmplbl_857   0x007366    program     static                          
             __tmplbl_856   0x007366    program     static                          
             __tmplbl_933   0x007370    program     static                          
             __tmplbl_861   0x007370    program     static                          
             __tmplbl_859   0x007370    program     static                          
             __tmplbl_860   0x007370    program     static                          
             __tmplbl_864   0x007370    program     static                          
             __tmplbl_837   0x007370    program     static                          
             __tmplbl_871   0x007370    program     static                          
             __tmplbl_932   0x007370    program     static                          
             __tmplbl_931   0x007370    program     static                          
  recuperer_trame_memoire   0x007384    program     extern C:\Users\LFRAD\Documents\CMS2Luc\ProjetsNettoyesCMSGit\ProjetCarteMere\project\CMSModifV1SD.c
 construire_trame_memoire   0x009102    program     extern C:\Users\LFRAD\Documents\CMS2Luc\ProjetsNettoyesCMSGit\ProjetCarteMere\project\CMSModifV1SD.c
               calcul_CRC   0x00ac16    program     extern C:\Users\LFRAD\Documents\CMS2Luc\ProjetsNettoyesCMSGit\ProjetCarteMere\project\CMSModifV1SD.c
             controle_CRC   0x00acae    program     extern C:\Users\LFRAD\Documents\CMS2Luc\ProjetsNettoyesCMSGit\ProjetCarteMere\project\CMSModifV1SD.c
                  resetTO   0x00ad22    program     extern C:\Users\LFRAD\Documents\CMS2Luc\ProjetsNettoyesCMSGit\ProjetCarteMere\project\CMSModifV1SD.c
        calcul_addmemoire   0x00ad7c    program     extern C:\Users\LFRAD\Documents\CMS2Luc\ProjetsNettoyesCMSGit\ProjetCarteMere\project\CMSModifV1SD.c
            choix_memoire   0x00b13c    program     extern C:\Users\LFRAD\Documents\CMS2Luc\ProjetsNettoyesCMSGit\ProjetCarteMere\project\CMSModifV1SD.c
              LIRE_EEPROM   0x00b308    program     extern C:\Users\LFRAD\Documents\CMS2Luc\ProjetsNettoyesCMSGit\ProjetCarteMere\project\CMSModifV1SD.c
                 delay_ms   0x00b55c    program     extern C:\Users\LFRAD\Documents\CMS2Luc\ProjetsNettoyesCMSGit\ProjetCarteMere\project\CMSModifV1SD.c
                 Init_I2C   0x00b5e0    program     extern C:\Users\LFRAD\Documents\CMS2Luc\ProjetsNettoyesCMSGit\ProjetCarteMere\project\CMSModifV1SD.c
        ECRIRE_EEPROMBYTE   0x00b5f2    program     extern C:\Users\LFRAD\Documents\CMS2Luc\ProjetsNettoyesCMSGit\ProjetCarteMere\project\CMSModifV1SD.c
            SERIALISATION   0x00b804    program     extern C:\Users\LFRAD\Documents\CMS2Luc\ProjetsNettoyesCMSGit\ProjetCarteMere\project\CMSModifV1SD.c
      identificationINTER   0x00b8f4    program     extern C:\Users\LFRAD\Documents\CMS2Luc\ProjetsNettoyesCMSGit\ProjetCarteMere\project\CMSModifV1SD.c
              AQUIENVOYER   0x00bd92    program     extern C:\Users\LFRAD\Documents\CMS2Luc\ProjetsNettoyesCMSGit\ProjetCarteMere\project\CMSModifV1SD.c
         REPOSAQUIENVOYER   0x00bef6    program     extern C:\Users\LFRAD\Documents\CMS2Luc\ProjetsNettoyesCMSGit\ProjetCarteMere\project\CMSModifV1SD.c
            reglerhorloge   0x00c032    program     extern C:\Users\LFRAD\Documents\CMS2Luc\ProjetsNettoyesCMSGit\ProjetCarteMere\project\CMSModifV1SD.c
             lire_horloge   0x00c03e    program     extern C:\Users\LFRAD\Documents\CMS2Luc\ProjetsNettoyesCMSGit\ProjetCarteMere\project\CMSModifV1SD.c
TRANSFORMER_TRAME_MEM_EN_COM   0x00c05c    program     extern C:\Users\LFRAD\Documents\CMS2Luc\ProjetsNettoyesCMSGit\ProjetCarteMere\project\CMSModifV1SD.c
               EFFACEMENT   0x00dc58    program     extern C:\Users\LFRAD\Documents\CMS2Luc\ProjetsNettoyesCMSGit\ProjetCarteMere\project\CMSModifV1SD.c
    PREPARATION_PAGE_AUTO   0x00dd70    program     extern C:\Users\LFRAD\Documents\CMS2Luc\ProjetsNettoyesCMSGit\ProjetCarteMere\project\CMSModifV1SD.c
             putstringI2C   0x00e1b8    program     extern C:\Users\LFRAD\Documents\CMS2Luc\ProjetsNettoyesCMSGit\ProjetCarteMere\project\CMSModifV1SD.c
                IntToChar   0x00e278    program     extern C:\Users\LFRAD\Documents\CMS2Luc\ProjetsNettoyesCMSGit\ProjetCarteMere\project\CMSModifV1SD.c
      MESURE_DES_TENSIONS   0x00e936    program     extern C:\Users\LFRAD\Documents\CMS2Luc\ProjetsNettoyesCMSGit\ProjetCarteMere\project\CMSModifV1SD.c
                      CAN   0x00ed32    program     extern C:\Users\LFRAD\Documents\CMS2Luc\ProjetsNettoyesCMSGit\ProjetCarteMere\project\CMSModifV1SD.c
                  AVERAGE   0x00ee34    program     extern C:\Users\LFRAD\Documents\CMS2Luc\ProjetsNettoyesCMSGit\ProjetCarteMere\project\CMSModifV1SD.c
     CONTROLE_CHARGE_BATT   0x00f0d8    program     extern C:\Users\LFRAD\Documents\CMS2Luc\ProjetsNettoyesCMSGit\ProjetCarteMere\project\CMSModifV1SD.c
INTERROGER_TOUT_LES_CAPTEURS   0x00f18a    program     extern C:\Users\LFRAD\Documents\CMS2Luc\ProjetsNettoyesCMSGit\ProjetCarteMere\project\CMSModifV1SD.c
            EFFACER_LISTE   0x00f49c    program     extern C:\Users\LFRAD\Documents\CMS2Luc\ProjetsNettoyesCMSGit\ProjetCarteMere\project\CMSModifV1SD.c
  METTRE_EN_MEMOIRE_LISTE   0x00f578    program     extern C:\Users\LFRAD\Documents\CMS2Luc\ProjetsNettoyesCMSGit\ProjetCarteMere\project\CMSModifV1SD.c
        GROUPE_EN_MEMOIRE   0x00f6a6    program     extern C:\Users\LFRAD\Documents\CMS2Luc\ProjetsNettoyesCMSGit\ProjetCarteMere\project\CMSModifV1SD.c
       envoyerHORLOGE_i2c   0x00f74a    program     extern C:\Users\LFRAD\Documents\CMS2Luc\ProjetsNettoyesCMSGit\ProjetCarteMere\project\CMSModifV1SD.c
           litHORLOGE_i2c   0x00f794    program     extern C:\Users\LFRAD\Documents\CMS2Luc\ProjetsNettoyesCMSGit\ProjetCarteMere\project\CMSModifV1SD.c
           ECRIRE_HORLOGE   0x00f7e8    program     extern C:\Users\LFRAD\Documents\CMS2Luc\ProjetsNettoyesCMSGit\ProjetCarteMere\project\CMSModifV1SD.c
             LIRE_HORLOGE   0x00f8c0    program     extern C:\Users\LFRAD\Documents\CMS2Luc\ProjetsNettoyesCMSGit\ProjetCarteMere\project\CMSModifV1SD.c
      creer_trame_horloge   0x00f93e    program     extern C:\Users\LFRAD\Documents\CMS2Luc\ProjetsNettoyesCMSGit\ProjetCarteMere\project\CMSModifV1SD.c
     entrer_trame_horloge   0x00fa7e    program     extern C:\Users\LFRAD\Documents\CMS2Luc\ProjetsNettoyesCMSGit\ProjetCarteMere\project\CMSModifV1SD.c
trouver_carte_suivantvoie   0x00fb28    program     extern C:\Users\LFRAD\Documents\CMS2Luc\ProjetsNettoyesCMSGit\ProjetCarteMere\project\CMSModifV1SD.c
                    TEMPO   0x00fcea    program     extern C:\Users\LFRAD\Documents\CMS2Luc\ProjetsNettoyesCMSGit\ProjetCarteMere\project\CMSModifV1SD.c
      SD_WriteSingleBlock   0x00fd82    program     extern C:\Users\LFRAD\Documents\CMS2Luc\ProjetsNettoyesCMSGit\ProjetCarteMere\project\CMSModifV1SD.c
       SD_ReadSingleBlock   0x00fedc    program     extern C:\Users\LFRAD\Documents\CMS2Luc\ProjetsNettoyesCMSGit\ProjetCarteMere\project\CMSModifV1SD.c
           SD_SendCommand   0x010074    program     extern C:\Users\LFRAD\Documents\CMS2Luc\ProjetsNettoyesCMSGit\ProjetCarteMere\project\CMSModifV1SD.c
            SPI_WriteByte   0x010184    program     extern C:\Users\LFRAD\Documents\CMS2Luc\ProjetsNettoyesCMSGit\ProjetCarteMere\project\CMSModifV1SD.c
                 sd_reset   0x0101a2    program     extern C:\Users\LFRAD\Documents\CMS2Luc\ProjetsNettoyesCMSGit\ProjetCarteMere\project\CMSModifV1SD.c
                  spi_low   0x0102f2    program     extern C:\Users\LFRAD\Documents\CMS2Luc\ProjetsNettoyesCMSGit\ProjetCarteMere\project\CMSModifV1SD.c
                 spi_high   0x0102f8    program     extern C:\Users\LFRAD\Documents\CMS2Luc\ProjetsNettoyesCMSGit\ProjetCarteMere\project\CMSModifV1SD.c
                 init_spi   0x0102fe    program     extern C:\Users\LFRAD\Documents\CMS2Luc\ProjetsNettoyesCMSGit\ProjetCarteMere\project\CMSModifV1SD.c
                 delay_us   0x01031a    program     extern C:\Users\LFRAD\Documents\CMS2Luc\ProjetsNettoyesCMSGit\ProjetCarteMere\project\CMSModifV1SD.c
            SAV_EXISTENCE   0x01034e    program     extern C:\Users\LFRAD\Documents\CMS2Luc\ProjetsNettoyesCMSGit\ProjetCarteMere\project\CMSModifV1SD.c
        intervertirOUT_IN   0x01053c    program     extern C:\Users\LFRAD\Documents\CMS2Luc\ProjetsNettoyesCMSGit\ProjetCarteMere\project\CMSModifV1SD.c
 RECHERCHE_DONNEES_GROUPE   0x0105ac    program     extern C:\Users\LFRAD\Documents\CMS2Luc\ProjetsNettoyesCMSGit\ProjetCarteMere\project\CMSModifV1SD.c
   EFFACER_CAPTEUR_SUR_CM   0x010614    program     extern C:\Users\LFRAD\Documents\CMS2Luc\ProjetsNettoyesCMSGit\ProjetCarteMere\project\CMSModifV1SD.c
MODIFICATION_TABLE_DEXISTENCE   0x0106fc    program     extern C:\Users\LFRAD\Documents\CMS2Luc\ProjetsNettoyesCMSGit\ProjetCarteMere\project\CMSModifV1SD.c
 CHERCHER_DONNNEES_CABLES   0x0109d8    program     extern C:\Users\LFRAD\Documents\CMS2Luc\ProjetsNettoyesCMSGit\ProjetCarteMere\project\CMSModifV1SD.c
       VALIDER_CAPTEUR_CM   0x010f20    program     extern C:\Users\LFRAD\Documents\CMS2Luc\ProjetsNettoyesCMSGit\ProjetCarteMere\project\CMSModifV1SD.c
       IDENTIF_TYPE_CARTE   0x01108c    program     extern C:\Users\LFRAD\Documents\CMS2Luc\ProjetsNettoyesCMSGit\ProjetCarteMere\project\CMSModifV1SD.c
          TROUVER_ROBINET   0x01139e    program     extern C:\Users\LFRAD\Documents\CMS2Luc\ProjetsNettoyesCMSGit\ProjetCarteMere\project\CMSModifV1SD.c
     REMISE_EN_FORME_PAGE   0x011524    program     extern C:\Users\LFRAD\Documents\CMS2Luc\ProjetsNettoyesCMSGit\ProjetCarteMere\project\CMSModifV1SD.c
                CRC_verif   0x0119b8    program     extern C:\Users\LFRAD\Documents\CMS2Luc\ProjetsNettoyesCMSGit\ProjetCarteMere\project\CMSModifV1SD.c
                    CRC16   0x011aca    program     extern C:\Users\LFRAD\Documents\CMS2Luc\ProjetsNettoyesCMSGit\ProjetCarteMere\project\CMSModifV1SD.c
               IntToChar5   0x011bca    program     extern C:\Users\LFRAD\Documents\CMS2Luc\ProjetsNettoyesCMSGit\ProjetCarteMere\project\CMSModifV1SD.c
            __tmplbl_1038   0x012422    program     static                          
                    SDWBN   0x01247e    program     extern C:\Users\LFRAD\Documents\CMS2Luc\ProjetsNettoyesCMSGit\ProjetCarteMere\project\CMSModifV1SD.c
                      SDW   0x012558    program     extern C:\Users\LFRAD\Documents\CMS2Luc\ProjetsNettoyesCMSGit\ProjetCarteMere\project\CMSModifV1SD.c
                    SDRBN   0x012af2    program     extern C:\Users\LFRAD\Documents\CMS2Luc\ProjetsNettoyesCMSGit\ProjetCarteMere\project\CMSModifV1SD.c
                      SDR   0x012c04    program     extern C:\Users\LFRAD\Documents\CMS2Luc\ProjetsNettoyesCMSGit\ProjetCarteMere\project\CMSModifV1SD.c
      envoyer_TRAME_PICSD   0x01316e    program     extern C:\Users\LFRAD\Documents\CMS2Luc\ProjetsNettoyesCMSGit\ProjetCarteMere\project\CMSModifV1SD.c
      reglerhorlogeautres   0x0138aa    program     extern C:\Users\LFRAD\Documents\CMS2Luc\ProjetsNettoyesCMSGit\ProjetCarteMere\project\CMSModifV1SD.c
                   stopIO   0x013a7a    program     extern C:\Users\LFRAD\Documents\CMS2Luc\ProjetsNettoyesCMSGit\ProjetCarteMere\project\CMSModifV1SD.c
         pic_eeprom_write   0x013a88    program     extern C:\Users\LFRAD\Documents\CMS2Luc\ProjetsNettoyesCMSGit\ProjetCarteMere\project\CMSModifV1SD.c
        ___while_lbl01866   0x013aac    program     static                          
        ___while_lbl01867   0x013ab0    program     static                          
       ___return_lbl01865   0x013ab4    program     static                          
          pic_eeprom_read   0x013abc    program     extern C:\Users\LFRAD\Documents\CMS2Luc\ProjetsNettoyesCMSGit\ProjetCarteMere\project\CMSModifV1SD.c
       controleheureRESET   0x013ade    program     extern C:\Users\LFRAD\Documents\CMS2Luc\ProjetsNettoyesCMSGit\ProjetCarteMere\project\CMSModifV1SD.c
                 FLO0832U   0x013ba8    program     extern E:\MPASM_MPLINK_PIC18_LT_Branch_3_42\pic18-lt\cxx-framework\src\traditional\math\cast08FP.asm
                 FLO0832S   0x013bac    program     extern E:\MPASM_MPLINK_PIC18_LT_Branch_3_42\pic18-lt\cxx-framework\src\traditional\math\cast08FP.asm
                jI2F08Beg   0x013bb6    program     static E:\MPASM_MPLINK_PIC18_LT_Branch_3_42\pic18-lt\cxx-framework\src\traditional\math\cast08FP.asm
                 FLO1632U   0x013bca    program     extern E:\MPASM_MPLINK_PIC18_LT_Branch_3_42\pic18-lt\cxx-framework\src\traditional\math\cast16FP.asm
                 FLO1632S   0x013bce    program     extern E:\MPASM_MPLINK_PIC18_LT_Branch_3_42\pic18-lt\cxx-framework\src\traditional\math\cast16FP.asm
                jI2F16Beg   0x013bde    program     static E:\MPASM_MPLINK_PIC18_LT_Branch_3_42\pic18-lt\cxx-framework\src\traditional\math\cast16FP.asm
                    FPS32   0x013bf4    program     extern E:\MPASM_MPLINK_PIC18_LT_Branch_3_42\pic18-lt\cxx-framework\src\traditional\math\addFP.asm
                    FPA32   0x013bf6    program     extern E:\MPASM_MPLINK_PIC18_LT_Branch_3_42\pic18-lt\cxx-framework\src\traditional\math\addFP.asm
                jBANotInf   0x013c14    program     static E:\MPASM_MPLINK_PIC18_LT_Branch_3_42\pic18-lt\cxx-framework\src\traditional\math\addFP.asm
                 jANotInf   0x013c1e    program     static E:\MPASM_MPLINK_PIC18_LT_Branch_3_42\pic18-lt\cxx-framework\src\traditional\math\addFP.asm
                 jBNotInf   0x013c2c    program     static E:\MPASM_MPLINK_PIC18_LT_Branch_3_42\pic18-lt\cxx-framework\src\traditional\math\addFP.asm
            jDifOrPosSign   0x013c40    program     static E:\MPASM_MPLINK_PIC18_LT_Branch_3_42\pic18-lt\cxx-framework\src\traditional\math\addFP.asm
             jNotBothZero   0x013c44    program     static E:\MPASM_MPLINK_PIC18_LT_Branch_3_42\pic18-lt\cxx-framework\src\traditional\math\addFP.asm
                 jAltBexp   0x013c70    program     static E:\MPASM_MPLINK_PIC18_LT_Branch_3_42\pic18-lt\cxx-framework\src\traditional\math\addFP.asm
              jAandWsetup   0x013c82    program     static E:\MPASM_MPLINK_PIC18_LT_Branch_3_42\pic18-lt\cxx-framework\src\traditional\math\addFP.asm
                 jANotNeg   0x013cb2    program     static E:\MPASM_MPLINK_PIC18_LT_Branch_3_42\pic18-lt\cxx-framework\src\traditional\math\addFP.asm
                 jWNotNeg   0x013cc6    program     static E:\MPASM_MPLINK_PIC18_LT_Branch_3_42\pic18-lt\cxx-framework\src\traditional\math\addFP.asm
               jShiftLoop   0x013ccc    program     static E:\MPASM_MPLINK_PIC18_LT_Branch_3_42\pic18-lt\cxx-framework\src\traditional\math\addFP.asm
               jShiftDone   0x013cda    program     static E:\MPASM_MPLINK_PIC18_LT_Branch_3_42\pic18-lt\cxx-framework\src\traditional\math\addFP.asm
                jSignDone   0x013d0a    program     static E:\MPASM_MPLINK_PIC18_LT_Branch_3_42\pic18-lt\cxx-framework\src\traditional\math\addFP.asm
               jFinalSign   0x013d1a    program     static E:\MPASM_MPLINK_PIC18_LT_Branch_3_42\pic18-lt\cxx-framework\src\traditional\math\addFP.asm
                    FPD32   0x013d22    program     extern E:\MPASM_MPLINK_PIC18_LT_Branch_3_42\pic18-lt\cxx-framework\src\traditional\math\divFP.asm
                 jANotInf   0x013d40    program     static E:\MPASM_MPLINK_PIC18_LT_Branch_3_42\pic18-lt\cxx-framework\src\traditional\math\divFP.asm
              jSignedZero   0x013d4a    program     static E:\MPASM_MPLINK_PIC18_LT_Branch_3_42\pic18-lt\cxx-framework\src\traditional\math\divFP.asm
                jANotZero   0x013d54    program     static E:\MPASM_MPLINK_PIC18_LT_Branch_3_42\pic18-lt\cxx-framework\src\traditional\math\divFP.asm
                    jLoop   0x013d7c    program     static E:\MPASM_MPLINK_PIC18_LT_Branch_3_42\pic18-lt\cxx-framework\src\traditional\math\divFP.asm
                jNoAdjust   0x013da0    program     static E:\MPASM_MPLINK_PIC18_LT_Branch_3_42\pic18-lt\cxx-framework\src\traditional\math\divFP.asm
                    jNext   0x013da2    program     static E:\MPASM_MPLINK_PIC18_LT_Branch_3_42\pic18-lt\cxx-framework\src\traditional\math\divFP.asm
                    FPM32   0x013dc8    program     extern E:\MPASM_MPLINK_PIC18_LT_Branch_3_42\pic18-lt\cxx-framework\src\traditional\math\mulFP.asm
                 jANotInf   0x013de6    program     static E:\MPASM_MPLINK_PIC18_LT_Branch_3_42\pic18-lt\cxx-framework\src\traditional\math\mulFP.asm
              jBothFinite   0x013df4    program     static E:\MPASM_MPLINK_PIC18_LT_Branch_3_42\pic18-lt\cxx-framework\src\traditional\math\mulFP.asm
                jHaveZero   0x013dfc    program     static E:\MPASM_MPLINK_PIC18_LT_Branch_3_42\pic18-lt\cxx-framework\src\traditional\math\mulFP.asm
             jBothNotZero   0x013e00    program     static E:\MPASM_MPLINK_PIC18_LT_Branch_3_42\pic18-lt\cxx-framework\src\traditional\math\mulFP.asm
                 FXD0808S   0x013ea2    program     extern E:\MPASM_MPLINK_PIC18_LT_Branch_3_42\pic18-lt\cxx-framework\src\traditional\math\fxd0808s.asm
                  DA0808S   0x013eae    program     static E:\MPASM_MPLINK_PIC18_LT_Branch_3_42\pic18-lt\cxx-framework\src\traditional\math\fxd0808s.asm
                   D0808S   0x013eb8    program     static E:\MPASM_MPLINK_PIC18_LT_Branch_3_42\pic18-lt\cxx-framework\src\traditional\math\fxd0808s.asm
                 D0808SOK   0x013ec2    program     static E:\MPASM_MPLINK_PIC18_LT_Branch_3_42\pic18-lt\cxx-framework\src\traditional\math\fxd0808s.asm
                D0808SNEG   0x013ec6    program     static E:\MPASM_MPLINK_PIC18_LT_Branch_3_42\pic18-lt\cxx-framework\src\traditional\math\fxd0808s.asm
                  D0808SX   0x013ecc    program     static E:\MPASM_MPLINK_PIC18_LT_Branch_3_42\pic18-lt\cxx-framework\src\traditional\math\fxd0808s.asm
                 FXD1616S   0x013ed6    program     extern E:\MPASM_MPLINK_PIC18_LT_Branch_3_42\pic18-lt\cxx-framework\src\traditional\math\fxd1616s.asm
                  DA1616S   0x013ee8    program     static E:\MPASM_MPLINK_PIC18_LT_Branch_3_42\pic18-lt\cxx-framework\src\traditional\math\fxd1616s.asm
                   D1616S   0x013ef8    program     static E:\MPASM_MPLINK_PIC18_LT_Branch_3_42\pic18-lt\cxx-framework\src\traditional\math\fxd1616s.asm
                 D1616SOK   0x013f02    program     static E:\MPASM_MPLINK_PIC18_LT_Branch_3_42\pic18-lt\cxx-framework\src\traditional\math\fxd1616s.asm
                D1616SNEG   0x013f06    program     static E:\MPASM_MPLINK_PIC18_LT_Branch_3_42\pic18-lt\cxx-framework\src\traditional\math\fxd1616s.asm
                  D1616SX   0x013f18    program     static E:\MPASM_MPLINK_PIC18_LT_Branch_3_42\pic18-lt\cxx-framework\src\traditional\math\fxd1616s.asm
                 FXM1616S   0x013f22    program     extern E:\MPASM_MPLINK_PIC18_LT_Branch_3_42\pic18-lt\cxx-framework\src\traditional\math\fxm1616s.asm
               TSIGN1616A   0x013f6e    program     static E:\MPASM_MPLINK_PIC18_LT_Branch_3_42\pic18-lt\cxx-framework\src\traditional\math\fxm1616s.asm
                 FXM1616U   0x013f7c    program     extern E:\MPASM_MPLINK_PIC18_LT_Branch_3_42\pic18-lt\cxx-framework\src\traditional\math\fxm1616u.asm
                  INT3208   0x013fb8    program     extern E:\MPASM_MPLINK_PIC18_LT_Branch_3_42\pic18-lt\cxx-framework\src\traditional\math\castFP08.asm
                     jMax   0x013fc8    program     static E:\MPASM_MPLINK_PIC18_LT_Branch_3_42\pic18-lt\cxx-framework\src\traditional\math\castFP08.asm
                  jMaxPos   0x013fcc    program     static E:\MPASM_MPLINK_PIC18_LT_Branch_3_42\pic18-lt\cxx-framework\src\traditional\math\castFP08.asm
                  jMaxNeg   0x013fd2    program     static E:\MPASM_MPLINK_PIC18_LT_Branch_3_42\pic18-lt\cxx-framework\src\traditional\math\castFP08.asm
                    jZero   0x013fd8    program     static E:\MPASM_MPLINK_PIC18_LT_Branch_3_42\pic18-lt\cxx-framework\src\traditional\math\castFP08.asm
                  jNotInf   0x013fdc    program     static E:\MPASM_MPLINK_PIC18_LT_Branch_3_42\pic18-lt\cxx-framework\src\traditional\math\castFP08.asm
                    jLoop   0x013fec    program     static E:\MPASM_MPLINK_PIC18_LT_Branch_3_42\pic18-lt\cxx-framework\src\traditional\math\castFP08.asm
                jLoopExit   0x013ffa    program     static E:\MPASM_MPLINK_PIC18_LT_Branch_3_42\pic18-lt\cxx-framework\src\traditional\math\castFP08.asm
                    jExit   0x014004    program     static E:\MPASM_MPLINK_PIC18_LT_Branch_3_42\pic18-lt\cxx-framework\src\traditional\math\castFP08.asm
                  TAGTB32   0x014006    program     extern E:\MPASM_MPLINK_PIC18_LT_Branch_3_42\pic18-lt\cxx-framework\src\traditional\math\gtFP.asm
              __FpCompare   0x014018    program     extern E:\MPASM_MPLINK_PIC18_LT_Branch_3_42\pic18-lt\cxx-framework\src\traditional\math\compFP.asm
             jBothNotZero   0x014036    program     static E:\MPASM_MPLINK_PIC18_LT_Branch_3_42\pic18-lt\cxx-framework\src\traditional\math\compFP.asm
                 jSignsEQ   0x01403a    program     static E:\MPASM_MPLINK_PIC18_LT_Branch_3_42\pic18-lt\cxx-framework\src\traditional\math\compFP.asm
                      jEQ   0x014052    program     static E:\MPASM_MPLINK_PIC18_LT_Branch_3_42\pic18-lt\cxx-framework\src\traditional\math\compFP.asm
                      jNE   0x014056    program     static E:\MPASM_MPLINK_PIC18_LT_Branch_3_42\pic18-lt\cxx-framework\src\traditional\math\compFP.asm
                    jExch   0x01405e    program     static E:\MPASM_MPLINK_PIC18_LT_Branch_3_42\pic18-lt\cxx-framework\src\traditional\math\compFP.asm
                  jNoExch   0x01407e    program     static E:\MPASM_MPLINK_PIC18_LT_Branch_3_42\pic18-lt\cxx-framework\src\traditional\math\compFP.asm
                   jFinal   0x014088    program     static E:\MPASM_MPLINK_PIC18_LT_Branch_3_42\pic18-lt\cxx-framework\src\traditional\math\compFP.asm
                  jAisNeg   0x014094    program     static E:\MPASM_MPLINK_PIC18_LT_Branch_3_42\pic18-lt\cxx-framework\src\traditional\math\compFP.asm
                   jShift   0x01409a    program     static E:\MPASM_MPLINK_PIC18_LT_Branch_3_42\pic18-lt\cxx-framework\src\traditional\math\compFP.asm
                   jExpEQ   0x0140a4    program     static E:\MPASM_MPLINK_PIC18_LT_Branch_3_42\pic18-lt\cxx-framework\src\traditional\math\compFP.asm
                  jRotate   0x0140b0    program     static E:\MPASM_MPLINK_PIC18_LT_Branch_3_42\pic18-lt\cxx-framework\src\traditional\math\compFP.asm
            __FpReturnNaN   0x0140c2    program     extern E:\MPASM_MPLINK_PIC18_LT_Branch_3_42\pic18-lt\cxx-framework\src\traditional\math\packFP.asm
                 __FpExit   0x0140ce    program     extern E:\MPASM_MPLINK_PIC18_LT_Branch_3_42\pic18-lt\cxx-framework\src\traditional\math\packFP.asm
        __FpReturnSignInf   0x0140d0    program     extern E:\MPASM_MPLINK_PIC18_LT_Branch_3_42\pic18-lt\cxx-framework\src\traditional\math\packFP.asm
         __FpReturnNegInf   0x0140d4    program     extern E:\MPASM_MPLINK_PIC18_LT_Branch_3_42\pic18-lt\cxx-framework\src\traditional\math\packFP.asm
         __FpReturnPosInf   0x0140da    program     extern E:\MPASM_MPLINK_PIC18_LT_Branch_3_42\pic18-lt\cxx-framework\src\traditional\math\packFP.asm
           jReturnPosInf0   0x0140de    program     static E:\MPASM_MPLINK_PIC18_LT_Branch_3_42\pic18-lt\cxx-framework\src\traditional\math\packFP.asm
               jZero1and2   0x0140e2    program     static E:\MPASM_MPLINK_PIC18_LT_Branch_3_42\pic18-lt\cxx-framework\src\traditional\math\packFP.asm
       __FpReturnSignZero   0x0140e8    program     extern E:\MPASM_MPLINK_PIC18_LT_Branch_3_42\pic18-lt\cxx-framework\src\traditional\math\packFP.asm
        __FpReturnNegZero   0x0140ec    program     extern E:\MPASM_MPLINK_PIC18_LT_Branch_3_42\pic18-lt\cxx-framework\src\traditional\math\packFP.asm
        __FpReturnPosZero   0x0140f4    program     extern E:\MPASM_MPLINK_PIC18_LT_Branch_3_42\pic18-lt\cxx-framework\src\traditional\math\packFP.asm
                 __FpPack   0x0140fa    program     extern E:\MPASM_MPLINK_PIC18_LT_Branch_3_42\pic18-lt\cxx-framework\src\traditional\math\packFP.asm
                  jPkLoop   0x014108    program     static E:\MPASM_MPLINK_PIC18_LT_Branch_3_42\pic18-lt\cxx-framework\src\traditional\math\packFP.asm
             jPkShiftDone   0x014124    program     static E:\MPASM_MPLINK_PIC18_LT_Branch_3_42\pic18-lt\cxx-framework\src\traditional\math\packFP.asm
               jPkRoundIt   0x01413a    program     static E:\MPASM_MPLINK_PIC18_LT_Branch_3_42\pic18-lt\cxx-framework\src\traditional\math\packFP.asm
              __FpReturnW   0x014152    program     extern E:\MPASM_MPLINK_PIC18_LT_Branch_3_42\pic18-lt\cxx-framework\src\traditional\math\packFP.asm
             jPkRoundDone   0x014152    program     static E:\MPASM_MPLINK_PIC18_LT_Branch_3_42\pic18-lt\cxx-framework\src\traditional\math\packFP.asm
              __FpUnPackA   0x014172    program     extern E:\MPASM_MPLINK_PIC18_LT_Branch_3_42\pic18-lt\cxx-framework\src\traditional\math\UnpackFP.asm
                  jUnpkA1   0x01417c    program     static E:\MPASM_MPLINK_PIC18_LT_Branch_3_42\pic18-lt\cxx-framework\src\traditional\math\UnpackFP.asm
                 jUnpkANZ   0x01418a    program     static E:\MPASM_MPLINK_PIC18_LT_Branch_3_42\pic18-lt\cxx-framework\src\traditional\math\UnpackFP.asm
                  jUnpkA2   0x014194    program     static E:\MPASM_MPLINK_PIC18_LT_Branch_3_42\pic18-lt\cxx-framework\src\traditional\math\UnpackFP.asm
                 jUnpkNaN   0x01419e    program     static E:\MPASM_MPLINK_PIC18_LT_Branch_3_42\pic18-lt\cxx-framework\src\traditional\math\UnpackFP.asm
              __FpUnPackB   0x0141a2    program     extern E:\MPASM_MPLINK_PIC18_LT_Branch_3_42\pic18-lt\cxx-framework\src\traditional\math\UnpackFP.asm
                  jUnpkB1   0x0141ac    program     static E:\MPASM_MPLINK_PIC18_LT_Branch_3_42\pic18-lt\cxx-framework\src\traditional\math\UnpackFP.asm
                 jUnpkBNZ   0x0141ba    program     static E:\MPASM_MPLINK_PIC18_LT_Branch_3_42\pic18-lt\cxx-framework\src\traditional\math\UnpackFP.asm
                  jUnpkB2   0x0141c4    program     static E:\MPASM_MPLINK_PIC18_LT_Branch_3_42\pic18-lt\cxx-framework\src\traditional\math\UnpackFP.asm
                WriteI2C1   0x0141ce    program     extern E:\MPASM_MPLINK_PIC18_LT_Branch_3_42\pic18-lt\cxx-framework\src\pmc_common\i2c\i2c1writ.c
                 getsI2C1   0x01424e    program     extern E:\MPASM_MPLINK_PIC18_LT_Branch_3_42\pic18-lt\cxx-framework\src\pmc_common\i2c\i2c1gets.c
                 OpenI2C1   0x0142c4    program     extern E:\MPASM_MPLINK_PIC18_LT_Branch_3_42\pic18-lt\cxx-framework\src\pmc_common\i2c\i2c1open.c
                 FXD1616U   0x0142fa    program     extern E:\MPASM_MPLINK_PIC18_LT_Branch_3_42\pic18-lt\cxx-framework\src\traditional\math\fxd1616u.c
                     loop   0x014304    program     static                          
                  endloop   0x014320    program     static                          
       ___return_lbl00000   0x014324    program     static                          
            __zero_memory   0x014326    program     extern E:\MPASM_MPLINK_PIC18_LT_Branch_3_42\pic18-lt\cxx-framework\src\traditional\proc\p18f8723.asm
                   loop_h   0x014334    program     static E:\MPASM_MPLINK_PIC18_LT_Branch_3_42\pic18-lt\cxx-framework\src\traditional\proc\p18f8723.asm
               zero_block   0x014334    program     static E:\MPASM_MPLINK_PIC18_LT_Branch_3_42\pic18-lt\cxx-framework\src\traditional\proc\p18f8723.asm
                compare_l   0x01433c    program     static E:\MPASM_MPLINK_PIC18_LT_Branch_3_42\pic18-lt\cxx-framework\src\traditional\proc\p18f8723.asm
                   loop_l   0x01433e    program     static E:\MPASM_MPLINK_PIC18_LT_Branch_3_42\pic18-lt\cxx-framework\src\traditional\proc\p18f8723.asm
                 FXD0808U   0x014346    program     extern E:\MPASM_MPLINK_PIC18_LT_Branch_3_42\pic18-lt\cxx-framework\src\traditional\math\fxd0808u.c
                     loop   0x01434e    program     static                          
                  endloop   0x01435c    program     static                          
       ___return_lbl00000   0x014360    program     static                          
                 ReadI2C1   0x014362    program     extern E:\MPASM_MPLINK_PIC18_LT_Branch_3_42\pic18-lt\cxx-framework\src\pmc_common\i2c\i2c1read.c
                 _startup   0x01437c    program     extern E:\MPASM_MPLINK_PIC18_LT_Branch_3_42\pic18-lt\cxx-framework\src\traditional\startup\c018.c
                     loop   0x014388    program     static                          
       ___return_lbl00001   0x014392    program     static                          
                   __init   0x014394    program     extern E:\MPASM_MPLINK_PIC18_LT_Branch_3_42\pic18-lt\cxx-framework\src\traditional\stdclib\__init.c
               __config_0   0x300001    program     static C:\Users\LFRAD\Documents\CMS2Luc\ProjetsNettoyesCMSGit\ProjetCarteMere\project\CMSModifV1SD.c
               __config_1   0x300002    program     static C:\Users\LFRAD\Documents\CMS2Luc\ProjetsNettoyesCMSGit\ProjetCarteMere\project\CMSModifV1SD.c
               __config_2   0x300003    program     static C:\Users\LFRAD\Documents\CMS2Luc\ProjetsNettoyesCMSGit\ProjetCarteMere\project\CMSModifV1SD.c
               __config_3   0x300004    program     static C:\Users\LFRAD\Documents\CMS2Luc\ProjetsNettoyesCMSGit\ProjetCarteMere\project\CMSModifV1SD.c
               __config_4   0x300005    program     static C:\Users\LFRAD\Documents\CMS2Luc\ProjetsNettoyesCMSGit\ProjetCarteMere\project\CMSModifV1SD.c
               __config_5   0x300006    program     static C:\Users\LFRAD\Documents\CMS2Luc\ProjetsNettoyesCMSGit\ProjetCarteMere\project\CMSModifV1SD.c
               __config_6   0x300008    program     static C:\Users\LFRAD\Documents\CMS2Luc\ProjetsNettoyesCMSGit\ProjetCarteMere\project\CMSModifV1SD.c
               __config_7   0x300009    program     static C:\Users\LFRAD\Documents\CMS2Luc\ProjetsNettoyesCMSGit\ProjetCarteMere\project\CMSModifV1SD.c
               __config_8   0x30000a    program     static C:\Users\LFRAD\Documents\CMS2Luc\ProjetsNettoyesCMSGit\ProjetCarteMere\project\CMSModifV1SD.c
               __config_9   0x30000b    program     static C:\Users\LFRAD\Documents\CMS2Luc\ProjetsNettoyesCMSGit\ProjetCarteMere\project\CMSModifV1SD.c
              __config_10   0x30000c    program     static C:\Users\LFRAD\Documents\CMS2Luc\ProjetsNettoyesCMSGit\ProjetCarteMere\project\CMSModifV1SD.c
              __config_11   0x30000d    program     static C:\Users\LFRAD\Documents\CMS2Luc\ProjetsNettoyesCMSGit\ProjetCarteMere\project\CMSModifV1SD.c
                     SIGN   0x000000       data     extern E:\MPASM_MPLINK_PIC18_LT_Branch_3_42\pic18-lt\cxx-framework\src\traditional\math\cmath18.asm
            __FPFLAGSbits   0x000001       data     extern E:\MPASM_MPLINK_PIC18_LT_Branch_3_42\pic18-lt\cxx-framework\src\traditional\math\cmath18.asm
                __FPFLAGS   0x000001       data     extern E:\MPASM_MPLINK_PIC18_LT_Branch_3_42\pic18-lt\cxx-framework\src\traditional\math\cmath18.asm
                  __REMB3   0x000002       data     extern E:\MPASM_MPLINK_PIC18_LT_Branch_3_42\pic18-lt\cxx-framework\src\traditional\math\aarg.asm
                 __AARGB7   0x000002       data     extern E:\MPASM_MPLINK_PIC18_LT_Branch_3_42\pic18-lt\cxx-framework\src\traditional\math\aarg.asm
                  __REMB2   0x000003       data     extern E:\MPASM_MPLINK_PIC18_LT_Branch_3_42\pic18-lt\cxx-framework\src\traditional\math\aarg.asm
                 __AARGB6   0x000003       data     extern E:\MPASM_MPLINK_PIC18_LT_Branch_3_42\pic18-lt\cxx-framework\src\traditional\math\aarg.asm
                 __AARGB5   0x000004       data     extern E:\MPASM_MPLINK_PIC18_LT_Branch_3_42\pic18-lt\cxx-framework\src\traditional\math\aarg.asm
                  __REMB1   0x000004       data     extern E:\MPASM_MPLINK_PIC18_LT_Branch_3_42\pic18-lt\cxx-framework\src\traditional\math\aarg.asm
                 __AARGB4   0x000005       data     extern E:\MPASM_MPLINK_PIC18_LT_Branch_3_42\pic18-lt\cxx-framework\src\traditional\math\aarg.asm
                  __REMB0   0x000005       data     extern E:\MPASM_MPLINK_PIC18_LT_Branch_3_42\pic18-lt\cxx-framework\src\traditional\math\aarg.asm
                 __AARGB3   0x000006       data     extern E:\MPASM_MPLINK_PIC18_LT_Branch_3_42\pic18-lt\cxx-framework\src\traditional\math\aarg.asm
                 __AARGB2   0x000007       data     extern E:\MPASM_MPLINK_PIC18_LT_Branch_3_42\pic18-lt\cxx-framework\src\traditional\math\aarg.asm
                 __AARGB1   0x000008       data     extern E:\MPASM_MPLINK_PIC18_LT_Branch_3_42\pic18-lt\cxx-framework\src\traditional\math\aarg.asm
                 __AARGB0   0x000009       data     extern E:\MPASM_MPLINK_PIC18_LT_Branch_3_42\pic18-lt\cxx-framework\src\traditional\math\aarg.asm
                   __AEXP   0x00000a       data     extern E:\MPASM_MPLINK_PIC18_LT_Branch_3_42\pic18-lt\cxx-framework\src\traditional\math\aarg.asm
                 __BARGB3   0x00000b       data     extern E:\MPASM_MPLINK_PIC18_LT_Branch_3_42\pic18-lt\cxx-framework\src\traditional\math\barg.asm
                 __BARGB2   0x00000c       data     extern E:\MPASM_MPLINK_PIC18_LT_Branch_3_42\pic18-lt\cxx-framework\src\traditional\math\barg.asm
                 __BARGB1   0x00000d       data     extern E:\MPASM_MPLINK_PIC18_LT_Branch_3_42\pic18-lt\cxx-framework\src\traditional\math\barg.asm
                 __BARGB0   0x00000e       data     extern E:\MPASM_MPLINK_PIC18_LT_Branch_3_42\pic18-lt\cxx-framework\src\traditional\math\barg.asm
                   __BEXP   0x00000f       data     extern E:\MPASM_MPLINK_PIC18_LT_Branch_3_42\pic18-lt\cxx-framework\src\traditional\math\barg.asm
                 __TEMPB3   0x000010       data     extern E:\MPASM_MPLINK_PIC18_LT_Branch_3_42\pic18-lt\cxx-framework\src\traditional\math\temparg.asm
                 __TEMPB2   0x000011       data     extern E:\MPASM_MPLINK_PIC18_LT_Branch_3_42\pic18-lt\cxx-framework\src\traditional\math\temparg.asm
                 __TEMPB1   0x000012       data     extern E:\MPASM_MPLINK_PIC18_LT_Branch_3_42\pic18-lt\cxx-framework\src\traditional\math\temparg.asm
                   __TEMP   0x000013       data     extern E:\MPASM_MPLINK_PIC18_LT_Branch_3_42\pic18-lt\cxx-framework\src\traditional\math\temparg.asm
                 __TEMPB0   0x000013       data     extern E:\MPASM_MPLINK_PIC18_LT_Branch_3_42\pic18-lt\cxx-framework\src\traditional\math\temparg.asm
                  __tmp_0   0x000014       data     static C:\Users\LFRAD\Documents\CMS2Luc\ProjetsNettoyesCMSGit\ProjetCarteMere\project\CMSModifV1SD.c
                  __tmp_0   0x000014       data     static E:\MPASM_MPLINK_PIC18_LT_Branch_3_42\pic18-lt\cxx-framework\src\pmc_common\i2c\i2c1writ.c
                 TRAMEOUT   0x000100       data     extern C:\Users\LFRAD\Documents\CMS2Luc\ProjetsNettoyesCMSGit\ProjetCarteMere\project\CMSModifV1SD.c
                  TRAMEIN   0x00017d       data     extern C:\Users\LFRAD\Documents\CMS2Luc\ProjetsNettoyesCMSGit\ProjetCarteMere\project\CMSModifV1SD.c
                  VOIECOD   0x000200       data     extern C:\Users\LFRAD\Documents\CMS2Luc\ProjetsNettoyesCMSGit\ProjetCarteMere\project\CMSModifV1SD.c
                     TYPE   0x000206       data     extern C:\Users\LFRAD\Documents\CMS2Luc\ProjetsNettoyesCMSGit\ProjetCarteMere\project\CMSModifV1SD.c
                     CMOD   0x000207       data     extern C:\Users\LFRAD\Documents\CMS2Luc\ProjetsNettoyesCMSGit\ProjetCarteMere\project\CMSModifV1SD.c
                     CCON   0x00020b       data     extern C:\Users\LFRAD\Documents\CMS2Luc\ProjetsNettoyesCMSGit\ProjetCarteMere\project\CMSModifV1SD.c
                     CREP   0x00020f       data     extern C:\Users\LFRAD\Documents\CMS2Luc\ProjetsNettoyesCMSGit\ProjetCarteMere\project\CMSModifV1SD.c
             CONSTITUTION   0x000213       data     extern C:\Users\LFRAD\Documents\CMS2Luc\ProjetsNettoyesCMSGit\ProjetCarteMere\project\CMSModifV1SD.c
              COMMENTAIRE   0x000220       data     extern C:\Users\LFRAD\Documents\CMS2Luc\ProjetsNettoyesCMSGit\ProjetCarteMere\project\CMSModifV1SD.c
                    CABLE   0x000234       data     extern C:\Users\LFRAD\Documents\CMS2Luc\ProjetsNettoyesCMSGit\ProjetCarteMere\project\CMSModifV1SD.c
                       JJ   0x000237       data     extern C:\Users\LFRAD\Documents\CMS2Luc\ProjetsNettoyesCMSGit\ProjetCarteMere\project\CMSModifV1SD.c
                       MM   0x000239       data     extern C:\Users\LFRAD\Documents\CMS2Luc\ProjetsNettoyesCMSGit\ProjetCarteMere\project\CMSModifV1SD.c
                       HH   0x00023b       data     extern C:\Users\LFRAD\Documents\CMS2Luc\ProjetsNettoyesCMSGit\ProjetCarteMere\project\CMSModifV1SD.c
                       mm   0x00023d       data     extern C:\Users\LFRAD\Documents\CMS2Luc\ProjetsNettoyesCMSGit\ProjetCarteMere\project\CMSModifV1SD.c
                       ii   0x00023f       data     extern C:\Users\LFRAD\Documents\CMS2Luc\ProjetsNettoyesCMSGit\ProjetCarteMere\project\CMSModifV1SD.c
                      COD   0x000240       data     extern C:\Users\LFRAD\Documents\CMS2Luc\ProjetsNettoyesCMSGit\ProjetCarteMere\project\CMSModifV1SD.c
                      POS   0x000242       data     extern C:\Users\LFRAD\Documents\CMS2Luc\ProjetsNettoyesCMSGit\ProjetCarteMere\project\CMSModifV1SD.c
                     iiii   0x000244       data     extern C:\Users\LFRAD\Documents\CMS2Luc\ProjetsNettoyesCMSGit\ProjetCarteMere\project\CMSModifV1SD.c
                 DISTANCE   0x000248       data     extern C:\Users\LFRAD\Documents\CMS2Luc\ProjetsNettoyesCMSGit\ProjetCarteMere\project\CMSModifV1SD.c
                     ETAT   0x00024d       data     extern C:\Users\LFRAD\Documents\CMS2Luc\ProjetsNettoyesCMSGit\ProjetCarteMere\project\CMSModifV1SD.c
                   VALEUR   0x00024f       data     extern C:\Users\LFRAD\Documents\CMS2Luc\ProjetsNettoyesCMSGit\ProjetCarteMere\project\CMSModifV1SD.c
                    SEUIL   0x000253       data     extern C:\Users\LFRAD\Documents\CMS2Luc\ProjetsNettoyesCMSGit\ProjetCarteMere\project\CMSModifV1SD.c
                TYPECARTE   0x000257       data     extern C:\Users\LFRAD\Documents\CMS2Luc\ProjetsNettoyesCMSGit\ProjetCarteMere\project\CMSModifV1SD.c
                    START   0x00025c       data     extern C:\Users\LFRAD\Documents\CMS2Luc\ProjetsNettoyesCMSGit\ProjetCarteMere\project\CMSModifV1SD.c
                      ID1   0x00025d       data     extern C:\Users\LFRAD\Documents\CMS2Luc\ProjetsNettoyesCMSGit\ProjetCarteMere\project\CMSModifV1SD.c
                      ID2   0x00025f       data     extern C:\Users\LFRAD\Documents\CMS2Luc\ProjetsNettoyesCMSGit\ProjetCarteMere\project\CMSModifV1SD.c
                 FONCTION   0x000261       data     extern C:\Users\LFRAD\Documents\CMS2Luc\ProjetsNettoyesCMSGit\ProjetCarteMere\project\CMSModifV1SD.c
                      CRC   0x000264       data     extern C:\Users\LFRAD\Documents\CMS2Luc\ProjetsNettoyesCMSGit\ProjetCarteMere\project\CMSModifV1SD.c
                     STOP   0x000269       data     extern C:\Users\LFRAD\Documents\CMS2Luc\ProjetsNettoyesCMSGit\ProjetCarteMere\project\CMSModifV1SD.c
              TYPE_ERREUR   0x00026a       data     extern C:\Users\LFRAD\Documents\CMS2Luc\ProjetsNettoyesCMSGit\ProjetCarteMere\project\CMSModifV1SD.c
       INFORMATION_ERREUR   0x00026c       data     extern C:\Users\LFRAD\Documents\CMS2Luc\ProjetsNettoyesCMSGit\ProjetCarteMere\project\CMSModifV1SD.c
       NBRECAPTEURS_CABLE   0x000280       data     extern C:\Users\LFRAD\Documents\CMS2Luc\ProjetsNettoyesCMSGit\ProjetCarteMere\project\CMSModifV1SD.c
             PRIO_AUTO_IO   0x000281       data     extern C:\Users\LFRAD\Documents\CMS2Luc\ProjetsNettoyesCMSGit\ProjetCarteMere\project\CMSModifV1SD.c
                  HORLOGE   0x000282       data     extern C:\Users\LFRAD\Documents\CMS2Luc\ProjetsNettoyesCMSGit\ProjetCarteMere\project\CMSModifV1SD.c
        CAPTEUR_A_EFFACER   0x00028e       data     extern C:\Users\LFRAD\Documents\CMS2Luc\ProjetsNettoyesCMSGit\ProjetCarteMere\project\CMSModifV1SD.c
   DEMANDE_INFOS_CAPTEURS   0x000293       data     extern C:\Users\LFRAD\Documents\CMS2Luc\ProjetsNettoyesCMSGit\ProjetCarteMere\project\CMSModifV1SD.c
             OEIL_CAPTEUR   0x00029d       data     extern C:\Users\LFRAD\Documents\CMS2Luc\ProjetsNettoyesCMSGit\ProjetCarteMere\project\CMSModifV1SD.c
                     PAGE   0x0002a2       data     extern C:\Users\LFRAD\Documents\CMS2Luc\ProjetsNettoyesCMSGit\ProjetCarteMere\project\CMSModifV1SD.c
              INSTRUCTION   0x0002a8       data     extern C:\Users\LFRAD\Documents\CMS2Luc\ProjetsNettoyesCMSGit\ProjetCarteMere\project\CMSModifV1SD.c
               capt_exist   0x0002c1       data     extern C:\Users\LFRAD\Documents\CMS2Luc\ProjetsNettoyesCMSGit\ProjetCarteMere\project\CMSModifV1SD.c
                     VDD1   0x0002c2       data     extern C:\Users\LFRAD\Documents\CMS2Luc\ProjetsNettoyesCMSGit\ProjetCarteMere\project\CMSModifV1SD.c
                     VDD2   0x0002c6       data     extern C:\Users\LFRAD\Documents\CMS2Luc\ProjetsNettoyesCMSGit\ProjetCarteMere\project\CMSModifV1SD.c
                     VDD3   0x0002ca       data     extern C:\Users\LFRAD\Documents\CMS2Luc\ProjetsNettoyesCMSGit\ProjetCarteMere\project\CMSModifV1SD.c
                     VDD4   0x0002ce       data     extern C:\Users\LFRAD\Documents\CMS2Luc\ProjetsNettoyesCMSGit\ProjetCarteMere\project\CMSModifV1SD.c
                     VDD5   0x0002d2       data     extern C:\Users\LFRAD\Documents\CMS2Luc\ProjetsNettoyesCMSGit\ProjetCarteMere\project\CMSModifV1SD.c
                    Vtemp   0x0002d6       data     extern C:\Users\LFRAD\Documents\CMS2Luc\ProjetsNettoyesCMSGit\ProjetCarteMere\project\CMSModifV1SD.c
                     VDD6   0x0002da       data     extern C:\Users\LFRAD\Documents\CMS2Luc\ProjetsNettoyesCMSGit\ProjetCarteMere\project\CMSModifV1SD.c
                     VBAT   0x0002de       data     extern C:\Users\LFRAD\Documents\CMS2Luc\ProjetsNettoyesCMSGit\ProjetCarteMere\project\CMSModifV1SD.c
              NORECEPTION   0x0002e2       data     extern C:\Users\LFRAD\Documents\CMS2Luc\ProjetsNettoyesCMSGit\ProjetCarteMere\project\CMSModifV1SD.c
          pointeur_out_in   0x0002e3       data     extern C:\Users\LFRAD\Documents\CMS2Luc\ProjetsNettoyesCMSGit\ProjetCarteMere\project\CMSModifV1SD.c
                      tmp   0x0002e5       data     extern C:\Users\LFRAD\Documents\CMS2Luc\ProjetsNettoyesCMSGit\ProjetCarteMere\project\CMSModifV1SD.c
                     tmp2   0x0002e6       data     extern C:\Users\LFRAD\Documents\CMS2Luc\ProjetsNettoyesCMSGit\ProjetCarteMere\project\CMSModifV1SD.c
                     TMPI   0x0002e7       data     extern C:\Users\LFRAD\Documents\CMS2Luc\ProjetsNettoyesCMSGit\ProjetCarteMere\project\CMSModifV1SD.c
                 ENTREES1   0x0002e9       data     extern C:\Users\LFRAD\Documents\CMS2Luc\ProjetsNettoyesCMSGit\ProjetCarteMere\project\CMSModifV1SD.c
                 ENTREES2   0x0002ea       data     extern C:\Users\LFRAD\Documents\CMS2Luc\ProjetsNettoyesCMSGit\ProjetCarteMere\project\CMSModifV1SD.c
                    HEURE   0x0002eb       data     extern C:\Users\LFRAD\Documents\CMS2Luc\ProjetsNettoyesCMSGit\ProjetCarteMere\project\CMSModifV1SD.c
                   MINUTE   0x0002ec       data     extern C:\Users\LFRAD\Documents\CMS2Luc\ProjetsNettoyesCMSGit\ProjetCarteMere\project\CMSModifV1SD.c
                  SECONDE   0x0002ed       data     extern C:\Users\LFRAD\Documents\CMS2Luc\ProjetsNettoyesCMSGit\ProjetCarteMere\project\CMSModifV1SD.c
                     MOIS   0x0002ee       data     extern C:\Users\LFRAD\Documents\CMS2Luc\ProjetsNettoyesCMSGit\ProjetCarteMere\project\CMSModifV1SD.c
                     JOUR   0x0002ef       data     extern C:\Users\LFRAD\Documents\CMS2Luc\ProjetsNettoyesCMSGit\ProjetCarteMere\project\CMSModifV1SD.c
                    ANNEE   0x0002f0       data     extern C:\Users\LFRAD\Documents\CMS2Luc\ProjetsNettoyesCMSGit\ProjetCarteMere\project\CMSModifV1SD.c
                     DATE   0x0002f1       data     extern C:\Users\LFRAD\Documents\CMS2Luc\ProjetsNettoyesCMSGit\ProjetCarteMere\project\CMSModifV1SD.c
                      TMP   0x000300       data     extern C:\Users\LFRAD\Documents\CMS2Luc\ProjetsNettoyesCMSGit\ProjetCarteMere\project\CMSModifV1SD.c
              P_RESERVOIR   0x00037d       data     extern C:\Users\LFRAD\Documents\CMS2Luc\ProjetsNettoyesCMSGit\ProjetCarteMere\project\CMSModifV1SD.c
                 P_SORTIE   0x00038c       data     extern C:\Users\LFRAD\Documents\CMS2Luc\ProjetsNettoyesCMSGit\ProjetCarteMere\project\CMSModifV1SD.c
                P_SECOURS   0x00039b       data     extern C:\Users\LFRAD\Documents\CMS2Luc\ProjetsNettoyesCMSGit\ProjetCarteMere\project\CMSModifV1SD.c
              POINT_ROSEE   0x0003aa       data     extern C:\Users\LFRAD\Documents\CMS2Luc\ProjetsNettoyesCMSGit\ProjetCarteMere\project\CMSModifV1SD.c
             DEBIT_GLOBAL   0x0003b5       data     extern C:\Users\LFRAD\Documents\CMS2Luc\ProjetsNettoyesCMSGit\ProjetCarteMere\project\CMSModifV1SD.c
       TEMPS_CYCLE_MOTEUR   0x0003c0       data     extern C:\Users\LFRAD\Documents\CMS2Luc\ProjetsNettoyesCMSGit\ProjetCarteMere\project\CMSModifV1SD.c
             TEMPS_MOTEUR   0x0003cb       data     extern C:\Users\LFRAD\Documents\CMS2Luc\ProjetsNettoyesCMSGit\ProjetCarteMere\project\CMSModifV1SD.c
            PRESENCE_220V   0x0003da       data     extern C:\Users\LFRAD\Documents\CMS2Luc\ProjetsNettoyesCMSGit\ProjetCarteMere\project\CMSModifV1SD.c
             PRESENCE_48V   0x0003e0       data     extern C:\Users\LFRAD\Documents\CMS2Luc\ProjetsNettoyesCMSGit\ProjetCarteMere\project\CMSModifV1SD.c
                  DATAFIX   0x0003e6       data     extern C:\Users\LFRAD\Documents\CMS2Luc\ProjetsNettoyesCMSGit\ProjetCarteMere\project\CMSModifV1SD.c
                   SAVTAB   0x000f00       data     extern C:\Users\LFRAD\Documents\CMS2Luc\ProjetsNettoyesCMSGit\ProjetCarteMere\project\CMSModifV1SD.c
               calculBLOC   0x000f19       data     extern C:\Users\LFRAD\Documents\CMS2Luc\ProjetsNettoyesCMSGit\ProjetCarteMere\project\CMSModifV1SD.c
 FONCTION_ACTIVATION_AUTO   0x000f1b       data     extern C:\Users\LFRAD\Documents\CMS2Luc\ProjetsNettoyesCMSGit\ProjetCarteMere\project\CMSModifV1SD.c
             numdecarteRI   0x000f1c       data     extern C:\Users\LFRAD\Documents\CMS2Luc\ProjetsNettoyesCMSGit\ProjetCarteMere\project\CMSModifV1SD.c
         TROPDENONREPONSE   0x000f1d       data     extern C:\Users\LFRAD\Documents\CMS2Luc\ProjetsNettoyesCMSGit\ProjetCarteMere\project\CMSModifV1SD.c
                 CRC_ETAT   0x000f1e       data     extern C:\Users\LFRAD\Documents\CMS2Luc\ProjetsNettoyesCMSGit\ProjetCarteMere\project\CMSModifV1SD.c
                  ETAT_IO   0x000f1f       data     extern C:\Users\LFRAD\Documents\CMS2Luc\ProjetsNettoyesCMSGit\ProjetCarteMere\project\CMSModifV1SD.c
              FIRST_DEMAR   0x000f20       data     extern C:\Users\LFRAD\Documents\CMS2Luc\ProjetsNettoyesCMSGit\ProjetCarteMere\project\CMSModifV1SD.c
                MODERAPID   0x000f21       data     extern C:\Users\LFRAD\Documents\CMS2Luc\ProjetsNettoyesCMSGit\ProjetCarteMere\project\CMSModifV1SD.c
             TYPECOMMANDE   0x000f22       data     extern C:\Users\LFRAD\Documents\CMS2Luc\ProjetsNettoyesCMSGit\ProjetCarteMere\project\CMSModifV1SD.c
         temoinfinvoieZIZ   0x000f23       data     extern C:\Users\LFRAD\Documents\CMS2Luc\ProjetsNettoyesCMSGit\ProjetCarteMere\project\CMSModifV1SD.c
                IOTRAVAIL   0x000f24       data     extern C:\Users\LFRAD\Documents\CMS2Luc\ProjetsNettoyesCMSGit\ProjetCarteMere\project\CMSModifV1SD.c
                  PASDE_S   0x000f25       data     extern C:\Users\LFRAD\Documents\CMS2Luc\ProjetsNettoyesCMSGit\ProjetCarteMere\project\CMSModifV1SD.c
                   cycleN   0x000f26       data     extern C:\Users\LFRAD\Documents\CMS2Luc\ProjetsNettoyesCMSGit\ProjetCarteMere\project\CMSModifV1SD.c
             RESCRUTATION   0x000f27       data     extern C:\Users\LFRAD\Documents\CMS2Luc\ProjetsNettoyesCMSGit\ProjetCarteMere\project\CMSModifV1SD.c
              NUMEROCARTE   0x000f28       data     extern C:\Users\LFRAD\Documents\CMS2Luc\ProjetsNettoyesCMSGit\ProjetCarteMere\project\CMSModifV1SD.c
            NBREDEMANDEIO   0x000f29       data     extern C:\Users\LFRAD\Documents\CMS2Luc\ProjetsNettoyesCMSGit\ProjetCarteMere\project\CMSModifV1SD.c
          PRESENCEDEBITSD   0x000f2a       data     extern C:\Users\LFRAD\Documents\CMS2Luc\ProjetsNettoyesCMSGit\ProjetCarteMere\project\CMSModifV1SD.c
                  R1NOREP   0x000f2b       data     extern C:\Users\LFRAD\Documents\CMS2Luc\ProjetsNettoyesCMSGit\ProjetCarteMere\project\CMSModifV1SD.c
                  R2NOREP   0x000f2c       data     extern C:\Users\LFRAD\Documents\CMS2Luc\ProjetsNettoyesCMSGit\ProjetCarteMere\project\CMSModifV1SD.c
                  R3NOREP   0x000f2d       data     extern C:\Users\LFRAD\Documents\CMS2Luc\ProjetsNettoyesCMSGit\ProjetCarteMere\project\CMSModifV1SD.c
                  R4NOREP   0x000f2e       data     extern C:\Users\LFRAD\Documents\CMS2Luc\ProjetsNettoyesCMSGit\ProjetCarteMere\project\CMSModifV1SD.c
                  R5NOREP   0x000f2f       data     extern C:\Users\LFRAD\Documents\CMS2Luc\ProjetsNettoyesCMSGit\ProjetCarteMere\project\CMSModifV1SD.c
               UNRESETRI1   0x000f30       data     extern C:\Users\LFRAD\Documents\CMS2Luc\ProjetsNettoyesCMSGit\ProjetCarteMere\project\CMSModifV1SD.c
               UNRESETRI2   0x000f31       data     extern C:\Users\LFRAD\Documents\CMS2Luc\ProjetsNettoyesCMSGit\ProjetCarteMere\project\CMSModifV1SD.c
               UNRESETRI3   0x000f32       data     extern C:\Users\LFRAD\Documents\CMS2Luc\ProjetsNettoyesCMSGit\ProjetCarteMere\project\CMSModifV1SD.c
               UNRESETRI4   0x000f33       data     extern C:\Users\LFRAD\Documents\CMS2Luc\ProjetsNettoyesCMSGit\ProjetCarteMere\project\CMSModifV1SD.c
               UNRESETRI5   0x000f34       data     extern C:\Users\LFRAD\Documents\CMS2Luc\ProjetsNettoyesCMSGit\ProjetCarteMere\project\CMSModifV1SD.c
              MINIRESETRI   0x000f35       data     extern C:\Users\LFRAD\Documents\CMS2Luc\ProjetsNettoyesCMSGit\ProjetCarteMere\project\CMSModifV1SD.c
          TYPEDECARTEOEIL   0x000f36       data     extern C:\Users\LFRAD\Documents\CMS2Luc\ProjetsNettoyesCMSGit\ProjetCarteMere\project\CMSModifV1SD.c
             TIMEOUTCYCLE   0x000f37       data     extern C:\Users\LFRAD\Documents\CMS2Luc\ProjetsNettoyesCMSGit\ProjetCarteMere\project\CMSModifV1SD.c
        scrutationunevoie   0x000f39       data     extern C:\Users\LFRAD\Documents\CMS2Luc\ProjetsNettoyesCMSGit\ProjetCarteMere\project\CMSModifV1SD.c
   ETATZIZCRATIONAUTOMATE   0x000f3a       data     extern C:\Users\LFRAD\Documents\CMS2Luc\ProjetsNettoyesCMSGit\ProjetCarteMere\project\CMSModifV1SD.c
             mouchardINT0   0x000f3b       data     extern C:\Users\LFRAD\Documents\CMS2Luc\ProjetsNettoyesCMSGit\ProjetCarteMere\project\CMSModifV1SD.c
             DEMANDEZIGIO   0x000f3c       data     extern C:\Users\LFRAD\Documents\CMS2Luc\ProjetsNettoyesCMSGit\ProjetCarteMere\project\CMSModifV1SD.c
           resetheurefixe   0x000f3d       data     extern C:\Users\LFRAD\Documents\CMS2Luc\ProjetsNettoyesCMSGit\ProjetCarteMere\project\CMSModifV1SD.c
             SAVAUTOCYCLE   0x000f3e       data     extern C:\Users\LFRAD\Documents\CMS2Luc\ProjetsNettoyesCMSGit\ProjetCarteMere\project\CMSModifV1SD.c
                  MAXBITE   0x000f3f       data     extern C:\Users\LFRAD\Documents\CMS2Luc\ProjetsNettoyesCMSGit\ProjetCarteMere\project\CMSModifV1SD.c
                  MAJBLOC   0x000f40       data     extern C:\Users\LFRAD\Documents\CMS2Luc\ProjetsNettoyesCMSGit\ProjetCarteMere\project\CMSModifV1SD.c
             DEMANDEZPLIO   0x000f41       data     extern C:\Users\LFRAD\Documents\CMS2Luc\ProjetsNettoyesCMSGit\ProjetCarteMere\project\CMSModifV1SD.c
                    ERRMM   0x000f42       data     extern C:\Users\LFRAD\Documents\CMS2Luc\ProjetsNettoyesCMSGit\ProjetCarteMere\project\CMSModifV1SD.c
                     NBMM   0x000f43       data     extern C:\Users\LFRAD\Documents\CMS2Luc\ProjetsNettoyesCMSGit\ProjetCarteMere\project\CMSModifV1SD.c
                   FCYCLE   0x000f44       data     extern C:\Users\LFRAD\Documents\CMS2Luc\ProjetsNettoyesCMSGit\ProjetCarteMere\project\CMSModifV1SD.c
                TESTCYCLE   0x000f45       data     extern C:\Users\LFRAD\Documents\CMS2Luc\ProjetsNettoyesCMSGit\ProjetCarteMere\project\CMSModifV1SD.c
             SSP2CON2bits   0x000f62       data     extern E:\MPASM_MPLINK_PIC18_LT_Branch_3_42\pic18-lt\cxx-framework\src\traditional\proc\p18f8723.asm
                 SSP2CON2   0x000f62       data     extern E:\MPASM_MPLINK_PIC18_LT_Branch_3_42\pic18-lt\cxx-framework\src\traditional\proc\p18f8723.asm
             SSP2CON1bits   0x000f63       data     extern E:\MPASM_MPLINK_PIC18_LT_Branch_3_42\pic18-lt\cxx-framework\src\traditional\proc\p18f8723.asm
                 SSP2CON1   0x000f63       data     extern E:\MPASM_MPLINK_PIC18_LT_Branch_3_42\pic18-lt\cxx-framework\src\traditional\proc\p18f8723.asm
                 SSP2STAT   0x000f64       data     extern E:\MPASM_MPLINK_PIC18_LT_Branch_3_42\pic18-lt\cxx-framework\src\traditional\proc\p18f8723.asm
             SSP2STATbits   0x000f64       data     extern E:\MPASM_MPLINK_PIC18_LT_Branch_3_42\pic18-lt\cxx-framework\src\traditional\proc\p18f8723.asm
                  SSP2ADD   0x000f65       data     extern E:\MPASM_MPLINK_PIC18_LT_Branch_3_42\pic18-lt\cxx-framework\src\traditional\proc\p18f8723.asm
                  SSP2BUF   0x000f66       data     extern E:\MPASM_MPLINK_PIC18_LT_Branch_3_42\pic18-lt\cxx-framework\src\traditional\proc\p18f8723.asm
                 ECCP2DEL   0x000f67       data     extern E:\MPASM_MPLINK_PIC18_LT_Branch_3_42\pic18-lt\cxx-framework\src\traditional\proc\p18f8723.asm
             ECCP2DELbits   0x000f67       data     extern E:\MPASM_MPLINK_PIC18_LT_Branch_3_42\pic18-lt\cxx-framework\src\traditional\proc\p18f8723.asm
                  ECCP2AS   0x000f68       data     extern E:\MPASM_MPLINK_PIC18_LT_Branch_3_42\pic18-lt\cxx-framework\src\traditional\proc\p18f8723.asm
              ECCP2ASbits   0x000f68       data     extern E:\MPASM_MPLINK_PIC18_LT_Branch_3_42\pic18-lt\cxx-framework\src\traditional\proc\p18f8723.asm
                 ECCP3DEL   0x000f69       data     extern E:\MPASM_MPLINK_PIC18_LT_Branch_3_42\pic18-lt\cxx-framework\src\traditional\proc\p18f8723.asm
             ECCP3DELbits   0x000f69       data     extern E:\MPASM_MPLINK_PIC18_LT_Branch_3_42\pic18-lt\cxx-framework\src\traditional\proc\p18f8723.asm
              ECCP3ASbits   0x000f6a       data     extern E:\MPASM_MPLINK_PIC18_LT_Branch_3_42\pic18-lt\cxx-framework\src\traditional\proc\p18f8723.asm
                  ECCP3AS   0x000f6a       data     extern E:\MPASM_MPLINK_PIC18_LT_Branch_3_42\pic18-lt\cxx-framework\src\traditional\proc\p18f8723.asm
               RCSTA2bits   0x000f6b       data     extern E:\MPASM_MPLINK_PIC18_LT_Branch_3_42\pic18-lt\cxx-framework\src\traditional\proc\p18f8723.asm
                   RCSTA2   0x000f6b       data     extern E:\MPASM_MPLINK_PIC18_LT_Branch_3_42\pic18-lt\cxx-framework\src\traditional\proc\p18f8723.asm
               TXSTA2bits   0x000f6c       data     extern E:\MPASM_MPLINK_PIC18_LT_Branch_3_42\pic18-lt\cxx-framework\src\traditional\proc\p18f8723.asm
                   TXSTA2   0x000f6c       data     extern E:\MPASM_MPLINK_PIC18_LT_Branch_3_42\pic18-lt\cxx-framework\src\traditional\proc\p18f8723.asm
                   TXREG2   0x000f6d       data     extern E:\MPASM_MPLINK_PIC18_LT_Branch_3_42\pic18-lt\cxx-framework\src\traditional\proc\p18f8723.asm
                   RCREG2   0x000f6e       data     extern E:\MPASM_MPLINK_PIC18_LT_Branch_3_42\pic18-lt\cxx-framework\src\traditional\proc\p18f8723.asm
                   SPBRG2   0x000f6f       data     extern E:\MPASM_MPLINK_PIC18_LT_Branch_3_42\pic18-lt\cxx-framework\src\traditional\proc\p18f8723.asm
              CCP5CONbits   0x000f70       data     extern E:\MPASM_MPLINK_PIC18_LT_Branch_3_42\pic18-lt\cxx-framework\src\traditional\proc\p18f8723.asm
                  CCP5CON   0x000f70       data     extern E:\MPASM_MPLINK_PIC18_LT_Branch_3_42\pic18-lt\cxx-framework\src\traditional\proc\p18f8723.asm
                    CCPR5   0x000f71       data     extern E:\MPASM_MPLINK_PIC18_LT_Branch_3_42\pic18-lt\cxx-framework\src\traditional\proc\p18f8723.asm
                   CCPR5L   0x000f71       data     extern E:\MPASM_MPLINK_PIC18_LT_Branch_3_42\pic18-lt\cxx-framework\src\traditional\proc\p18f8723.asm
                   CCPR5H   0x000f72       data     extern E:\MPASM_MPLINK_PIC18_LT_Branch_3_42\pic18-lt\cxx-framework\src\traditional\proc\p18f8723.asm
              CCP4CONbits   0x000f73       data     extern E:\MPASM_MPLINK_PIC18_LT_Branch_3_42\pic18-lt\cxx-framework\src\traditional\proc\p18f8723.asm
                  CCP4CON   0x000f73       data     extern E:\MPASM_MPLINK_PIC18_LT_Branch_3_42\pic18-lt\cxx-framework\src\traditional\proc\p18f8723.asm
                   CCPR4L   0x000f74       data     extern E:\MPASM_MPLINK_PIC18_LT_Branch_3_42\pic18-lt\cxx-framework\src\traditional\proc\p18f8723.asm
                    CCPR4   0x000f74       data     extern E:\MPASM_MPLINK_PIC18_LT_Branch_3_42\pic18-lt\cxx-framework\src\traditional\proc\p18f8723.asm
                   CCPR4H   0x000f75       data     extern E:\MPASM_MPLINK_PIC18_LT_Branch_3_42\pic18-lt\cxx-framework\src\traditional\proc\p18f8723.asm
                    T4CON   0x000f76       data     extern E:\MPASM_MPLINK_PIC18_LT_Branch_3_42\pic18-lt\cxx-framework\src\traditional\proc\p18f8723.asm
                T4CONbits   0x000f76       data     extern E:\MPASM_MPLINK_PIC18_LT_Branch_3_42\pic18-lt\cxx-framework\src\traditional\proc\p18f8723.asm
                      PR4   0x000f77       data     extern E:\MPASM_MPLINK_PIC18_LT_Branch_3_42\pic18-lt\cxx-framework\src\traditional\proc\p18f8723.asm
                     TMR4   0x000f78       data     extern E:\MPASM_MPLINK_PIC18_LT_Branch_3_42\pic18-lt\cxx-framework\src\traditional\proc\p18f8723.asm
                 ECCP1DEL   0x000f79       data     extern E:\MPASM_MPLINK_PIC18_LT_Branch_3_42\pic18-lt\cxx-framework\src\traditional\proc\p18f8723.asm
             ECCP1DELbits   0x000f79       data     extern E:\MPASM_MPLINK_PIC18_LT_Branch_3_42\pic18-lt\cxx-framework\src\traditional\proc\p18f8723.asm
             BAUDCON2bits   0x000f7c       data     extern E:\MPASM_MPLINK_PIC18_LT_Branch_3_42\pic18-lt\cxx-framework\src\traditional\proc\p18f8723.asm
                 BAUDCON2   0x000f7c       data     extern E:\MPASM_MPLINK_PIC18_LT_Branch_3_42\pic18-lt\cxx-framework\src\traditional\proc\p18f8723.asm
                  SPBRGH2   0x000f7d       data     extern E:\MPASM_MPLINK_PIC18_LT_Branch_3_42\pic18-lt\cxx-framework\src\traditional\proc\p18f8723.asm
             BAUDCON1bits   0x000f7e       data     extern E:\MPASM_MPLINK_PIC18_LT_Branch_3_42\pic18-lt\cxx-framework\src\traditional\proc\p18f8723.asm
                 BAUDCON1   0x000f7e       data     extern E:\MPASM_MPLINK_PIC18_LT_Branch_3_42\pic18-lt\cxx-framework\src\traditional\proc\p18f8723.asm
                  BAUDCON   0x000f7e       data     extern E:\MPASM_MPLINK_PIC18_LT_Branch_3_42\pic18-lt\cxx-framework\src\traditional\proc\p18f8723.asm
              BAUDCONbits   0x000f7e       data     extern E:\MPASM_MPLINK_PIC18_LT_Branch_3_42\pic18-lt\cxx-framework\src\traditional\proc\p18f8723.asm
                  SPBRGH1   0x000f7f       data     extern E:\MPASM_MPLINK_PIC18_LT_Branch_3_42\pic18-lt\cxx-framework\src\traditional\proc\p18f8723.asm
                   SPBRGH   0x000f7f       data     extern E:\MPASM_MPLINK_PIC18_LT_Branch_3_42\pic18-lt\cxx-framework\src\traditional\proc\p18f8723.asm
                PORTAbits   0x000f80       data     extern E:\MPASM_MPLINK_PIC18_LT_Branch_3_42\pic18-lt\cxx-framework\src\traditional\proc\p18f8723.asm
                    PORTA   0x000f80       data     extern E:\MPASM_MPLINK_PIC18_LT_Branch_3_42\pic18-lt\cxx-framework\src\traditional\proc\p18f8723.asm
                PORTBbits   0x000f81       data     extern E:\MPASM_MPLINK_PIC18_LT_Branch_3_42\pic18-lt\cxx-framework\src\traditional\proc\p18f8723.asm
                    PORTB   0x000f81       data     extern E:\MPASM_MPLINK_PIC18_LT_Branch_3_42\pic18-lt\cxx-framework\src\traditional\proc\p18f8723.asm
                PORTCbits   0x000f82       data     extern E:\MPASM_MPLINK_PIC18_LT_Branch_3_42\pic18-lt\cxx-framework\src\traditional\proc\p18f8723.asm
                    PORTC   0x000f82       data     extern E:\MPASM_MPLINK_PIC18_LT_Branch_3_42\pic18-lt\cxx-framework\src\traditional\proc\p18f8723.asm
                PORTDbits   0x000f83       data     extern E:\MPASM_MPLINK_PIC18_LT_Branch_3_42\pic18-lt\cxx-framework\src\traditional\proc\p18f8723.asm
                    PORTD   0x000f83       data     extern E:\MPASM_MPLINK_PIC18_LT_Branch_3_42\pic18-lt\cxx-framework\src\traditional\proc\p18f8723.asm
                    PORTE   0x000f84       data     extern E:\MPASM_MPLINK_PIC18_LT_Branch_3_42\pic18-lt\cxx-framework\src\traditional\proc\p18f8723.asm
                PORTEbits   0x000f84       data     extern E:\MPASM_MPLINK_PIC18_LT_Branch_3_42\pic18-lt\cxx-framework\src\traditional\proc\p18f8723.asm
                    PORTF   0x000f85       data     extern E:\MPASM_MPLINK_PIC18_LT_Branch_3_42\pic18-lt\cxx-framework\src\traditional\proc\p18f8723.asm
                PORTFbits   0x000f85       data     extern E:\MPASM_MPLINK_PIC18_LT_Branch_3_42\pic18-lt\cxx-framework\src\traditional\proc\p18f8723.asm
                    PORTG   0x000f86       data     extern E:\MPASM_MPLINK_PIC18_LT_Branch_3_42\pic18-lt\cxx-framework\src\traditional\proc\p18f8723.asm
                PORTGbits   0x000f86       data     extern E:\MPASM_MPLINK_PIC18_LT_Branch_3_42\pic18-lt\cxx-framework\src\traditional\proc\p18f8723.asm
                PORTHbits   0x000f87       data     extern E:\MPASM_MPLINK_PIC18_LT_Branch_3_42\pic18-lt\cxx-framework\src\traditional\proc\p18f8723.asm
                    PORTH   0x000f87       data     extern E:\MPASM_MPLINK_PIC18_LT_Branch_3_42\pic18-lt\cxx-framework\src\traditional\proc\p18f8723.asm
                PORTJbits   0x000f88       data     extern E:\MPASM_MPLINK_PIC18_LT_Branch_3_42\pic18-lt\cxx-framework\src\traditional\proc\p18f8723.asm
                    PORTJ   0x000f88       data     extern E:\MPASM_MPLINK_PIC18_LT_Branch_3_42\pic18-lt\cxx-framework\src\traditional\proc\p18f8723.asm
                 LATAbits   0x000f89       data     extern E:\MPASM_MPLINK_PIC18_LT_Branch_3_42\pic18-lt\cxx-framework\src\traditional\proc\p18f8723.asm
                     LATA   0x000f89       data     extern E:\MPASM_MPLINK_PIC18_LT_Branch_3_42\pic18-lt\cxx-framework\src\traditional\proc\p18f8723.asm
                 LATBbits   0x000f8a       data     extern E:\MPASM_MPLINK_PIC18_LT_Branch_3_42\pic18-lt\cxx-framework\src\traditional\proc\p18f8723.asm
                     LATB   0x000f8a       data     extern E:\MPASM_MPLINK_PIC18_LT_Branch_3_42\pic18-lt\cxx-framework\src\traditional\proc\p18f8723.asm
                 LATCbits   0x000f8b       data     extern E:\MPASM_MPLINK_PIC18_LT_Branch_3_42\pic18-lt\cxx-framework\src\traditional\proc\p18f8723.asm
                     LATC   0x000f8b       data     extern E:\MPASM_MPLINK_PIC18_LT_Branch_3_42\pic18-lt\cxx-framework\src\traditional\proc\p18f8723.asm
                     LATD   0x000f8c       data     extern E:\MPASM_MPLINK_PIC18_LT_Branch_3_42\pic18-lt\cxx-framework\src\traditional\proc\p18f8723.asm
                 LATDbits   0x000f8c       data     extern E:\MPASM_MPLINK_PIC18_LT_Branch_3_42\pic18-lt\cxx-framework\src\traditional\proc\p18f8723.asm
                     LATE   0x000f8d       data     extern E:\MPASM_MPLINK_PIC18_LT_Branch_3_42\pic18-lt\cxx-framework\src\traditional\proc\p18f8723.asm
                 LATEbits   0x000f8d       data     extern E:\MPASM_MPLINK_PIC18_LT_Branch_3_42\pic18-lt\cxx-framework\src\traditional\proc\p18f8723.asm
                 LATFbits   0x000f8e       data     extern E:\MPASM_MPLINK_PIC18_LT_Branch_3_42\pic18-lt\cxx-framework\src\traditional\proc\p18f8723.asm
                     LATF   0x000f8e       data     extern E:\MPASM_MPLINK_PIC18_LT_Branch_3_42\pic18-lt\cxx-framework\src\traditional\proc\p18f8723.asm
                 LATGbits   0x000f8f       data     extern E:\MPASM_MPLINK_PIC18_LT_Branch_3_42\pic18-lt\cxx-framework\src\traditional\proc\p18f8723.asm
                     LATG   0x000f8f       data     extern E:\MPASM_MPLINK_PIC18_LT_Branch_3_42\pic18-lt\cxx-framework\src\traditional\proc\p18f8723.asm
                     LATH   0x000f90       data     extern E:\MPASM_MPLINK_PIC18_LT_Branch_3_42\pic18-lt\cxx-framework\src\traditional\proc\p18f8723.asm
                 LATHbits   0x000f90       data     extern E:\MPASM_MPLINK_PIC18_LT_Branch_3_42\pic18-lt\cxx-framework\src\traditional\proc\p18f8723.asm
                     LATJ   0x000f91       data     extern E:\MPASM_MPLINK_PIC18_LT_Branch_3_42\pic18-lt\cxx-framework\src\traditional\proc\p18f8723.asm
                 LATJbits   0x000f91       data     extern E:\MPASM_MPLINK_PIC18_LT_Branch_3_42\pic18-lt\cxx-framework\src\traditional\proc\p18f8723.asm
                     DDRA   0x000f92       data     extern E:\MPASM_MPLINK_PIC18_LT_Branch_3_42\pic18-lt\cxx-framework\src\traditional\proc\p18f8723.asm
                 DDRAbits   0x000f92       data     extern E:\MPASM_MPLINK_PIC18_LT_Branch_3_42\pic18-lt\cxx-framework\src\traditional\proc\p18f8723.asm
                TRISAbits   0x000f92       data     extern E:\MPASM_MPLINK_PIC18_LT_Branch_3_42\pic18-lt\cxx-framework\src\traditional\proc\p18f8723.asm
                    TRISA   0x000f92       data     extern E:\MPASM_MPLINK_PIC18_LT_Branch_3_42\pic18-lt\cxx-framework\src\traditional\proc\p18f8723.asm
                     DDRB   0x000f93       data     extern E:\MPASM_MPLINK_PIC18_LT_Branch_3_42\pic18-lt\cxx-framework\src\traditional\proc\p18f8723.asm
                    TRISB   0x000f93       data     extern E:\MPASM_MPLINK_PIC18_LT_Branch_3_42\pic18-lt\cxx-framework\src\traditional\proc\p18f8723.asm
                TRISBbits   0x000f93       data     extern E:\MPASM_MPLINK_PIC18_LT_Branch_3_42\pic18-lt\cxx-framework\src\traditional\proc\p18f8723.asm
                 DDRBbits   0x000f93       data     extern E:\MPASM_MPLINK_PIC18_LT_Branch_3_42\pic18-lt\cxx-framework\src\traditional\proc\p18f8723.asm
                     DDRC   0x000f94       data     extern E:\MPASM_MPLINK_PIC18_LT_Branch_3_42\pic18-lt\cxx-framework\src\traditional\proc\p18f8723.asm
                    TRISC   0x000f94       data     extern E:\MPASM_MPLINK_PIC18_LT_Branch_3_42\pic18-lt\cxx-framework\src\traditional\proc\p18f8723.asm
                TRISCbits   0x000f94       data     extern E:\MPASM_MPLINK_PIC18_LT_Branch_3_42\pic18-lt\cxx-framework\src\traditional\proc\p18f8723.asm
                 DDRCbits   0x000f94       data     extern E:\MPASM_MPLINK_PIC18_LT_Branch_3_42\pic18-lt\cxx-framework\src\traditional\proc\p18f8723.asm
                 DDRDbits   0x000f95       data     extern E:\MPASM_MPLINK_PIC18_LT_Branch_3_42\pic18-lt\cxx-framework\src\traditional\proc\p18f8723.asm
                    TRISD   0x000f95       data     extern E:\MPASM_MPLINK_PIC18_LT_Branch_3_42\pic18-lt\cxx-framework\src\traditional\proc\p18f8723.asm
                TRISDbits   0x000f95       data     extern E:\MPASM_MPLINK_PIC18_LT_Branch_3_42\pic18-lt\cxx-framework\src\traditional\proc\p18f8723.asm
                     DDRD   0x000f95       data     extern E:\MPASM_MPLINK_PIC18_LT_Branch_3_42\pic18-lt\cxx-framework\src\traditional\proc\p18f8723.asm
                 DDREbits   0x000f96       data     extern E:\MPASM_MPLINK_PIC18_LT_Branch_3_42\pic18-lt\cxx-framework\src\traditional\proc\p18f8723.asm
                TRISEbits   0x000f96       data     extern E:\MPASM_MPLINK_PIC18_LT_Branch_3_42\pic18-lt\cxx-framework\src\traditional\proc\p18f8723.asm
                    TRISE   0x000f96       data     extern E:\MPASM_MPLINK_PIC18_LT_Branch_3_42\pic18-lt\cxx-framework\src\traditional\proc\p18f8723.asm
                     DDRE   0x000f96       data     extern E:\MPASM_MPLINK_PIC18_LT_Branch_3_42\pic18-lt\cxx-framework\src\traditional\proc\p18f8723.asm
                 DDRFbits   0x000f97       data     extern E:\MPASM_MPLINK_PIC18_LT_Branch_3_42\pic18-lt\cxx-framework\src\traditional\proc\p18f8723.asm
                     DDRF   0x000f97       data     extern E:\MPASM_MPLINK_PIC18_LT_Branch_3_42\pic18-lt\cxx-framework\src\traditional\proc\p18f8723.asm
                TRISFbits   0x000f97       data     extern E:\MPASM_MPLINK_PIC18_LT_Branch_3_42\pic18-lt\cxx-framework\src\traditional\proc\p18f8723.asm
                    TRISF   0x000f97       data     extern E:\MPASM_MPLINK_PIC18_LT_Branch_3_42\pic18-lt\cxx-framework\src\traditional\proc\p18f8723.asm
                TRISGbits   0x000f98       data     extern E:\MPASM_MPLINK_PIC18_LT_Branch_3_42\pic18-lt\cxx-framework\src\traditional\proc\p18f8723.asm
                    TRISG   0x000f98       data     extern E:\MPASM_MPLINK_PIC18_LT_Branch_3_42\pic18-lt\cxx-framework\src\traditional\proc\p18f8723.asm
                 DDRGbits   0x000f98       data     extern E:\MPASM_MPLINK_PIC18_LT_Branch_3_42\pic18-lt\cxx-framework\src\traditional\proc\p18f8723.asm
                     DDRG   0x000f98       data     extern E:\MPASM_MPLINK_PIC18_LT_Branch_3_42\pic18-lt\cxx-framework\src\traditional\proc\p18f8723.asm
                TRISHbits   0x000f99       data     extern E:\MPASM_MPLINK_PIC18_LT_Branch_3_42\pic18-lt\cxx-framework\src\traditional\proc\p18f8723.asm
                    TRISH   0x000f99       data     extern E:\MPASM_MPLINK_PIC18_LT_Branch_3_42\pic18-lt\cxx-framework\src\traditional\proc\p18f8723.asm
                 DDRHbits   0x000f99       data     extern E:\MPASM_MPLINK_PIC18_LT_Branch_3_42\pic18-lt\cxx-framework\src\traditional\proc\p18f8723.asm
                     DDRH   0x000f99       data     extern E:\MPASM_MPLINK_PIC18_LT_Branch_3_42\pic18-lt\cxx-framework\src\traditional\proc\p18f8723.asm
                     DDRJ   0x000f9a       data     extern E:\MPASM_MPLINK_PIC18_LT_Branch_3_42\pic18-lt\cxx-framework\src\traditional\proc\p18f8723.asm
                 DDRJbits   0x000f9a       data     extern E:\MPASM_MPLINK_PIC18_LT_Branch_3_42\pic18-lt\cxx-framework\src\traditional\proc\p18f8723.asm
                TRISJbits   0x000f9a       data     extern E:\MPASM_MPLINK_PIC18_LT_Branch_3_42\pic18-lt\cxx-framework\src\traditional\proc\p18f8723.asm
                    TRISJ   0x000f9a       data     extern E:\MPASM_MPLINK_PIC18_LT_Branch_3_42\pic18-lt\cxx-framework\src\traditional\proc\p18f8723.asm
              OSCTUNEbits   0x000f9b       data     extern E:\MPASM_MPLINK_PIC18_LT_Branch_3_42\pic18-lt\cxx-framework\src\traditional\proc\p18f8723.asm
                  OSCTUNE   0x000f9b       data     extern E:\MPASM_MPLINK_PIC18_LT_Branch_3_42\pic18-lt\cxx-framework\src\traditional\proc\p18f8723.asm
                   MEMCON   0x000f9c       data     extern E:\MPASM_MPLINK_PIC18_LT_Branch_3_42\pic18-lt\cxx-framework\src\traditional\proc\p18f8723.asm
               MEMCONbits   0x000f9c       data     extern E:\MPASM_MPLINK_PIC18_LT_Branch_3_42\pic18-lt\cxx-framework\src\traditional\proc\p18f8723.asm
                     PIE1   0x000f9d       data     extern E:\MPASM_MPLINK_PIC18_LT_Branch_3_42\pic18-lt\cxx-framework\src\traditional\proc\p18f8723.asm
                 PIE1bits   0x000f9d       data     extern E:\MPASM_MPLINK_PIC18_LT_Branch_3_42\pic18-lt\cxx-framework\src\traditional\proc\p18f8723.asm
                 PIR1bits   0x000f9e       data     extern E:\MPASM_MPLINK_PIC18_LT_Branch_3_42\pic18-lt\cxx-framework\src\traditional\proc\p18f8723.asm
                     PIR1   0x000f9e       data     extern E:\MPASM_MPLINK_PIC18_LT_Branch_3_42\pic18-lt\cxx-framework\src\traditional\proc\p18f8723.asm
                 IPR1bits   0x000f9f       data     extern E:\MPASM_MPLINK_PIC18_LT_Branch_3_42\pic18-lt\cxx-framework\src\traditional\proc\p18f8723.asm
                     IPR1   0x000f9f       data     extern E:\MPASM_MPLINK_PIC18_LT_Branch_3_42\pic18-lt\cxx-framework\src\traditional\proc\p18f8723.asm
                 PIE2bits   0x000fa0       data     extern E:\MPASM_MPLINK_PIC18_LT_Branch_3_42\pic18-lt\cxx-framework\src\traditional\proc\p18f8723.asm
                     PIE2   0x000fa0       data     extern E:\MPASM_MPLINK_PIC18_LT_Branch_3_42\pic18-lt\cxx-framework\src\traditional\proc\p18f8723.asm
                 PIR2bits   0x000fa1       data     extern E:\MPASM_MPLINK_PIC18_LT_Branch_3_42\pic18-lt\cxx-framework\src\traditional\proc\p18f8723.asm
                     PIR2   0x000fa1       data     extern E:\MPASM_MPLINK_PIC18_LT_Branch_3_42\pic18-lt\cxx-framework\src\traditional\proc\p18f8723.asm
                 IPR2bits   0x000fa2       data     extern E:\MPASM_MPLINK_PIC18_LT_Branch_3_42\pic18-lt\cxx-framework\src\traditional\proc\p18f8723.asm
                     IPR2   0x000fa2       data     extern E:\MPASM_MPLINK_PIC18_LT_Branch_3_42\pic18-lt\cxx-framework\src\traditional\proc\p18f8723.asm
                 PIE3bits   0x000fa3       data     extern E:\MPASM_MPLINK_PIC18_LT_Branch_3_42\pic18-lt\cxx-framework\src\traditional\proc\p18f8723.asm
                     PIE3   0x000fa3       data     extern E:\MPASM_MPLINK_PIC18_LT_Branch_3_42\pic18-lt\cxx-framework\src\traditional\proc\p18f8723.asm
                     PIR3   0x000fa4       data     extern E:\MPASM_MPLINK_PIC18_LT_Branch_3_42\pic18-lt\cxx-framework\src\traditional\proc\p18f8723.asm
                 PIR3bits   0x000fa4       data     extern E:\MPASM_MPLINK_PIC18_LT_Branch_3_42\pic18-lt\cxx-framework\src\traditional\proc\p18f8723.asm
                 IPR3bits   0x000fa5       data     extern E:\MPASM_MPLINK_PIC18_LT_Branch_3_42\pic18-lt\cxx-framework\src\traditional\proc\p18f8723.asm
                     IPR3   0x000fa5       data     extern E:\MPASM_MPLINK_PIC18_LT_Branch_3_42\pic18-lt\cxx-framework\src\traditional\proc\p18f8723.asm
               EECON1bits   0x000fa6       data     extern E:\MPASM_MPLINK_PIC18_LT_Branch_3_42\pic18-lt\cxx-framework\src\traditional\proc\p18f8723.asm
                   EECON1   0x000fa6       data     extern E:\MPASM_MPLINK_PIC18_LT_Branch_3_42\pic18-lt\cxx-framework\src\traditional\proc\p18f8723.asm
                   EECON2   0x000fa7       data     extern E:\MPASM_MPLINK_PIC18_LT_Branch_3_42\pic18-lt\cxx-framework\src\traditional\proc\p18f8723.asm
                   EEDATA   0x000fa8       data     extern E:\MPASM_MPLINK_PIC18_LT_Branch_3_42\pic18-lt\cxx-framework\src\traditional\proc\p18f8723.asm
                    EEADR   0x000fa9       data     extern E:\MPASM_MPLINK_PIC18_LT_Branch_3_42\pic18-lt\cxx-framework\src\traditional\proc\p18f8723.asm
                   EEADRH   0x000faa       data     extern E:\MPASM_MPLINK_PIC18_LT_Branch_3_42\pic18-lt\cxx-framework\src\traditional\proc\p18f8723.asm
                RCSTAbits   0x000fab       data     extern E:\MPASM_MPLINK_PIC18_LT_Branch_3_42\pic18-lt\cxx-framework\src\traditional\proc\p18f8723.asm
               RCSTA1bits   0x000fab       data     extern E:\MPASM_MPLINK_PIC18_LT_Branch_3_42\pic18-lt\cxx-framework\src\traditional\proc\p18f8723.asm
                   RCSTA1   0x000fab       data     extern E:\MPASM_MPLINK_PIC18_LT_Branch_3_42\pic18-lt\cxx-framework\src\traditional\proc\p18f8723.asm
                    RCSTA   0x000fab       data     extern E:\MPASM_MPLINK_PIC18_LT_Branch_3_42\pic18-lt\cxx-framework\src\traditional\proc\p18f8723.asm
                    TXSTA   0x000fac       data     extern E:\MPASM_MPLINK_PIC18_LT_Branch_3_42\pic18-lt\cxx-framework\src\traditional\proc\p18f8723.asm
                   TXSTA1   0x000fac       data     extern E:\MPASM_MPLINK_PIC18_LT_Branch_3_42\pic18-lt\cxx-framework\src\traditional\proc\p18f8723.asm
               TXSTA1bits   0x000fac       data     extern E:\MPASM_MPLINK_PIC18_LT_Branch_3_42\pic18-lt\cxx-framework\src\traditional\proc\p18f8723.asm
                TXSTAbits   0x000fac       data     extern E:\MPASM_MPLINK_PIC18_LT_Branch_3_42\pic18-lt\cxx-framework\src\traditional\proc\p18f8723.asm
                    TXREG   0x000fad       data     extern E:\MPASM_MPLINK_PIC18_LT_Branch_3_42\pic18-lt\cxx-framework\src\traditional\proc\p18f8723.asm
                   TXREG1   0x000fad       data     extern E:\MPASM_MPLINK_PIC18_LT_Branch_3_42\pic18-lt\cxx-framework\src\traditional\proc\p18f8723.asm
                   RCREG1   0x000fae       data     extern E:\MPASM_MPLINK_PIC18_LT_Branch_3_42\pic18-lt\cxx-framework\src\traditional\proc\p18f8723.asm
                    RCREG   0x000fae       data     extern E:\MPASM_MPLINK_PIC18_LT_Branch_3_42\pic18-lt\cxx-framework\src\traditional\proc\p18f8723.asm
                    SPBRG   0x000faf       data     extern E:\MPASM_MPLINK_PIC18_LT_Branch_3_42\pic18-lt\cxx-framework\src\traditional\proc\p18f8723.asm
                   SPBRG1   0x000faf       data     extern E:\MPASM_MPLINK_PIC18_LT_Branch_3_42\pic18-lt\cxx-framework\src\traditional\proc\p18f8723.asm
                   PSPCON   0x000fb0       data     extern E:\MPASM_MPLINK_PIC18_LT_Branch_3_42\pic18-lt\cxx-framework\src\traditional\proc\p18f8723.asm
               PSPCONbits   0x000fb0       data     extern E:\MPASM_MPLINK_PIC18_LT_Branch_3_42\pic18-lt\cxx-framework\src\traditional\proc\p18f8723.asm
                    T3CON   0x000fb1       data     extern E:\MPASM_MPLINK_PIC18_LT_Branch_3_42\pic18-lt\cxx-framework\src\traditional\proc\p18f8723.asm
                T3CONbits   0x000fb1       data     extern E:\MPASM_MPLINK_PIC18_LT_Branch_3_42\pic18-lt\cxx-framework\src\traditional\proc\p18f8723.asm
                    TMR3L   0x000fb2       data     extern E:\MPASM_MPLINK_PIC18_LT_Branch_3_42\pic18-lt\cxx-framework\src\traditional\proc\p18f8723.asm
                    TMR3H   0x000fb3       data     extern E:\MPASM_MPLINK_PIC18_LT_Branch_3_42\pic18-lt\cxx-framework\src\traditional\proc\p18f8723.asm
                CMCONbits   0x000fb4       data     extern E:\MPASM_MPLINK_PIC18_LT_Branch_3_42\pic18-lt\cxx-framework\src\traditional\proc\p18f8723.asm
                    CMCON   0x000fb4       data     extern E:\MPASM_MPLINK_PIC18_LT_Branch_3_42\pic18-lt\cxx-framework\src\traditional\proc\p18f8723.asm
                   CVRCON   0x000fb5       data     extern E:\MPASM_MPLINK_PIC18_LT_Branch_3_42\pic18-lt\cxx-framework\src\traditional\proc\p18f8723.asm
               CVRCONbits   0x000fb5       data     extern E:\MPASM_MPLINK_PIC18_LT_Branch_3_42\pic18-lt\cxx-framework\src\traditional\proc\p18f8723.asm
              ECCP1ASbits   0x000fb6       data     extern E:\MPASM_MPLINK_PIC18_LT_Branch_3_42\pic18-lt\cxx-framework\src\traditional\proc\p18f8723.asm
                  ECCP1AS   0x000fb6       data     extern E:\MPASM_MPLINK_PIC18_LT_Branch_3_42\pic18-lt\cxx-framework\src\traditional\proc\p18f8723.asm
             ECCP3CONbits   0x000fb7       data     extern E:\MPASM_MPLINK_PIC18_LT_Branch_3_42\pic18-lt\cxx-framework\src\traditional\proc\p18f8723.asm
                 ECCP3CON   0x000fb7       data     extern E:\MPASM_MPLINK_PIC18_LT_Branch_3_42\pic18-lt\cxx-framework\src\traditional\proc\p18f8723.asm
              CCP3CONbits   0x000fb7       data     extern E:\MPASM_MPLINK_PIC18_LT_Branch_3_42\pic18-lt\cxx-framework\src\traditional\proc\p18f8723.asm
                  CCP3CON   0x000fb7       data     extern E:\MPASM_MPLINK_PIC18_LT_Branch_3_42\pic18-lt\cxx-framework\src\traditional\proc\p18f8723.asm
                   CCPR3L   0x000fb8       data     extern E:\MPASM_MPLINK_PIC18_LT_Branch_3_42\pic18-lt\cxx-framework\src\traditional\proc\p18f8723.asm
